:100000000C94EC120C940B130C940B130C940B1318
:100010000C94FF2A0C940B130C940B130C940A2CC5
:100020000C940B130C940B130C940B130C940B13D8
:100030000C940B130C940B130C940B130C940B13C8
:100040000C940B130C940B130C940B130C940B13B8
:100050000C940B130C940B130C9450310C940B1345
:100060000C940B130C940B130C940B130C940B1398
:100070000C940B130C940B130C940B130C94692617
:100080000C940B130C940B130C940B130C940B1378
:100090000C940B130C940B130C940B130C940B1368
:1000A0000C940B135645523A3234303632350082B6
:1000B000164618131860184C157B182F140518379E
:1000C00014D21487232B182F142F149024AD162F1D
:1000D000144618131860184C157B1899170518E862
:1000E00016D21487232B18A7142F149024AD162F83
:1000F000144618131860184C157B18651505183B25
:1001000015D21487232B18AD142F149024AD162F5D
:10011000144618131860184C157B18C71505183E9F
:1001200015D21487232B18F5172F149024AD1659C8
:10013000144618131860184C157B182F1405184214
:1001400015D21487232B18A9162F149024AD1659F5
:10015000144618131860184C157B189B140518DBEF
:1001600016D21487232B18AE182F149024AD1659CD
:10017000144618131860184C157B18A1140518178D
:1001800017D21487232B1839142F149024AD165925
:10019000142F142F142F144C152F1493182F144AA6
:1001A00014D21487232F142F142F1490242F142FBC
:1001B000144618131860184C157B182F1405185185
:1001C00016D21487232B184C162F149024AD162FFB
:1001D000144618131860184C157B18081505188359
:1001E00016D21487232B18B3142F149024AD162F76
:1001F000144618131860184C157B1810150518872D
:1002000016D21487232B182F142F149024AD162FD9
:10021000144618131860184C157B18151505181876
:1002200013D21487232B1869172F149024AD162F7F
:10023000144618131860184C157B182F1405180D48
:1002400013D21487232B188B162F149024AD162F3E
:10025000144618131860184C157B18DD140518A3E4
:1002600018D21487232B18D0182F149024AD162FD2
:10027000144618131860184C157B18E91405185EFD
:1002800017D21487232B18DA172F149024AD162FAA
:1002900014DA14BB175C164C152115F4142D153007
:1002A00014D21487232F14C4142F1490242F149CB9
:1002B000ACCCB6F400C111214191A131B171F19CD6
:1002C000ACCCB6F4367491A1C111214131F1710663
:1002D0000709FF001210070FFF000F0506FF0010AF
:1002E0000A0B0811FF000E0F090DFF00050C0E0A86
:1002F00005FF00C0C1C2FFC4C5C618808182C38487
:100300008586877071728374757677303132733475
:1003100035363710111213141516170304050A0881
:10032000060BFF0209070D010C00FF53554E4D4F00
:100330004E545545574544544855465249534154E7
:10034000004A414E4645424D41524150524D41595D
:100350004A554E4A554C4155475345504F43544ECC
:100360004F564445430000030205000305010406FF
:10037000020480002C0F870C082A0CD5557CEBFF5B
:100380000C00000CFFFF0CFFFFFC83F80C0F810C2E
:10039000081F0CD5FF5C83FC2C0FAF0C0A0A0CD590
:1003A000F57CFE03FCE1C3FC00000CFFD7FC003C25
:1003B0002C0C3F0C0C2A0C5F557C80002C0F0F0C72
:1003C0000F0A0C5FD57C0FFFFC0F800C081FFC553B
:1003D000FFFC80A02C0F0F0C0A0A0CD5F57C802C9A
:1003E0002C0F0F0C0A0A0CD5557CFFFFFCFAFAFC07
:1003F000F5F5FCFFFFFCFFFFFCFAFAECF5F57CFFDE
:10040000FFFCFF8BFCF874BCC7FF4CFFFFFCFAFA43
:10041000FCF0F0FCF0F0FCFFFFFCEFFFECD2FE1C68
:10042000FD21FCFFDFFC83FFFC0F830C0A1FFCD5C2
:10043000FFFCFFFFFCFFFFFCFFFFFCFFFFFCE000F9
:100440000C07C3FC4282ACF5555C00000C0F0F0C8E
:100450000A0A0CD5F57C80002C07FD0C0BFE0CD78E
:10046000FD7C00000C0FFF0C42A81CF555FC0000A1
:100470000C0F0F0C0F5F0C5FFF5C00000C0F0FFCEC
:100480000F5FFC5FFFFC80002C0FFF0C0FC20CDF26
:10049000D57C00000CFF0FFCAA0AAC55555C0FFF81
:1004A0000C00000C0FFF0CFFFFFCAFFC2C0FFF0C2F
:1004B00000001C5FFFFC00000CFF0FFCA0F0AC5F15
:1004C000FF5C00000CFFFF0CFFFF0CFFFF5C000057
:1004D0000CD2FFFC82AAAC55555C40000CF4BFFC6A
:1004E000AA0AAC55555C80002C0FFF0C0AAA0CD54B
:1004F000557C00000C0F0FFC0A0FFCD57FFC800020
:100500002C0FEB0C0AA00CD5557C00000C0F0BFC3B
:100510000A042CD57F5C802F2C0F0F0C0F0A0CDFE8
:10052000D57C0FFFFC00000C0FFFFCFFFFFC000060
:100530002CFFFF0CAAAA0C55557C0002FCFFFD2CD9
:10054000AAA87C5557FC00001CFFE1FCAAA0BC55E2
:10055000555C0AFA0CF505FCA050AC5FFF5C00AFDF
:10056000FCFF000C005FFCFFFFFC0FF80C0F870C7A
:10057000087F0C57FF5CAAAAAC05550C0FFF0CFFB7
:10058000FFFC4BFFFCF52FFCFFD4BCFFFF5CAFFF73
:10059000AC0FFF0C00000CFFFFFCFF0FFCFF0FFC7B
:1005A000FF0FFCFF5FFCFFFF0CFFFF0CFFFF0CFFCA
:1005B000FF5C00000C3FFFCC3FFFCC3FFFCC3FFF78
:1005C000CC3FFFCC3FFFCC2AAA8C54015C00000C2E
:1005D0003AAACC3555CC3FFFCC3FFFCC3FFFCC3FB8
:1005E000FFCC2AAA8C54015C00000C3AAACC3555E9
:1005F000CC3000CC3FFFCC3FFFCC3FFFCC2AAA8CB5
:1006000054015C00000C3AAACC3555CC3000CC3AF1
:10061000AACC3555CC3FFFCC2AAA8C54015C0000F3
:100620000C3AAACC3555CC3000CC3AAACC3555CCB6
:100630003000CC2AAA8C54015C00000000000000AD
:1006400000000000000000003FFF3C000000000030
:10065000003FC0000000001540002A800017D7D4DA
:100660002BEBE83FFFFC02828007F4D01F7DF40FE4
:100670003DF0020A803C0078001E8007A01428008C
:10068000281FCFF43C343C3DCAF80A0208000000A1
:100690001440002A000000000007FFD03E00BC20EC
:1006A000000800000034001C2F55F802AA8000004A
:1006B00000024C60017F50006E40020820003C00A8
:1006C00003FFC0003C000000000000000003D80051
:1006D0000000000000003C00003C00003C0000283E
:1006E000000000000000F0000000000000000078A2
:1006F000001E8007A0002800001FFFF43C1E3C3DA8
:10070000F57C0AAAA005003C3FFFFC00003C00006D
:10071000001F01FC3C1FBC3DF83C0A80281F00F470
:100720003C143C3D7D7C0A82A0007F00078F003F87
:10073000FFFC000A003FF0F43CF03C3CF57C282A2A
:10074000A01FFFF43C3C3C3C3D7C280AA03C000040
:100750003C1FFC3DF8002A80001FD7F43C3C3C3D88
:100760007D7C0A82A01FF4F43C3C3C3D7D7C0AAABF
:10077000A000000001414002828000000000000053
:100780000141440282A0000000001D0001E2D00EE1
:10079000002C00000001414003C3C003C3C000009F
:1007A000000400040B407800B7800008001F000020
:1007B0003C1F3C3D78000A800006AAA431AA4C24C4
:1007C000AA4C02AA0007FFFC3E0F002F5F5402AAAA
:1007D000A83FFFFC3C3C3C3D7D7C0A82A01FFFF40F
:1007E0003E00BC3D007C0A00A03FFFFC3C003C2FCB
:1007F00055F802AA803FFFFC3C3C3C3C283C2800CA
:10080000283FFFFC3C3C003C28002800001FFFF470
:100810003C003C3C0F7C080AA03FFFFC003C00155C
:100820007D542AAAA83C003C3FFFFC3C003C000051
:10083000001400F43C003C3FFFF82800003FFFFCA0
:10084000003C0017C3D42800283FFFFC00003C00F8
:10085000003C0000283FFFFC0B40001F55542AAA13
:10086000A82FFFFC02D000157D542AAAA81FFFF470
:100870003C003C3D557C0AAAA03FFFFC3C3C003DAF
:100880007C000AA0001FFFF43C053C3D57FC0AAA6F
:10089000A03FFFFC3C3D003D7EF40AA0281FF4343D
:1008A0003C3C3C3C3D7C080AA03C00003FFFFC3C3B
:1008B00000000000003FFFF400003C15557C2AAA10
:1008C000A03FFF400000B41555E02AAA003FFFF802
:1008D0000007801557D02AAAA83D417C02BE801788
:1008E000EBD42800283FD400003FFC3FE800000084
:1008F000003C01FC3C1E3C3DE03C2A0028155554C0
:100900003EAABC3C003C0000002D000002B40000E8
:100910000AD00000281400143C003C3FFFFC0000FB
:100920000001E0001E00000B400000A00000003CA1
:1009300000003C00003C0000282D000002D0000018
:1009400000000000000051F400F33C00F774002A9E
:10095000A83FFFFC00F03C00F57C002AA0007FF4DB
:1009600000F03C00F03C002020007FF400FC3C152F
:100970007D7C2AAAA8007FF400F33C00F73C002A03
:1009800020057D543EBEA83D28000A0000007D14CD
:1009900000F33C00F77C002AA03FFFFC0078000039
:1009A000F554002AA80050003CFFFC0000000000A5
:1009B000000000F401403CF3FFF80000000FFFFCD2
:1009C0000007D000382C0000081400003FFFFC0096
:1009D000000000000000FFFC002D00007D5400AA74
:1009E000A800BFFC00F80000BD54002AA8007FF456
:1009F00000F03C00F57C002AA003FFFC01E2D003DC
:100A0000D5F000AA8001FFD003C0F001F7D402AAFC
:100A1000A800FFFC00780000F400002800007D3CE6
:100A200000F33C00F37C00A0A015F5502AFABC00AE
:100A3000007C0000A000FFF400003C00557C00AAF0
:100A4000A000FF400000B40055E000AA0000FFFC39
:100A50000001E00055F400AAA800F47C002BA000DF
:100A60007EF400A02803FD14000F3C015F7C02AA65
:100A7000A000F07C00F3BC00FE3C00A028007D003C
:100A80001F82F42000080000000000000000005554
:100A9000555500000035005C0AD7A0002800000072
:100AA00000001E00002D00001E00002800007D0038
:100AB00002BE80003C00002800005FFF07A0057810
:100AC00007FEF03E00F03FFFBD2AAA0AF555FFD40D
:100AD00000502B40BFC2F007C0BCFF007CABC0A0E1
:100AE0005F80001FFFFFFFFFFFFF800FFF000FFF72
:100AF000400FFFFFFF2FFFFFFFFFFCFFFFFCF00099
:100B000000F00000F00000FFFFFCFFFFFCFFFFFF14
:100B1000FFFFFFFF003FFF003FFF407FFFFFFF2F72
:100B2000FFE0FFFFFCFFFFFCC003FCC003FCD0079D
:100B3000FCFFFFFCBFFFE01FFFFFFFFFFFFF800088
:100B4000FF0000FF4000FFF0002FF000FFFFD0FF8C
:100B5000FFFC000BFC0003FC0007FC00FFFC00FF97
:100B6000E0FFFFFFFFFFFFFF0000FF0000FF40006E
:100B70003FFFFF0AFFFFFFFFFCFFFFFC0003FC003D
:100B800003FC0007FCFFFFF0FFFE80FFFFFFFFFFFD
:100B9000FFFF003FFF003FFF003FFF0000FF00009E
:100BA000FFFFFCFFFFFCC003FCC003FCC003FC0014
:100BB00003FC0003FCFFFFFFFFFFFFFF003FFF0000
:100BC0003FFF002AFF0000FF0000FFFFFCFFFFFCCB
:100BD000C00000C000008000000000000000001FF6
:100BE000FFFFFFFFFFFF8000FF0000FF4000FFF05E
:100BF000002FF000FFFFD0FFFFFC000BFC0003FC08
:100C0000FF07FCFFFFFCFFFFE0FFFFFFFFFFFF0010
:100C1000003F00003F00003FFFFFFFFFFFFFFFFF1F
:100C2000FCFFFFFCC00000C00000C00000FFFFFC94
:100C3000FFFFFCFF0000FF0000FF5555FFFFFFFF17
:100C4000AAAAFF0000FF00000003FC0003FC5557A8
:100C5000FCFFFFFCAAABFC0003FC0003FC0000004F
:100C6000000000FF0000FF0000FFFFFFFFFFFFFF8D
:100C7000000000FFD000FFFC000BFC0007FCFFFFA2
:100C8000FCFFFFE0000000FFFFFFFFFFFF00003F51
:100C90000001FF001FF8FFFF80FFF800FFFFFCFFCF
:100CA000FFFCD00000FD0000BFD0000BFFFC00BF28
:100CB000FCFFFFFFFFFFFF0000000000000000003E
:100CC000000000000000FFFFFCFFFFFC0003FC0031
:100CD00003FC0003FC0003FC0003FCFFFFFFFFFF1D
:100CE000FF0AFF50000FFF05FFA0FFFFFFFFFFFF00
:100CF000FFFFFCFFFFFC000000000000000000FF01
:100D0000FFFCFFFFFCFFFFFFFFFFFF2BFF50002B4F
:100D1000FF00002BFFFFFFFFFFFFFFFFFCFFFFFCBB
:100D2000000000500000FF5000FFFFFCFFFFFC1F11
:100D3000FFFFFFFFFFFF8000FF0000FF4000FFFFFD
:100D4000FF2FFFFFFFFFD0FFFFFC000BFC0003FCA9
:100D50000007FCFFFFFCFFFFE0FFFFFFFFFFFFFFBF
:100D6000003FFF003FFF407FFFFFFF2FFFFEFFFF21
:100D7000FCFFFFFCC00000C00000C00000C000007D
:100D800000000017FFFF7FFFFFFF8000FF0000FF54
:100D90004000BFFFFF2BFFFFFFFF50FFFFF0000BE6
:100DA000FC0FF6FC0AFF6CFDBFF4FFDBFCFFFFFF4E
:100DB000FFFFFFFF003FFF003FFF407FFFFFFF2FD0
:100DC000FFFEFFFFFCFFFFFCFF0000FFD000EFFD78
:100DD00000C2FFFC002FFC17FFF57FFFFFFF80BF65
:100DE000FF003FFF403FBFF02F2BF00A003F504075
:100DF0003FF4C00BFCC003FCD007FCFFFFF8FFFF73
:100E0000A0FF0000FF0000FF5555FFFFFFFFAAAA4B
:100E1000FF0000FF0000000000000000555554FFD7
:100E2000FFFCAAAAA8000000000000FFFFFFFFFFD0
:100E3000FF000000000000000000FFFFFFFFFFFFB9
:100E4000FFFF50FFFFF4000BFC0003FC0007FCFF5A
:100E5000FFF8FFFFA0FFFFFFFFFFFF000000000003
:100E600000000000FFFFFFFFFFFFFFD000FFFD00BD
:100E700000BFD0000FFC007FE0FFFE00FFE000FF9E
:100E8000FFFFFFFFFF000000000000000000FFFF69
:100E9000FFFFFFFFFFFFFCFFFFFC017FA03FF00013
:100EA00002BF50FFFFFCFFFFFCFF5000FFFF5000A0
:100EB000AFFF00003F005FFFFFFFA0FFA000001793
:100EC000FC17FFFCFFE800F00000FFD4002BFFFC44
:100ED000002BFCFFFFD0FFFFFD0000BF00000F0054
:100EE000007FFFFFFEFFFFE0000000000000D5557F
:100EF00054FFFFFCEAAAA8000000000000FF000069
:100F0000FF0000FF0007FF007FFF07FFFFFFFEFF5E
:100F1000FFE007FFFC7FFFFCFFE3FCFE03FCE003B8
:100F2000FC0003FC0003FCFFFFFFFFFFFFFF0000CE
:100F3000FF0000FF0000FF0000FF0000FFFFFCFFBC
:100F4000FFFC0003FC0003FC0003FC0003FC0003A7
:100F5000FC1400003FD4002BFFD4002BFF00002B1B
:100F6000000000000000000000000000000000D4AD
:100F70000000FFD4002BFFC0002BC0FF0000FF00CB
:100F800000FF0000FF0000FF0000FFFFFFFFFFFF6A
:100F90000003FC0003FC0003FC0003FC0003FCFF57
:100FA000FFFCFFFFFC001F0001FF001FFFFFFFFF12
:100FB000FF2FFFFF02FF00002F00000000000000D5
:100FC000FFFFFCFFFFFCFFFFFC0000000000000033
:100FD0000000000000000000000000000000000011
:100FE000000000000003FC0003FC0003FC0003FC05
:100FF0000003FC0003FC0003FC00000000000000F4
:1010000000000000000000000000000000000000E0
:1010100000000000000000000000000000000000D0
:10102000000000000000000000555555FFFFFFAA1A
:10103000AAAA0000000000000000000000005541C6
:1010400054FFC3FCAA82A800000000000055550010
:10105000FFFF00AAAA00000000000000FFFF00FF41
:10106000FF00000000000000000000000000000081
:1010700000000000000000000FF00FFFFF0FFFFF57
:10108000000FF00FFFFF0FFFFF000FF03FC000FF4A
:10109000FFC0FFFFC03FC000FFFFC0FFFFC03FC059
:1010A0000000555407FFFF0FE02FFFFFFFAFEAAF2F
:1010B0000FF40F02FC0200540040FF40C02FC0FF9D
:1010C000FFFCEAAFE8F57FC0FFFE0001540003FC1F
:1010D0000002A80100017F017FFE3FFE803E8000EC
:1010E000000140017FC07FFE80FE80008000000381
:1010F000FC0003FC0000000101551F1FFFFF3E0321
:10110000FF3FDFE00AFA00000003FFFD40EAAFF016
:101110004002FCF500FCBFF5F802FFD0FFFAB0007A
:101120000000FFFF00FFFF000000000000000000C3
:1011300000000000000000000000000000000000AF
:101140000000000000000000000000000007FF0198
:10115000FFFF0FFA007E0000A80000000000000062
:1011600000FF4000FFFD0002BFC00002F40000A825
:10117000000000000000F400003F40000BFD55009F
:10118000BFFF0002AF00000000000000007C00076D
:10119000F055FF80FFF800EA0000000000003D0F5E
:1011A000000BDF0015FF003FFF002AFF0007EF00E4
:1011B0003E0FF07C00F7E000FF5400FFFC00FFA8AA
:1011C00000FBD000F0BC0000000F00000F00155F16
:1011D000003FFF002AAF00000F00000FF00000F0FA
:1011E0000000F55400FFFC00FAA800F00000F00039
:1011F0000000000700000F00000F00005B0007CF99
:1012000001FA0F00000B400000C00000C000009475
:101210000000CF4000C2BD008000000000050000BB
:101220000F00000F00000F00000F00000F00000F64
:10123000500000F00000F00000F00000F00000F0AE
:101240000000F0000000000702F50F000BCF0000C7
:10125000A700000F00000F00000B400000C17E003F
:10126000CF8000680000C00000C0000080000000C7
:10127000000000000000000100017F017FFE3FFE32
:10128000803E8000000140017FC07FFE80FE800024
:1012900080000000000000000017FFFF7FFFFFFF3D
:1012A0008001FF001FFF41FFBFFFFF2BFFFFFFFF7C
:1012B00050FFFFF4FF8BFCF803FC8007FCFFFFF8F6
:1012C000FFFFA000000007FC007FFD55FFFFFFAA05
:1012D000AAAA0000000000000003FC0003FC555710
:1012E000FCFFFFFCAAABFC0003FC0003FC1FF000AA
:1012F0007FF000FF8000FF0001FF401FFFFFFF2F76
:10130000FFF8001FFC01FFFC1FFBFCFF83FCF80340
:10131000FC8003FC0003FC1FF000FFF000FF8000D6
:10132000FF003FFF407FFFFFFF2FFFE0003FD000A7
:101330003FFC000BFCC003FCD007FCFFFFFCBFFF21
:10134000E000007F0007FF007FF807FF807FFD556A
:10135000FFFFFFAAAAAAFF0000FF0000FF0000FF96
:101360000000FF5554FFFFFCFFAAA8FFFFFDFFFF91
:10137000FFFF00FFFF00FFFF00FFFF00FFFF002F48
:10138000003FD0003FFC000BFC0003FC4007FCFFCB
:10139000FFFCFFFFE01FFFFFFFFFFFFF807FFF005D
:1013A000FFFF00FFFF00FFAA002FFFFFD0FFFFFCA1
:1013B000800BFC0003FC4007FCFFFFFCFFFFE05537
:1013C0000000FF0000FF0000FF0001FF001FFFFF03
:1013D000FFFFFFF8000000000000155554FFFFFC60
:1013E000FAAAA88000000000001FFFD0FFFFFFFF47
:1013F00080BFFF003FFF407FFFFFFF2FFFE27FFF27
:10140000D0FFFFFCE00BFCC003FCD007FCFFFFFC9F
:10141000FFFFE01FFFF5FFFFFFFF80BFFF003FFF63
:10142000407FFFFFFF2FFFFF003FD0403FFCC00B7E
:10143000FCC003FCC007FCFFFFFCFFFFE06FFFF9EF
:10144000F6AA8FFCAF4FFC555BFC054FFCAA0FE7DB
:10145000FFDBBFFFE4CAAA7CC7E8FC9554FCC5408B
:10146000FCC2A8FC9FFF6C00000700000F00000FEB
:1014700000000B000000000000000000400000C061
:101480001500C7E8009E00000000000000000000FA
:101490000000000700007F0007F8007F8007F800C9
:1014A0003F8000380000400000F40000BF40000B07
:1014B000F40000BF40000BF00000B0000FF0000F80
:1014C000F0000FF0000FF0000FF0000FF0000FF031
:1014D0000FF0000FF0000FF0000FF0000FF0000F02
:1014E000F0000FF0003400003F40000BF40000BF9C
:1014F00040000BF40000BF00000B0000700007F07C
:10150000007F8007F8007F8000F80000800000174F
:10151000FC007FFC00FF8001FF001FFF41FFBFFFB9
:10152000F82BFF80000000000000555154FFF3FC31
:10153000AAA2A80000000000002FFFF902AA8F0055
:10154000000F00000B000000000000000000BFFFC3
:10155000E0CAAA00C00000800000000000000000F7
:10156000000000000000003FC0003FC0003FC0007E
:101570003FD0003FFF000BFF1FFFD0FFFFFCFF8BA2
:10158000FCFF03FCFF03F8FFFFFCFFFFFC0FFFFF66
:101590000FFFFF00001F00003F00003F00003F0062
:1015A000000BFFFFFCFFFFFCF80BFCC003FCD007A7
:1015B000FCFFFFFCFFFFE000007F0003FF0003FED5
:1015C0000003FC0003FD0003FF0000BFFFFFD0FF8E
:1015D000FFFC000BFC0003FC0007FC000FFC000FED
:1015E000E000000100001F00003F00003F00002F4E
:1015F0000FFFFF0FFFFFFFFFD0FFFFFCE00BFCC062
:1016000003FCD007FCFFFFFCFFFFFC00007F000392
:10161000FF0003FE0003FC0003FD0003FF0000BF0A
:10162000FFFFD0FFFFFC3FCBFC3FC3FC3FC3FCFFF1
:10163000C3FCFFC3FC400000F40000FC0000FC0001
:1016400000FC0000FC0000E00000000000000000C2
:10165000000000000000000000000000000000404A
:101660000000F40000FC0000FDFFF4FCAAA0FC0058
:1016700000E000000000000000000000000000008A
:10168000000000000000000000400000F40000FC2A
:101690000000FDFFFDFCAAA8FC0000E00000000027
:1016A0000000150007E800AA00000000000000008C
:1016B000000000400000F40000FC0000FDFFFDFC05
:1016C000AAA8FC0000E0000000000000150007E8E8
:1016D00000AA0000AF400002BD0000000040000171
:1016E000F4000FFC000FFDFFF7FCAAA0FC0000E0D7
:1016F0000000000000C01500C7E8002A0000AF404D
:101700000002BD00000000400001F4000FFC000FCB
:10171000FDFFF7FCAAA7FC000FE0000B000000C0D3
:101720001500C7E8002A00006F4000C2BD0080001D
:101730000000001500003F00000000000500000F41
:10174000000000000000555550FFFEA000BF0055EE
:101750005F00FFFF00001600000000000FF0000F08
:10176000F0000FF0000FF5000FFF15FFF03FAFF096
:101770000FF5FC0FFFA85FF000FFF0000FF0000F67
:10178000F0000FF000FD4000FFFD40FC2BFDFC00D1
:101790002FFD0002FFC000FFC0000005FC05FFFC9C
:1017A000FFA0FCE000FC0001FC000FFC000FFC00AF
:1017B00000000000000000000000070001FE007FA4
:1017C000800FE0000001FC007FFC1FE0FCFF00FC3C
:1017D0000BD0FC00BFFC0000FC00000100000F006B
:1017E000003F00003F00003F00003F00003EF001CE
:1017F000F0C17FF0DFFA00E00550DFFFF0EA03F010
:10180000000A0000000500007F0003FF0003F8004D
:1018100003FD0001FF0003FAFFFF40FFFFF0A00FF0
:10182000F0001FE057FF50FFFFF0AA03F017FFFF83
:101830003FEAAAFE0054FC00FCFF01FD3FFFFF0B46
:10184000FE8FFFFFFFABFEAA00FF0000FF0001FFBD
:1018500000FFFE00FFF80000000114001FFC007FE5
:10186000FC00FCFD403F3FFFFF0ABFFF5FF500FFAC
:10187000FFF08002FC0003F8517FE0FFFE00EA80E9
:1018800000001FD401FFFD07F82F0FF00F0FF00F1E
:101890000FF00A02FC001FFD00FFFFD0F00BF4E088
:1018A00003FCC003FC8003FC000FF00000150000E7
:1018B0003F07FFFF3FFFFFFE003FFC002ABF000085
:1018C0000003FC015FFCFFFFFCFEA3FC0003FC0027
:1018D00003FC0003FC0000FC005FFF0FFEFE3F80E6
:1018E000FCFE00FCFD00FC3F4000FC0000FFD400BB
:1018F000FEFFC0FC0BF0FC02FCFC01FC0007E0005A
:1019000000140001F80013F007F3C0FE83F0A002FA
:10191000FF00000A0155001FFFD07E02FCFC00FC06
:10192000FC07E0FFFFFCAAAAA800001F0001FE01BF
:1019300073F05FE3F0F803F50000BF00000AFFFF5B
:1019400040FEAFF4FC02FCFC00FCFC01FCFC03F0DC
:10195000A800000000500000F0007CF51FE0FF3EF2
:1019600000000000000000000000FC0000FC5555D5
:10197000FCFFFFFC0000FC0000FC00000000005F1A
:101980000001FE01F3F05FA3F0F802FF00002B005E
:101990000000FFFD40AAAFF40002FC0001FC555F0F
:1019A000F8FFFE800000000003FF0010AA45F000D1
:1019B0003F80002801FF0002AA000000FFFFD0AA1C
:1019C000ABFC0000FC0005F8FFFFFCAAAAA8000081
:1019D0000000000000000005FFFF3FFFFFFE0000C9
:1019E0003C000000000000001F00003FFFFFFFFF61
:1019F000FFE8000000000000000000001FE0003FC2
:101A0000C0003FD0000FF00003FC0003FC001FF0FB
:101A10007F8000FF0000FF00003FC0000FF0000FBC
:101A2000F0007F80000000FF07F0FF0F007E0BD367
:101A3000F007F3FD0F80FF00002FFFFFFCFFFFFC0E
:101A4000000000000000000000FFFFFCFFFFFC00A2
:101A500017FF01FFEA0FE8000FC0000FD40002FFDC
:101A6000D5002BFFFF50FCAFFDFC000BFC0000007D
:101A70000007FC5FFEFCFA80FC400000F40000FC64
:101A80000000FDFFF4FCAAA0FC0000E00000000044
:101A90000000000000000000000000000000000046
:101AA0000000000000000003FC0003FC0003FC0039
:101AB00003FD0003FF0000BF07FFD03FFFFC3F8B8B
:101AC000FC3F03FC3F03F8FFFFFCFFFFFC0FFFFFA1
:101AD0000FFFFF00001F00003F00003F00003F001D
:101AE000000BFFFFFCFFFFFCF80BFCC003FCD00762
:101AF000FCFFFFFCFFFFE000000700003F00003F8D
:101B000000003F00003F00003F00000BFFFFD0FF40
:101B1000FFFCE00BFCC003FCC003FCF00FFCF00F6B
:101B2000E000000100001F00003F00003F00002F08
:101B30000FFFFF0FFFFFFFFFD0FFFFFCE00BFCC01C
:101B400003FCD003FCFFFFFCFFFFFC0000010000D2
:101B50001F00003F00003F00003F00003F00000B5F
:101B6000555540FFFFF4EFEFFC0FC3FC4FC3FCFFE4
:101B7000C3FCFFC3FC000003007FFF03FFFF03FE65
:101B80000303FD0303FFC000BFC0FC0000FFFFFC18
:101B9000FFFFFCFC0000FC00000000000000000053
:101BA000007F0003FF0003FE0003FC0003FD0003B1
:101BB000FF0000BFFD03F4FFC3FF2FC0BF0FC03FF6
:101BC0001FC07FFFFFFFFFFFF803FFFF03FFFF00C2
:101BD000000700000F00000F00000F000002FFFFD1
:101BE000FCFFFFFCF80000F00000F40000FFFFFC29
:101BF000FFFFFC00000000000000001500FF3F0098
:101C0000FF3F000000000000000000000000400056
:101C100000FFFFFCFFFFFC000000000000000000D0
:101C200000000000000000000000001500FF3F0061
:101C3000FF3F0003F40003FF0000BF00003F40002F
:101C40007FFFFFFFFFFFF800FFFF00FFFF00000026
:101C500000000100003F00003E000000FFFFFCFF0D
:101C6000FFFC1FF400FEBF40E00BFC0000BC0000C6
:101C700000000000000000000000003FFF003FFFE8
:101C8000000000000000000000000000000000FF55
:101C9000FFFCFFFFFC000000000000000007000048
:101CA0003F00003F00000F00003F00003F00000B1E
:101CB000FFFFFCFAAAA8D40000FFC000E80000F56E
:101CC0005554FFFFFC00003F00003F00001F0000D4
:101CD0003F00003F00003F00000BFFFFFCFFFFFC48
:101CE000E00000C00000C00000FFFFFCFFFFFC00A0
:101CF000000700003F00003F00003F00003F0000E1
:101D00003F00000BFFFFD0FFFFFCE00BFCC003FC1B
:101D1000D007FCFFFFFCFFFFE0003FFF003FFF009C
:101D200007FE000FF0000FF4000FFF0002FFFFFF9F
:101D3000FCFFFFFC02FD0000FF0001FF00FFFF00B1
:101D4000FFF80000007F0007FF000FF8000FF00011
:101D50000BF4003FFF003FFFFFF400FFFF0002FF16
:101D60000000FF0001FE00FFFFFCFFFFFC00003F42
:101D700000003F00000700003F00003F00003F0060
:101D8000000BFFFFFCFFFFFCFE0000E00000D000A6
:101D900000FC0000FC000000001F0000FF0000FE2F
:101DA0000000FC0000FC0000FF0000BFFD0FD0FFA2
:101DB000CFFC2FC2FC0FC0FC0FD1FC0FFFFC02FFB9
:101DC000E000000301555703FFFF02AAAB00000328
:101DD000000000000000FC0000FD5540FFFFF4FE85
:101DE000ABFCFC01FC003FFC003FE000003F0000BA
:101DF0003F00000000000000000000003F00003F26
:101E0000FFFFD0FFFFFC000BFC0003FC0007FCFF02
:101E1000FFFCFFFFE000003F00003F00000000006B
:101E20000000000000003F00003FFFD000FFFD0069
:101E300002FFD0003FFC01FFE0FFFE00FFE00000DA
:101E4000003F00002A000000000000000000000029
:101E50001500003FFFFFD0AAAFFC0007FC03FFF016
:101E6000000BFC555FFCFFFFE000003F00002B0073
:101E7000000000000000000000001700003F4001CB
:101E8000FCF41FE8BFFE000FF0007FFD00F82FD428
:101E90008002FC00003F00003F0000000000000046
:101EA000001500003F00003FFD03F4FFC3FC2FC0FE
:101EB000BC1FC03CFF807CFFFFFCFFFFF800003F21
:101EC00000003F00003F00003F00003F00003F00D7
:101ED000003FC001FCC01FFCC1FFFCDFFFFCFFE3B3
:101EE000FCFE03FCE003FC00000000000301400FC7
:101EF0007FFFFFFEAAA8F00000A00000000000C0C5
:101F00000000F00140FFFFFD2AAABF00000F000003
:101F10000A000000000000555555FFFFFFAAAAAABD
:101F2000000000000000000000000000555554FFB4
:101F3000FFFCAAAAA8000000000000000000F000BA
:101F400000FC0000FFFFFD2BEAAF000003000002D1
:101F500000000000000F00001F1FFFFFFAABE8E0C9
:101F60000000800000FD4000FFFD40FC2BFDFC0058
:101F70002FFD0002FFC000FFC0000005FC05FFFCB4
:101F8000FFA0FCE000FC0001FC000FFC000FFC1FA8
:101F9000FFFFFFFFFFFF800FFF000FFF400FFFFF5E
:101FA000FF2FFFFFFFFFD0FFFFFCC00BFCC003FCB7
:101FB000C007FCFFFFFCFFFFE00000000000000086
:101FC0000000000000000000000000000000000011
:101FD000000000000001540003FC0002A8055000AE
:101FE0000FF0000AA000000550000FF0000AA0004A
:101FF0000000000000000000001547003FFE002A1E
:10200000A038000230F8703082A03D55573EBFF036
:102010003000003FFFF03FFFFF383F8030F81030C6
:1020200081F03D5FF5383FC230FAF030A0A03D5F4F
:10203000573FE03F3E1C3F3000003FFD7F3003C272
:1020400030C3F030C2A035F55738000230F0F03020
:10205000F0A035FD5730FFFF30F8003081FF355FCD
:10206000FF380A0230F0F030A0A03D5F573802C2BE
:1020700030F0F030A0A03D55573FFFFF3FAFAF3FDE
:102080005F5F3FFFFF3FFFFF3FAFAE3F5F573FFF49
:10209000FF3FF8BF3F874B3C7FF43FFFFF3FAFAFB1
:1020A0003F0F0F3F0F0F3FFFFF3EFFFE3D2FE13F72
:1020B000D21F3FFDFF383FFF30F83030A1FF3D5FBA
:1020C000FF3FFF823AAA0134BBFF3F5FFF3E0000A3
:1020D000307C3F34282A3F555530000030F0F03036
:1020E000A0A03D5F57380002307FD030BFE03D7F79
:1020F000D730000030FFF0342A813F555F300000B8
:1021000030F0F030F5F035FFF530000030F0FF3002
:10211000F5FF35FFFF38000230FFF030FC203DFDB9
:10212000573000003FF0FF3AA0AA35555530FFF078
:1021300030000030FFF03FFFFF3AFFC230FFF030C9
:10214000000135FFFF3000003FF0FF3A0F0A35FF76
:10215000F53000003FFFF03FFFF03FFFF53000009B
:102160003D2FFF382AAA3555553400003F4BFF3A22
:10217000A0AA35555538000230FFF030AAA03D55D1
:102180005730000030F0FF30A0FF3D57FF3800020D
:1021900030FEB030AA003D555730000030F0BF305F
:1021A000A0423D57F53802F230F0F030F0A03DFD8E
:1021B0005730FFFF30000030FFFF3FFFFF300002CD
:1021C0003FFFF03AAAA035555730002F3FFFD23AD3
:1021D000AA8735557F3000013FFE1F3AAA0B3555BF
:1021E0005530AFA03F505F3A050A35FFF5300AFF82
:1021F0003FF0003005FF3FFFFF30FF8030F87030C8
:1022000087F0357FF53AAAAA30555030FFF03FFFEE
:10221000FF34BFFF3F52FF3FFD4B3FFFF53AFFFA50
:1022200030FFF03000003FFFFF3F87FF387FFF3D6A
:102230002FFF3FD7FF3FFFFF3FFFFF3FFFFF3FFF66
:10224000FF07FFFD0F078F0F7D5F02AAA801400F58
:102250000FFFFF00000F00000007C07F0F07EF0F08
:102260007E0F02A00A07C03D0F050F0F5F5F02A09F
:10227000A8001FC001E3C00FFFFF00028001FFFFA5
:102280000F83C00BD7D500AAAA0FFFFF0F000F0BBB
:10229000D57E00AAA00FFFFF0F0F0F0F0A0F0A0035
:1022A0000A0FFFFF0F0F000F0A000A000007FFFDD3
:1022B0000F000F0F03DF0202A80FFFFF000F000542
:1022C0005F550AAAAA0F000F0FFFFF0F000F0000B3
:1022D000000FFFFF00000F00000F00000A0FFFFFBC
:1022E00002F50007F5550AAAAA0FFFFF0F0F000F0E
:1022F0005F0002A8000FFFFF0F0F400F5FBD02A895
:102300000A07FD0D0F0F0F0F0F5F0202A80F00004D
:102310000FFFFF0F00000000000FFFFD00000F0582
:10232000555F0AAAA8010101FF02EB0202D7680269
:10233000D10102C0F607C128282828140005C206CA
:1023400006060602CB0802B3940BB4E56685FFFFD0
:102350005285FFFF5202B03F03B20005011101FF99
:1023600003C7A6E9023620023A1102B8090120018A
:10237000FF02B9230138012900010101FF02EB022C
:1023800002D76802D10102C08007C128282828147A
:102390000005C20000000002CB1702B3940BB4A5E5
:1023A00066010000400100004002B03F03B2010599
:1023B000011101FF03C7A6E9023620023A1102B853
:1023C000090120012902B9E301FF02B92301390003
:1023D000010101FF02EB0202D76802D10102C080B5
:1023E00007C128282828140005C20000000002CBDD
:1023F000170BB4E577F1FFFF4FF1FFFF4F02B06419
:10240000011101FF03C7A6E9023620023A1102B802
:102410000902D01F0120012902B9E301FF02B923FB
:10242000027200013900454D5054590046696E61F1
:102430006E63655F314400454D50545900454D5021
:102440005459004D6174685F314400537461745F86
:1024500031420041647655312F41647655325F3107
:1024600042004164764C315F314200454D50545931
:1024700000454D5054590054494D45522F4358463C
:10248000554E533100454D50545900435846554E12
:10249000533000584E555432205000584E55543148
:1024A00000584E555430004D4F44530053495A453F
:1024B0003A00524547533A00464C41475300494E73
:1024C000464F00535045454400434F4D00534C4543
:1024D0004550005649455700424545500044495330
:1024E00050004D454E5532004D454E550005504764
:1024F000383A46055047303A37044D4F445304505C
:10250000524556044E45585405464C4147530452D3
:1025100045475301580258590258410458595A54D2
:102520004255494C543A204A756E20323720323099
:1025300032342031303A33343A3335005645523A4A
:1025400020302E3930300053504545443A00424146
:10255000543A00534E3A002A2A2050582D34314321
:1025600058202A2A00054E4556455204344D494EFE
:1025700004324D494E04314D494E0533324D485ACF
:102580000532344D485A0531364D485A04384D48C5
:102590005A05405F4F464604405F4F4E044C4F4142
:1025A000440444554D5004455849540352544E0573
:1025B000534C454550044D4F524504564945570428
:1025C000494E464F05535045454403434F4D044241
:1025D000454550044449535011241FBECFEFCDBF91
:1025E000DFE7DEBF10E4A0E0B0E4E6EFFCE700E0E8
:1025F0000BBF02C007900D92AC3AB107D9F72EE598
:10260000ACEAB0E401C01D92A130B207E1F70E942C
:10261000B2390C94793E0C9400009091F05D81E009
:1026200098279093F05D809307408093064008952B
:102630001092F05D81E08093074080930540809385
:10264000064008958091D042813019F08EEC92E4DA
:1026500008958FEC92E408958031910508F0C097B9
:10266000E8E8F2E427E0289FB001299F700D1124CB
:1026700090E080E0DC01A60FB71FAD51BD4B258D6A
:1026800030E1239FA0011124248D242B2C9301964B
:1026900032968730910571F70895CF93DF93DC016F
:1026A000EB013EE049914D933A95E1F7DF91CF91EF
:1026B0000895CF93DF93342FDC01EB01231BA30F8D
:1026C000B11DC30FD11D49914D932A95E2F7DF91BA
:1026D000CF910895242FDC01261BA60FB11D1D925A
:1026E0002A95EAF70895CF93DF93342FDC01EB01AD
:1026F000231BA30FB11DC30FD11D4C9158815D93B6
:1027000049932A95D2F7DF91CF910895CF93DF9324
:10271000DC01022E000C330B51E0E42FF0E02E1709
:102720003F071CF4DF91CF91089580E0611571059A
:1027300021F0EB01CE0FDF1F8881EA0FFB1F908194
:10274000C0919A5D9C0F980F90838091E0429817FA
:1027500030F0981B908350939A5D4F5FDECF1092BC
:102760009A5DFBCF0F93FC0131E0021714F40F9137
:10277000089590E06115710531F0DB01A20FB11DE4
:1027800027FDBA959C9180E04115510531F0DA01A1
:10279000A20FB11D27FDBA958C91981B80919A5D6F
:1027A000981B97FF0FC08091E042980F30939A5D7D
:1027B000309731F0DF01A20FB11D27FDBA959C9330
:1027C0002F5FD3CF10929A5DF3CFCF93DF93242F57
:1027D000EC01C60FD11D261B498149932A95E2F7CA
:1027E0001A92DF91CF910895CF93DF93DC0110927D
:1027F0009A5D2417A4F0E42F042E000CFF0B90E048
:102800006115710521F0EB01CE0FDF1F9881EA0FF2
:10281000FB1F8081891731F081E080939A5DDF9101
:10282000CF9108954F5FE5CFA5EDB2E48D919C91D6
:102830001197E7EDF2E4208131812D933C93A9EDCE
:10284000B2E42D913C91119720833183EBEDF2E4BA
:10285000208131812D933C93108211820895089537
:102860000E9414148093D1429093D24208950C9404
:1028700014140E941414E8E8F2E4292F22952F7012
:1028800022A39F7091A3982F92959F7090A38F7011
:10289000878F0895E8E8F2E482A1829591A1892BBF
:1028A00090A19295278D922BE1EDF2E490838183A4
:1028B0000895CF92DF92EF92FF928295837090E01D
:1028C0009C01220F331F227095958795822B909142
:1028D000D442292F22952F7030E02D523E4BF90122
:1028E0009081A3EDB1E4F4E08F02A001112430E067
:1028F00020E06D91691315C0F90164E0EE0FFF1F30
:102900006A95E1F7E40FF51FED53FF4BC080D180CE
:10291000E280F380CD28CE28CF2819F0FD017197F1
:1029200080832F5F3F4F2031310519F7FF90EF90E3
:10293000DF90CF90089564EA72E482EB92E40C9405
:102940004D1362EB72E484EA92E40C944D1364EA52
:1029500072E480EC92E40C944D1360EC72E484EA2F
:1029600092E40C944D13E8E8F2E4968D858D8295FF
:10297000807F248D822B8093BE5D9093BF5D1092EB
:10298000FC411092FD410895E8E8F2E4858D20E1D4
:10299000829FC0011124248D822B8093FC4190934F
:1029A000FD41089582958F708093955D85E08093B9
:1029B000C05D08951092E1420895E8E8F2E4858D43
:1029C00090E1899F90011124848D822B8093E142B4
:1029D0000895E8E8F2E48091E142982F9F70948F87
:1029E00082958F70858F0895E8E8F2E4A1EEB2E455
:1029F0008C91958D40E1949F90011124948D922BA0
:102A00009C93982F9F70948F82958F70858F0895D7
:102A10008091E1428093DF4280EA80930704089529
:102A20008091DF428093E1420895A1EEB2E48C915F
:102A3000EFEDF2E490819C93808380EA8093070419
:102A400008950E942213FC019081911103C08DE032
:102A5000808308959150908308950E942213FC0171
:102A600090819F5F90830E942213FC0120812E3071
:102A700008F0108208951092D042089581E080936A
:102A8000D04208959091CE428091CF42981303C0D6
:102A900081E080939A5D0895CF93C82F0E942213FE
:102AA000DC01EC91F0E0E857FD4BC295CF70C48F8C
:102AB0000E942213FC019081911104C08DE080835B
:102AC000CF91089591509083FBCFCF93DF930E94D5
:102AD0002213DC01EC91D091DE42C091DD42ED3059
:102AE000B1F48091AD40982F9F7B953B11F0873FCB
:102AF00049F4C093B142D093DD42C093DE42DF91EE
:102B0000CF910895D093B142C093A442F8CF809161
:102B1000AC408D3079F58091AD40853F61F0982FC4
:102B20009F70973039F582958F70982F977F9730E7
:102B300009F18B30F9F0D093DD42C093DE420E9460
:102B40002213DC01EC91F0E0E857FD4BC58F0E94A9
:102B50002213DC01EC91F0E0E857FD4BD48F0E948A
:102B60002213DC01EC91F0E0E857FD4B858D80935A
:102B7000A442C5CFF0E0E857FD4BD58F0E94221349
:102B8000DC01EC91F0E0E857FD4BC48FB8CFCF9358
:102B9000DF930E942213DC018C91C091DD428D30C5
:102BA00001F59091AD408091B142292F2F7B253BBB
:102BB00011F0973F49F48093DE428093DD42C09349
:102BC000B142DF91CF9108959091DE422091A442CD
:102BD0002093DD428093DE429093B142C093A442A1
:102BE000F0CF2091AC40D091DE4290E02D3099F5AD
:102BF0002091AD40253F61F0322F3F70373059F5BD
:102C000022952F70322F377F373029F12B3019F171
:102C100088579D4BFC01858D8093DE420E942213D4
:102C2000DC01EC91F0E0E857FD4B848D8093DD42B0
:102C30000E942213FC019091A442E081F0E0E85749
:102C4000FD4B958F0E942213DC01EC91F0E0E857D8
:102C5000FD4BD48FC3CF88579D4BFC01858D80934E
:102C6000DE420E942213DC01EC91F0E0E857FD4BBC
:102C7000848D8093DD420E942213DC01EC91F0E010
:102C8000E857FD4BD58F0E942213DC01EC91F0E058
:102C9000E857FD4BC48F95CF809187428093D142F6
:102CA000089580918742E8E8F2E4982F92959F700A
:102CB00090A38F70878F08958091F15D9091F25D60
:102CC000892B91F08091F15D9091F25D0197809355
:102CD000F15D9093F25D81E09091FB41911101C013
:102CE00080E080939A5D08958091985D823099F795
:102CF0001092985D1092FB411092874280917C4225
:102D000090E0E5CF089580E18093E04208958AE065
:102D10008093E0420895E8E8F2E482A1829591A1CF
:102D2000892B90A19295278D922B9093C1408093EF
:102D3000C24082E08093C05D0895E8E8F2E4968F97
:102D4000982F92959F70958F8F70848F1092C05D91
:102D5000089583E08093C05D0895CF93DF93CDB74E
:102D6000DEB72E97CDBFDEBF82958F70E82FF0E0E3
:102D7000E55EFC4FE491DE0111969E01215F3F4F1D
:102D8000BD0181E08E0F0E2E000CFF0BE857FD4BAE
:102D9000948D9D93E0E08E300CF4E82FA217B307DA
:102DA00081F784EA92E40E944D132E96CDBFDEBFD8
:102DB000DF91CF91089590917F42809108409813C0
:102DC00004C081E080939A5D089510929A5D089501
:102DD00084E08093C05D0895F8948091D35D88234A
:102DE000B9F0E091D15DF0E0EF53F24A808190912B
:102DF000D15D9F5F9093D15D9091D15D9F709093D5
:102E0000D15D9091D35D91509093D35D7894089566
:102E100080E0FCCF9091240895FFFCCF809322089E
:102E200008952EE0FC0111922A95E9F7089588E8AB
:102E300092E40E94111786E992E40E94111784EA35
:102E400092E40C941117E3EEF2E480EB9AE1DF01D7
:102E50009C011D9221503040E1F70895CF93DF93FC
:102E6000DC01FC013B966B3061F41B968C911B9747
:102E700092919183EA17FB07D9F78083DF91CF9175
:102E800008958C91ED0199819993CE17DF07D9F7B9
:102E90001B968C93F3CF9C014097C09768F0211547
:102EA00082E0380749F0C901805F9240419720F0E5
:102EB00081E0203F334008F080E008958091864211
:102EC000811106C00E9414148093D1429093D24283
:102ED0000895CF93DF938091FC419091FD4100973D
:102EE00031F08D3F910589F0DF91CF910895C09128
:102EF000BE5DD091BF5DCE010E944B178823A1F328
:102F0000CE01DF91CF910C942C132091A642809199
:102F1000A54230E1839FC0011124922B2091A4424D
:102F2000822B8093EC5D9093ED5D81E08093064071
:102F3000DBCF0E942213DC01EC91ED30A1F49091E3
:102F4000AD408091B142292F2F7B253B11F0973F57
:102F500039F49091DE429093DD428093DE420895F1
:102F60009091A442F8CFF0E0E857FD4B848D809318
:102F7000DD42858DF2CF8091F15D9091F25D892BDC
:102F800051F08091F15D9091F25D01978093F15D38
:102F90009093F25D08958091985D8130D9F780918A
:102FA0000B428111F7CF82E08093985D80917C4243
:102FB00090E0ECCF8EE0815078F4809186428823B7
:102FC00051F08091965D8D3031F48091A4428093D0
:102FD000B142809395420895E82FF0E0E857FD4B09
:102FE000948D20819223948FE6CFCF93DF93A4EA30
:102FF000B2E4C0ECD2E43EE04C9158815D93499339
:103000003A95D1F7DF91CF910895CF9382958F7044
:10301000E82FF0E0E55EFC4FC4910E942213FC0112
:10302000C083CF91089582958F70E82FF0E0E55E20
:10303000FC4FE491A1EEB2E421E030E002C0220FA7
:10304000331FEA95E2F78D919C911197822B932B78
:103050008D939C9308952091935D3091945D82951A
:103060008F70E82FF0E0E55EFC4FE49181E090E0A6
:1030700002C0880F991FEA95E2F78223932321E08B
:10308000892B09F420E020939A5D089582958F7032
:10309000E82FF0E0E55EFC4FE491A1EEB2E481E0C0
:1030A00090E002C0880F991FEA95E2F7809590950D
:1030B0002D913C911197822393238D939C93089596
:1030C00082958F70E82FF0E0E55EFC4FE49181E09F
:1030D00090E002C0880F991FEA95E2F72091E14243
:1030E0003091E2428223932321E0892B09F420E0EE
:1030F00020939A5D0895CF93C82F0E942213C29502
:10310000CF70EC2FF0E0E55EFC4FE491DC018C9198
:103110000E2E000CFF0B8E171F0619F481E0809312
:103120009A5DCF910895CF93DF93A4EAB2E4C2EB06
:10313000D2E43EE04C9158815D9349933A95D1F7A2
:10314000DF91CF91089580918642882331F00E94CB
:1031500014148093D1429093D2420895E8E8F2E4A7
:1031600082A1829591A1892B90A19295278D922B76
:10317000E9EDF2E4208131812093DB423093DC429F
:10318000A7EDB2E42D913C91119720833183E5EDB9
:10319000F2E4208131812D933C93908381830895C3
:1031A0008EE0815078F480918642882351F080919E
:1031B000965D8D3031F48091A4428093B14280932A
:1031C00095420895E82FF0E0E857FD4B948D20815B
:1031D000922B948FE6CFE0E4F4E081818D608183CF
:1031E000E0E0F4E0818180648183E0E6F9E084E05E
:1031F000818381E3808308958093640980916309CA
:1032000087FFFCCF08951F93CF93DF93C0E0D4E0F6
:1032100010E41E830E94FC181D83DF91CF911F9143
:103220000895CF93C82F8AE20E94031982E20E9478
:10323000FC1883E20E94FC188BE20E9403198C2F79
:103240000E94FC188C2F0E94FC188CE20E9403192B
:10325000C6E080E00E94FC18C150D9F7CF910895D4
:103260001F93CF93DF93C82F162F8AE20E94031972
:10327000C75E8C2F0E94FC188C2F0E94FC188BE2DA
:103280000E94031980E00E94FC188CE70E94FC1841
:103290008CE20E940319C7E7D1E0812F0E94FC183D
:1032A0002197D9F7DF91CF911F910895CF93DF93A5
:1032B0008AE20E94031989E10E94FC1889E10E94B8
:1032C000FC188BE20E94031980E00E94FC188CE736
:1032D0000E94FC188CE20E940319C7E7D1E08FEF2F
:1032E0000E94FC188FEF0E94FC188CEF0E94FC18C3
:1032F0002197A9F7DF91CF910895FF920F931F9324
:10330000CF93DF93C62F8053990B2CE0289F800129
:10331000299F100D11240E581C4F8AE20E94031998
:1033200089E10E94FC1889E10E94FC188BE20E944E
:1033300003198C2F0E94FC1884E0F82EFC0E83E009
:103340008C0F0E94FC188CE20E940319D0E0C0E0B0
:10335000F801EC0FFD1F84910E94FC182196CC30DF
:10336000D105B1F78F2DDF91CF911F910F91FF9074
:1033700008950F931F93CF938C01C0E0F801EC0FD9
:10338000F11D8081811105C0862FCF911F910F9172
:1033900008950E947D19682FCF5FF0CFEF92FF92C2
:1033A0000F931F93CF93DF93042F10E0D0E0C0E082
:1033B0007C01649FE00CF11C1124C017D10741F47B
:1033C000822FDF91CF911F910F91FF90EF90089581
:1033D000F701EC0FFD1F8491622F0E947D19282FA9
:1033E0002196EBCFEF92FF920F931F93CF93DF9332
:1033F000F62E142F9CE0899F200D311D1124E90128
:10340000C058D1408AE20E940319175E812F0E94A2
:10341000FC18812F0E94FC188BE20E9403198F2D4B
:103420000E94FC1814E01F0D83E08F0D0E94FC1811
:103430008CE20E940319F12CE12CFE01EE0DFF1D20
:10344000849180270E94FC188FEFE81AF80A9CE00C
:10345000E916F10491F7812FDF91CF911F910F9120
:10346000FF90EF9008950F931F93CF93DF93C62F94
:103470009BE1899F800111240E541A4F8AE20E9419
:10348000031989E10E94FC1889E10E94FC188BE273
:103490000E9403198C2F0E94FC1888E08C0F0E9458
:1034A000FC188CE20E940319D0E0C0E0F801EC0F98
:1034B000FD1F84910E94FC182196CB31D105B1F7F4
:1034C000DF91CF911F910F910895FF920F931F935A
:1034D000CF93DF93C62F8053990B2CE0289F800158
:1034E000299F100D11240F5F1F4D8AE20E940319BE
:1034F00082E20E94FC1882E20E94FC188BE20E9489
:1035000003198C2F0E94FC1884E0F82EFC0E83E037
:103510008C0F0E94FC188CE20E940319D0E0C0E0DE
:10352000F801EC0FFD1F84910E94FC182196CC300D
:10353000D105B1F78F2DDF91CF911F910F91FF90A2
:103540000895FF920F931F93CF93DF93EC01862F83
:10355000FE01F49069E170E0F4E0FF9E60197109EA
:1035600011247595679599E1899F600D711D11244E
:103570006F5F7F4F8E01802F8C1B8F1530F0DF9196
:10358000CF911F910F91FF9008950F5F1F4FF8018A
:1035900084910E94651A682FEECF1F93CF93DF931B
:1035A000C9E18C9FC02D112411E01C0F8AE20E94FA
:1035B000031983E20E94FC1883E20E94FC188BE24C
:1035C0000E940319812F0E94FC1887E18C0F0E9432
:1035D000FC188CE20E940319D5E48FEC0E94FC18C1
:1035E000D150D9F78AE20E94031982E20E94FC18A6
:1035F00082E20E94FC188BE20E940319812F0E9434
:10360000FC1882E08C0F0E94FC188CE20E940319C7
:103610008DE30E94FC1880E00E94FC188FE10E945C
:10362000FC188FE30E94FC1881ED0E94FC188FEFBC
:10363000DF91CF911F910C94FC18CF938AE20E94E6
:10364000031982E20E94FC1882E20E94FC188BE2BD
:103650000E94031980E00E94FC188CE70E94FC186D
:103660008CE20E940319CDE78FE30E94FC188FEFD4
:103670000E94FC188FEF0E94FC18C150A9F76FEF51
:103680008AE00E943019CC3728F48C2F0E9411193F
:10369000CC2321F08FEF8C0F0E941119C75EC63921
:1036A00091F7CF910895EF92FF920F931F93CF93CD
:1036B000DF937C01D42F122FC0E0F701EC0FF11D36
:1036C0008081811108C0862FDF91CF911F910F91CA
:1036D000FF90EF900895012F29E336E04D2F0E94CF
:1036E000F219682FCF5FE9CFEF92FF920F931F93EC
:1036F000CF93DF937C01D42F122FC0E0F701EC0FA2
:10370000F11D8491811107C0DF91CF911F910F911D
:10371000FF90EF900895012F29E336E04D2F0E948E
:10372000F219682FCF5FEACFAF92BF92CF92DF92AC
:10373000EF920F931F93CF93DF93362F102FC42E4A
:10374000D12C622FD0E0C0E05C01349FA00CB11CF2
:103750001124CC15DD0559F4862FDF91CF911F91EF
:103760000F91EF90DF90CF90BF90AF900895F5014B
:10377000EC0FFD1F84910E2D29E336E0412F0E94AE
:10378000F219682F2196E5CFFF920F931F93CF93E5
:10379000DF93C62F9CE0899F800111240F5B1D4D94
:1037A0008AE20E94031982E20E94FC1882E20E94CF
:1037B000FC188BE20E9403198C2F0E94FC1884E0F5
:1037C000F82EFC0E83E08C0F0E94FC188CE20E9405
:1037D0000319D0E0C0E0F801EC0FFD1F84910E94B6
:1037E000FC182196CC30D105B1F78F2DDF91CF9108
:1037F0001F910F91FF9008950F931F93CF938C010A
:10380000C0E0F801EC0FF11D84918F3F21F4CF91BE
:103810001F910F9108950E94C41B682FCF5FF1CFB5
:10382000EF92FF920F931F93CF93DF93162FC42F26
:10383000022F2AE2829FC00111249C012754354F98
:1038400079018AE20E94031989E18C0F0E94FC1819
:103850008AE18C0F0E94FC188BE20E940319812FD1
:103860000E94FC1886E0810F0E94FC188CE20E94E6
:103870000319D0E0C0E0F701EC0FFD1F8491802315
:103880000E94FC182196CA32D105A9F787E0810F62
:10389000DF91CF911F910F91FF90EF900895FF92CC
:1038A0000F931F93CF93DF938C01D62FF42E65E0F7
:1038B000C0E0F801EC0FF11D8081811106C0DF919D
:1038C000CF911F910F91FF9008952F2D4D2F805470
:1038D0000E94101C63E0680FCF5FEBCFEF92FF9266
:1038E0001F93CF93DF93162FC42F22E1829FC00135
:1038F00011249C012754304E79018AE20E94031959
:1039000089E18C0F0E94FC188AE18C0F0E94FC1840
:103910008BE20E940319812F0E94FC1882E0810F24
:103920000E94FC188CE20E940319D0E0C0E0F7016D
:10393000EC0FFD1F84910E94FC182196C231D10525
:10394000B1F783E0810FDF91CF911F91FF90EF904E
:103950000895CF93DF938AE20E94031989E10E94C0
:10396000FC1883E20E94FC188BE20E94031980E09D
:103970000E94FC188CE70E94FC188CE20E9403193C
:10398000CDE1D0E180E00E94FC182197D9F7DF91CA
:10399000CF91089580E10C94031981E10C940319EF
:1039A000262F2150330BF901EA59FC4FE49191E0A5
:1039B000633008F090E0891B282F26952695280F64
:1039C0003327331F64E60E94153DB901681B710956
:1039D000CB018E0F911D840F911D67E070E00E9456
:1039E000433D8F5F0895823021F4637081F48DE14F
:1039F00008958150990B67E070E00E94433D62E0BA
:103A000070E00E94433D9FE1981B892F08958CE14F
:103A100008958D3010F08C500895811101C08CE014
:103A20000895CF93DF93DC01362F4423C1F06A3031
:103A3000B0F4E0E0222311F02C93E1E0ED01CE0F91
:103A4000D11D832F6AE00E94153D905D9883EF5F42
:103A5000EA0FFB2FF11D1082DF91CF910895832F84
:103A60006AE00E94153D805D8C93E7CFFF920F9333
:103A70001F93CF93DF93CDB7DEB72597CDBFDEBFC2
:103A800001E712E4F80160896150282F43E08BE2DE
:103A900093E00E94CE19682F8EE50E947D19F801EF
:103AA00067816150282F43E081E493E00E94CE19A2
:103AB000682F8EE50E947D19F82EF801608520E0C0
:103AC00041E0CE0101960E94111D6F2DCE0101969D
:103AD0000E94B9192596CDBFDEBFDF91CF911F910E
:103AE0000F91FF9008951F93CF93DF93CDB7DEB76B
:103AF0002597CDBFDEBF182F80917342811136C04C
:103B00006091804220E441E0CE0101960E94111DA7
:103B1000612FCE0101960E94B919682F8AE30E9495
:103B20007D19182F6091754220E040E0CE0101968A
:103B30000E94111D612FCE0101960E94B919682FB4
:103B40008091734281110BC0809174428C309CF043
:103B500080E50E947D19682F8DE40E947D192596CD
:103B6000CDBFDEBFDF91CF911F9108956091744268
:103B700020E440E0C9CF81E4ECCF82EA91EEA0E0FE
:103B8000BB27E3ECF0E480839183A283B38310929C
:103B9000D34182EA9DECA0E0BB27808B918BA28B66
:103BA000B38B1092D44182EA99EBA0E0BB2780A3AB
:103BB00091A3A2A3B3A31092D54182EA95EAA0E013
:103BC000BB2780AB91ABA2ABB3AB81E08093D64176
:103BD00042EA51E960E07727409313415093144142
:103BE00060931541709316418093D84142EA5DE796
:103BF00060E0772740931741509318416093194133
:103C000070931A4140E050ED61E0772740934341C3
:103C10005093444160934541709346418093DB410A
:103C200040E05CEB61E0772740935341509354416F
:103C300060935541709356418093DC4180E098EA4F
:103C4000A1E0BB278093574190935841A0935941DD
:103C5000B0935A4180E094E9A1E0BB27809363418F
:103C600090936441A0936541B09366411092DD4109
:103C700080E090E8A1E0BB2780937341909374416A
:103C8000A0937541B09376411092DE4180E090E0C0
:103C9000A1E0BB278093A3419093A441A093A541A9
:103CA000B093A6411092E141089581E08093005EB7
:103CB0001092D1421092D24280939A5DE8E8F2E4E9
:103CC00011921586138E11A617AA22E4E639F2077F
:103CD000B9F71092DD421092DE421092DF4210924C
:103CE000E1421092E2421092935D1092945D109224
:103CF000CE421092CF421092D04280E18093E042B7
:103D00001092C05D1092985DE3ECF0E480E291E0E7
:103D1000DF019C011D9221503040E1F70C94BD1D44
:103D2000CF93DF931092F05DE5EBF0E4C4EFDDE5B7
:103D3000A0EBBDE5119219921D9280E4E13CF807D9
:103D4000C9F71092EC5D1092ED5DDF91CF9108956F
:103D50000F938091EC5D9091ED5D8370992700E069
:103D600029E336E048E061E0892B29F488E50E94E8
:103D7000F2190F91089580E2FACF60E089E00E9485
:103D800030190E94A81E8091EC5D80FF05C068E696
:103D90008CEE92E00E94FC1B8091EC5D81FF05C0DF
:103DA00065E586EE92E00E94FC1B8091EC5D82FF4F
:103DB00004C06EE484E00E94C41B8091EC5D83FF2C
:103DC00004C06AE483E00E94C41B8091EC5D84FF20
:103DD00004C066E482E00E94C41B8091EC5D85FF14
:103DE00004C062E481E00E94C41B8091EC5D86FF08
:103DF00004C06EE380E00E94C41B8091EC5D87FFED
:103E000005C067E28FED92E00E94FC1B8091EC5DA3
:103E10009091ED5D90FF05C068E18AED92E00E940F
:103E2000FC1B8091EC5D9091ED5D91FF04C064E11D
:103E300089E00E94C41B8091EC5D9091ED5D92FF42
:103E400005C061E084ED92E00E94FC1B8091EC5D76
:103E50009091ED5D88279370892B29F468E18FECB0
:103E600092E00C94FC1B08950F931F93CF93DF9364
:103E70008091F05D882331F100E01EE520EB3DE507
:103E8000C5EBD0E4E3EEF1E464EF7DE5D8019E916B
:103E90008D01D9011B968C91B4E08B9FA001112458
:103EA000892F8370842B8295807F4B85840F868B2E
:103EB00096959695978B21503109219732976017E7
:103EC000710721F7DF91CF911F910F910895CF9343
:103ED000DF9388E1E3EEF1E4A4EDBDE501900D92FE
:103EE0008A95E1F7C3EED1E485E02FEF47E0682F34
:103EF0008E890E94101C47E0682F8F890E946E1CDB
:103F0000229791E4CB3CD90781F7DF91CF910895B7
:103F1000E3EEF1E4A4EDBDE591918D91981306C017
:103F200081E4EA3FF807C1F781E0089580E0089551
:103F3000DC011596FB0135963E912291321305C0A6
:103F4000A817B907C9F781E0089580E00895FC013A
:103F5000108211821282138214820895DC01159658
:103F6000FB0135963E912291231728F0321728F055
:103F7000A817B907B9F781E0089580E008956F9216
:103F80007F928F929F92AF92BF92CF92DF92EF92E9
:103F9000FF920F931F93CF93DF938B01DB011D9251
:103FA0001D921D921C921397EC0122963C01BEE0DB
:103FB0006B0E711CC12CD12C7601C394A991B0E079
:103FC000A70196010E94893DF80180809180A2801E
:103FD000B380DC01CB01880D991DAA1DBB1D808318
:103FE0009183A283B383AAE0B0E00E94893D6B0174
:103FF0007C016C167D0611F7DF91CF911F910F9117
:10400000FF90EF90DF90CF90BF90AF909F908F90F8
:104010007F906F900895AC0190E070E0292F092EF9
:10402000000C330B261737070CF00895240F351FAB
:10403000F90110829F5FF2CF4F925F926F927F9251
:104040008F929F92AF92BF92CF92DF92EF92FF92A8
:10405000CF93DF9300D000D0CDB7DEB7F894BE0188
:104060006F5F7F4F8DE192E40E94BF1F7894C980FB
:10407000DA80EB80FC808CE3882E912CA12CB12C73
:10408000C701B601A50194010E94573D6093764295
:10409000CA01B901A50194010E94573D6093754280
:1040A000C701B60120E13EE040E050E00E94573DEC
:1040B000CA01B90128E130E040E050E00E94573DDC
:1040C00060937442809174420E94091D80938042E3
:1040D000C701B60120E831E541E050E00E94573DBC
:1040E00069017A01C982DA82EB82FC82CA01B901D4
:1040F0006C557C498F4F9F4F22E0660F771F881FBA
:10410000991F2A95D1F721EB3AE342E050E00E9453
:10411000573D215F3F4F4F4F5F4F82EAC80E8FEDF3
:10412000D81E84E2E81EF11CC20ED31EE41EF51E4A
:1041300062E056954795379527956A95D1F7C21A4B
:10414000D30AE40AF50AA4E1B0E0A70196010E94AF
:10415000893D2B013C012AE8421A29E0520A6108F4
:104160007108C301B20129E83CE140E050E00E943F
:10417000573D49015A01ADE6B1E00E94893DC61A9A
:10418000D70AE80AF90AC301B20124E232E740E0A3
:1041900050E00E94573DC21AD30AE40AF50AA8EE7D
:1041A000B3E0A70196010E94893D29E837E740E086
:1041B00050E00E94573D29013A018EE1289FC01826
:1041C0001124A9E5B2E00E94893D28EE33E040E0E9
:1041D00050E00E94573DC21AC09279422EE042162A
:1041E00051046104710480F58CE6881A82E1980A12
:1041F000A108B10821E0421A51086108710880E362
:10420000880E809277424092784240917942609144
:104210007842809177420E94D01C8093814281E055
:104220008093B1402496CDBFDEBFDF91CF91FF9048
:10423000EF90DF90CF90BF90AF909F908F907F9046
:104240006F905F904F9008958BE6881A82E1980AEC
:10425000A108B1082DE0421A510861087108CFCFBA
:104260002F923F924F925F926F927F928F929F9286
:10427000AF92BF92CF92DF92EF92FF920F931F9374
:10428000CF93DF93CDB7DEB72997CDBFDEBFC09008
:1042900077420C2C000CDD0820E3C21A28EFD20A6A
:1042A0000D2C000CEE08FF0830917842232E022CD2
:1042B000000C330829823A8291012330310548F4F9
:1042C000245F3F4F29833A8331E0C31AD108E108C4
:1042D000F10810917942ADE6B1E0A70196010E9484
:1042E000893D4601570122E0B694A794979487949C
:1042F0002A95D1F7860E971EA81EB91EC701B601D2
:1043000020E931E040E050E00E94573D820E931ECC
:10431000A41EB51EC701B60124E630E040E050E01F
:104320000E94573D821A930AA40AB50A29813A814C
:104330002F5F3F4FC901880F991F820F931F65E0C0
:1043400070E00E942F3D2EE129803A80229DC0011D
:10435000239D900D1124810F911D17FD9A95FB014E
:10436000E80FF91F9F0150E040E060E070E0CB01F2
:10437000E9833A834B835C836D837E838F83988745
:104380009401A50160E070E080E090E0A980BA802F
:10439000C12CD12CE12CF12C00E010E00E94533E06
:1043A0002A5E36494A40510961097109810991091A
:1043B000E0E8AE2EF1E5BF2ECC24C3940E949C3DD4
:1043C00059016A017B018C01A091744240917542B0
:1043D000409076420A2E000CBB0B20E13EE00E948A
:1043E000823D042C000C550866087708DC01CB01DF
:1043F000840D951DA61DB71D3CE34302A0011124A9
:10440000840F951FA11DB11D1C012D01612C712C64
:1044100043013A82AB835C826D827E828F82988672
:104420009C01AD0160E070E080E090E00E94533EAE
:1044300029014A01698779831C01F8941092995DDA
:10444000AFE16A2EA2E47A2E8AE0A82EB12CC12C0C
:10445000D12CE12CF12C00E010E09201A40169853F
:104460007981C1010E94F43DF30121933F01920142
:10447000A40169857981C1010E94F63D29014A01A3
:10448000698779831C012BE232E426153705E1F6B2
:104490006DE172E485E592E40E944D1378942996CB
:1044A000CDBFDEBFDF91CF911F910F91FF90EF90B5
:1044B000DF90CF90BF90AF909F908F907F906F9044
:1044C0005F904F903F902F900895FC0195E020E081
:1044D0008191980FDF0111979A3060F49C9390E0DE
:1044E000211101C09E5F2F5F2E3011F09111F0CF8E
:1044F000892F08959A509C9391E0F2CFCF93803109
:1045000008F06FC0E82FF0E0E857FD4D0C94793DBE
:104510009822A522BD22C82201232023F12236237E
:104520003C234F2360236823702378238023842334
:1045300080911C422EE0829FC001112464EA72E443
:10454000835E9D4BCF910C944D1380911C42CEE025
:104550008C9FC001112464EA72E4835E9D4B0E942B
:104560004D13E0911C42CE9FF0011124E45FFD4BFE
:10457000118A128ACF910C941C2080911C422EE04B
:10458000829FC001112464EA72E4875C9D4BDACFFC
:1045900080911C42811127C090910C422091A5422C
:1045A00080E1289F900111248091A442806C822B8D
:1045B000892380930C4280910C428F7391F48091F7
:1045C000935D9091945D9F7D8093935D9093945DB6
:1045D0008091935D9091945D9F7E8093935D909385
:1045E000945DCF91089523E040E065EA72E48EE0A7
:1045F00092E40E945913809111428170809311427C
:10460000F0CF80911C422EE0829FC001112464EA09
:1046100072E48B5A9D4B0E944D138091644282FB41
:10462000882780F920917342022E000C330B8217E9
:104630001306B9F28093734281E08093B140D1CFE9
:1046400024E040E064EA72E487E192E40E945913B6
:1046500082E192E40E94A71F80910C4290910D424A
:10466000946080930C4290930D42BBCF80910C429A
:1046700090910D429B7FF5CF40910C4250910D429D
:1046800020911C42255F81E090E002C0880F991FB5
:104690002A95E2F78095909584239523E2CF409167
:1046A0000C4250910D4220911C42255F81E090E028
:1046B00002C0880F991F2A95E2F7842B952BD1CF42
:1046C00040910C4250910D4220911C42285FDBCF5B
:1046D00040910C4250910D4220911C42285FE6CF40
:1046E00040910C4250910D4220911C422A5FCBCF49
:1046F00040910C4250910D4220911C422A5FD6CF2E
:1047000081E080931C426DCF10921C426ACF7F9251
:104710008F929F92AF92BF92CF92DF92EF92FF92D1
:104720000F931F93CF93DF93082F02950F70C02F25
:10473000D0E0E090BE5DF090BF5D20EFE22223E08C
:10474000F222E02AFD2AE092BE5DF092BF5DC70131
:104750000E944B17182F882381F0C701DF91CF915A
:104760001F910F91FF90EF90DF90CF90BF90AF908F
:104770009F908F907F900C942C138091FC4190918E
:10478000FD418B3F910509F469C08D3F910541F5CD
:10479000C154DD4FFE01C49180E0C7FD8BE0FC2FCA
:1047A000FF709F2E00E02C2F2071822EDBE0D81BA3
:1047B00090E0FC01EB54FF4B7F01FC2FF0727F2E49
:1047C0009C012C50324A6901C074FC01E055F24A48
:1047D0005F01901213C081E08093074080930540F1
:1047E000DF91CF911F910F91FF90EF90DF90CF90CD
:1047F000BF90AF909F908F907F900895882069F030
:104800006D2F85EB90E40E942E17E12FF0E0E85722
:10481000FD4B848DF70180831F5F772069F06D2F3A
:1048200084EF9DE50E942E17E12FF0E0E857FD4B45
:10483000848DF60180831F5FCC2371F06D2F80EB98
:104840009DE50E942E17E12FF0E0E857FD4B848D87
:104850008170F50180831F5F0F5FBBCF802FDF91D9
:10486000CF911F910F91FF90EF90DF90CF90BF906D
:10487000AF909F908F907F900C947E228230A1F019
:1048800038F08430E9F1C8F0853009F442C0089569
:1048900060911C428EE0689FB0011124635E7D4BE5
:1048A00084EA92E40C944D1360911C428EE0689F60
:1048B000B0011124675C7D4BF3CF80911C428111C4
:1048C00017C080910C428F708093A44280910C425B
:1048D00082958F708093A54280910D428F70809356
:1048E000A64280910D42829581708093A7420895DF
:1048F00023E040E06EE072E485EA92E40C94591300
:1049000060911C428EE0689FB00111246B5A7D4B70
:10491000C7CF24E040E067E172E484EA92E4EECF9E
:104920006F927F928F929F92AF92BF92CF92DF92BF
:10493000EF92FF920F931F93CF93DF93182F12954F
:104940001F7084EA92E40E9411178091FC419091BB
:10495000FD418B3F910509F4B9C08D3F910509F4E4
:1049600040C0892B79F5112359F08091BE5D90915B
:10497000BF5D807F9370812B8093BE5D9093BF5D00
:104980000091BE5D1091BF5DC8010E944B17882346
:10499000C9F00031110510F00053110987E0809F24
:1049A000E001819FD00D1124CD51DD4BA4EAB2E48A
:1049B00067E04991542F52955F704F704D935D930E
:1049C0006A95B9F7DF91CF911F910F91FF90EF900A
:1049D000DF90CF90BF90AF909F908F907F906F901F
:1049E0000895153001F58091EC5D9091ED5D909307
:1049F000A6429C0194E0369527959A95E1F72F7091
:104A00002093A5428F708093A4428091F05D88230B
:104A1000C9F21330B8F21530A9F281E08093074053
:104A200080930540CFCFE12FF0E0E155FD4FC491D9
:104A30000BE0C7FF00E02C2F2F70822ED0E0912CCE
:104A40003C2F3071732E802F90E0DC01AB54BF4BB4
:104A50007D01BC2FB0726B2E9C012C50324A690133
:104A6000C074DC01A055B24A5D01891471F277204F
:104A700069F0ED2FF0E0E857FD4BD7018C91848F62
:104A8000DF5F602F85EB90E40E942E17662069F0AF
:104A9000ED2FF0E0E857FD4BD6018C91848FDF5F5E
:104AA000602F84EF9DE50E942E17CC2369F0ED2F37
:104AB000F0E0E857FD4BD5018C91848FDF5F602FCC
:104AC00080EB9DE50E942E179394CFCF812FDF912D
:104AD000CF911F910F91FF90EF90DF90CF90BF90FB
:104AE000AF909F908F907F906F900C943E246EE0DB
:104AF0008DE192E40E940B206EE089E392E40E9433
:104B00000B206EE085E592E40E940B206EE08BE2C4
:104B100092E40E940B206EE087E492E40E940B2056
:104B20006EE083E692E40E940B2064E08EE092E463
:104B30000E940B2082E192E40E94A71FECE0F2E4C5
:104B4000108A8081918180648083918380819181AA
:104B50009160808391834AE050E069E070E08AE4EC
:104B600092E40E94723E0C943021E62FE69527E0F5
:104B7000AC01249FC001259F900D112488579D4BA7
:104B8000E80FF92FF11DE55AFF4F808160FD8295F6
:104B90008F700895CF92DF92EF92FF929C01232FA6
:104BA000332722952F70F901ED53FE4BE081220F40
:104BB000331F220F331FE20FF32FF11DEE0FFF1FE4
:104BC000EE0FFF1FED53FF4BC080D180E280F380DA
:104BD000C114D104E104F10469F19F70B701A60189
:104BE000480F591F611D711D6BBFFA01A791AC01E0
:104BF000569547955695479570E060E0505F6F4F2A
:104C00007F4F4C0D5D1D6E1D7F1D6BBFFA014791DF
:104C100050E0880F991F8670992702C055954795D7
:104C20008A95E2F78A2F942F9370FF90EF90DF9090
:104C3000CF90089580E090E0F8CF8091D35D8823F5
:104C4000E1F30E94EC1690ED980F9A3030F09FE956
:104C5000980F963020F499EA980F892F08959FEBCA
:104C6000980F963010F499ECF7CF803231F390E042
:104C7000F4CF8A3310F08755089580530895F8943F
:104C8000E1ECFDE5108A118A128A78940895F8946F
:104C90009091D35D9031B1F0E091D25DF0E0EF53AF
:104CA000F24A80838091D25D8F5F8093D25D809144
:104CB000D25D803110F01092D25D8091D35D8F5F14
:104CC0008093D35D789408958091240886FFFCCF6B
:104CD00008951F920F920FB60F9211240BB60F92E8
:104CE0008F93EF93FF93E091D25DF0E080912008E5
:104CF000EF53F24A80838091D25D8F5F8093D25DC3
:104D00008091D25D8F708093D25D8091D35D8F3022
:104D100028F48091D35D8F5F8093D35DFF91EF91F5
:104D20008F910F900BBE0F900FBE0F901F90189594
:104D30000F931F93CF93DF93EC018C01FE01019041
:104D40000020E9F73197EC1BFD0BC8018C1B9D0B74
:104D50008E179F0728F0DF91CF911F910F91089533
:104D6000F80181918F010E940A17E8CF813408F081
:104D7000875F8F70089547E0489F9001499F300DED
:104D8000112428573D4BBC016C5F7F4F8617970756
:104D900010F080E0089550E040E0FA01E55AFF4F3E
:104DA000E20FF31FE081E11109C04F5F5F4F473011
:104DB000510599F70196295F3F4FE8CF81E00895AB
:104DC00097E0899FB001112430E020E0A901460F4F
:104DD000571FFA01E556F24A4D515D4BDA019C919D
:104DE00090832F5F3F4F2730310581F7089527E0EB
:104DF000829FC001112430E020E0A901480F591F13
:104E0000FA01E556F24A4D515D4B6081FA0140814D
:104E1000641307C02F5F3F4F2730310571F781E0E2
:104E2000089580E00895FB016AE00E94153D905DC1
:104E30009283811107C080E2818380E28083838333
:104E400014820895805DF8CFCF93DF93EC01FB01CE
:104E50006AE070E00E942F3D9B01805D82836A3092
:104E6000710570F0CE0164E670E00E942F3D605D38
:104E70006083C9016AE070E00E942F3D805D04C03C
:104E800080E38083672BA9F781831382DF91CF9121
:104E90000895FB019EE291832AE0622F0E94153D56
:104EA000905D92830E94153D905D908386E583839B
:104EB0001482089581E08093000684E030E020E0D1
:104EC00091E090930A0640910D0640FFFCCF40917F
:104ED000100650911106240F351F815091F7C9011A
:104EE000969587959695879562E370E00E942F3D91
:104EF0006093084055E0369527955A95E1F784E090
:104F0000263B50F483E02B3A38F482E0213A20F437
:104F100081E0273908F480E0109200060895262FDA
:104F200030E0082E000C990BB9010E94433D820F1E
:104F3000931FB9010E94433D0895E62FE69527E0AF
:104F4000829FC001112488579D4BE80FF92FF11D56
:104F5000E55AFF4F808160FD82958F70089527E0AC
:104F6000289FD001299FB00D112430E020E0F901E5
:104F7000EA0FFB1FED51FD4B9081492F4F70FB0154
:104F8000408392959F7091832F5F3F4F6E5F7F4F5D
:104F90002730310561F708956F927F928F929F922B
:104FA000AF92BF92CF92DF92EF92FF920F931F9337
:104FB000CF93DF93CDB7DEB7A697CDBFDEBF982ED8
:104FC0000E94E026AE014F5F5F4F7A015E015DE017
:104FD000A50EB11C670180E2F60181936F01138673
:104FE000AE16BF06C9F7892D90E027E0289FF00193
:104FF000299FF00D1124E751FD4B3081303109F02C
:105000003FC0929E9001112484E090E050E0F901AD
:10501000E80FF91FEC51FD4B4081442331F0F701BB
:10502000E50FF11D4F7340835F5F01978E3FFFEFE8
:105030009F0769F7990C939485E02FEF492D682F0E
:10504000F70181917F010E94101C492D682FF70103
:1050500083850E946E1CCE14DF0479F7A696CDBF1F
:10506000DEBFDF91CF911F910F91FF90EF90DF9006
:10507000CF90BF90AF909F908F907F906F9008954A
:105080008E01075E1F4FB8010E94AF2780904843F2
:10509000A1E0B3E083FC02C0A3E0B1E090914643FD
:1050A00092959C70309147433F70432F898D2A8D94
:1050B000682F5AE0259F600D1124262F5B8D552304
:1050C000F9F054E6561B252F51E09830D9F4E22F21
:1050D000022E000CFF0B632F70E06F5F7F4F6E1787
:1050E0007F070CF457C051E0E617F70721F49DA1A4
:1050F00051E0953018F098E02A3024F090E002C09A
:105100009830C9F36EA1662311F06DE26983943083
:1051100009F4BAC0983009F43FC0911107C1552372
:1051200011F08DE28A87822F6AE00E94213D90E390
:10513000980F9B8790E3920FF6EF8F9F900D1124AD
:105140009C87AE87383008F09CC0F801E31BF1095A
:1051500091E08385853008F490E031E0340F6DE014
:1051600070E0E32F032E000CFF0BDB01AE1BBF0B27
:10517000A00FB11F8C91890F90E08A3010F080E071
:1051800091E0EE0DFF1D805D8083315051F72111BC
:10519000D3C050CF51E0B2CF5130A1F53F5F832F44
:1051A000821BF801E81BF10987FDF39591E08485E6
:1051B000853008F490E0422F220F550B6DE070E02F
:1051C0003701640E751E032F032E000C110B5801BE
:1051D000A41AB50AB7FC0CC05B01A01AB10AA60C50
:1051E000B71CF501808D890F90E08A3010F091E0B6
:1051F00080E00E0D1F1D805DF8018083315019F78E
:10520000AE8718CF8F5F380F3A303CF541E0F80198
:10521000E31BF10937FDF3958485853008F440E000
:10522000832F330F990B081B190B035F1F4F1816A1
:10523000BCF0E1E0E20FEA0DFB2DF11DA08322504E
:1052400082FEF8CE12160CF0F5CEF501E20FF11D3C
:1052500027FDFA95B0832350F5CF452F3AE0E0CFF4
:10526000F80131918F01340F452F3A3010F0352F6E
:1052700041E0B701680F791F305DFB013083019772
:10528000D6CF90E047E069CF383008F046C0F8014B
:10529000E31BF109B1E08385853008F4B0E0882490
:1052A0008394840E6DE070E0882D082C000C990B1F
:1052B000FB01E81BF90BE00FF11F30813B0FB0E061
:1052C0003A3010F0B1E030E08E0D9F1D305DFC01F2
:1052D00030838A948110E8CF552309F1121614F413
:1052E0008DE28A872E5F33E0822F632F0E94213D5B
:1052F000391B291BA30EB11CF501A083822F6AE084
:105300000E94213D90E3980F9B8790E3920FF6EF68
:105310008F9F900D11249C873ACF47E0BFCF822FFB
:1053200063E00E94213D31E0390FE3CF222309F4ED
:1053300081CE983009F47ECE8A81803309F07ACE0E
:105340002336A9F421E0042E000C550B4F5F5F4F6C
:1053500039E305C08E0D9F1DFC0130832F5F822F26
:10536000022E000C990B48175907A4F763CE81E36E
:105370008A83552379F02150822F6AE00E94213DD3
:1053800090E3980F9B87205DF6EF8F9F200D1124EF
:105390002C8750CE2F5FF0CF0895F894EEEFF1E414
:1053A00011861086128613861486158678940895C1
:1053B0008F708A3010F0895A0895805D0895CF93D8
:1053C000C82F82958F700E94D8290E940A178C2FAF
:1053D0008F700E94D829CF910C940A171F93CF93F6
:1053E000DF9327E0289FE001299FD00D1124C651AB
:1053F000DD4B16E08A9182958F700E94D8290E9419
:105400000A1788818F700E94D8290E940A171150AC
:1054100088F7DF91CF911F9108950F931F93CF933A
:10542000DF938C01EC012E968A918F700E94D8290F
:105430000E940A170C171D07B9F7DF91CF911F9132
:105440000F9108950F931F93CF93DF938C01EC017D
:1054500025968A918F700E94D8290E940A170C17EE
:105460001D07B9F7DF91CF911F910F910895CF9349
:10547000C82F892F0E94D829803311F00E940A1763
:105480008C2F82958F700E94D8290E940A178C2F2A
:105490000E94D829CF910C940A170F931F93CF9392
:1054A000DF93D82F162FC42F82958F700E94D82992
:1054B00000E029E336E04C2F612F0E94F219182FEB
:1054C0008D2F0E94D82929E336E04C2F612F0E94AE
:1054D000F219DF91CF911F910F910895EF92FF92F2
:1054E0000F931F93CF93DF93E82EC62FD42F0E94E4
:1054F0004D2A68E06C0F00E029E336E04D2F8AE387
:105500000E94F219C45F87E0E89E7001112410E048
:1055100000E0F701E01BF10BE751FD4B4D2F6C2F25
:1055200080810E944D2A0F5F1F4FC85F0730110511
:1055300081F7DF91CF911F910F91FF90EF90089528
:10554000909108429730BCF4E0910642F0E0E250BE
:10555000FE4B8083809106428F5F8093064280914C
:105560000642877080930642809108428F5F809345
:10557000084281E0089580E00895F89480910842FF
:105580001816BCF4E0910742F0E0E250FE4B808137
:10559000909107429F5F90930742909107429770C6
:1055A00090930742909108429150909308427894CA
:1055B00008958FEFFCCF8091005E811104C080912F
:1055C000F05D8823D9F08091985D811117C00E9409
:1055D000BD2A8F3F99F0E82FF0E0ED50FD4FE491A8
:1055E000E093874281E08093FB418093985D8091B6
:1055F0007C4290E08093F15D9093F25D08951F925C
:105600000F920FB60F9211240BB60F922F933F9368
:105610004F935F936F937F938F939F93AF93BF93BA
:10562000CF93DF93EF93FF938091995D8F5F80938A
:10563000995D8091995D83708093995D80910C4212
:1056400090910D4286FF0FC08DE192E40E94652289
:10565000882349F080910C4290910D4282608093A2
:105660000C4290930D4280910C4290910D4287FF25
:105670000FC08BE292E40E946522882349F080915A
:105680000C4290910D42886080930C4290930D42A1
:1056900080910C4290910D4292FF19C082E192E4F8
:1056A0000E94652267E172E482E192E40E94AE1FEB
:1056B000882369F082E192E40E94A71F80910C4246
:1056C00090910D42806180930C4290930D428091A5
:1056D0000C428F73D9F08091935D9091945D9062AC
:1056E0008093935D9093945D8091935D9091945D90
:1056F00090618093935D9093945D81E08093005ED0
:105700008091AF40813011F41092AF408091995D4B
:10571000811168C08091AF40823049F08091F35D83
:10572000882329F08091F35D81508093F35D80910F
:1057300076428F5F80937642809176428C330CF470
:1057400051C0C1E0C093B140109276428091754241
:105750008F5F80937542809175428C330CF442C008
:1057600010927542809174428F5F80937442809151
:10577000744288318CF110927442809179428F5F2B
:1057800080937942D09179426091774280917842BA
:105790000E94F31C2D2FDD0F330B8217130694F498
:1057A000C0937942809178428F5F80937842809154
:1057B00078428D303CF0C0937842809177428F5F81
:1057C000809377424091794260917842809177420C
:1057D0000E94D01C80938142809174420E94091DD6
:1057E0008093804281E080935301FF91EF91DF919C
:1057F000CF91BF91AF919F918F917F916F915F9169
:105800004F913F912F910F900BBE0F900FBE0F90B5
:105810001F9018951F920F920FB60F9211242F937D
:105820003F934F938F939F9381E08093B0408091FB
:105830000B42813089F58091094081508093094065
:1058400080910940811128C080917D428093094058
:105850004EB18091EE5D9091EF5D880F991F21E030
:1058600030E04F3F11F430E020E0822B932B809307
:10587000EE5D9093EF5D8091EE5D9091EF5D892BF1
:1058800059F410920B42109202408FEF8FB99DE0B5
:1058900090936B0480936C0481E080930B0A9F913A
:1058A0008F914F913F912F910F900FBE0F901F90AE
:1058B00018958091B140813079F40E9456190E9468
:1058C0005A2763E70E94331A82E00E94361D80E364
:1058D0000E94731D1092B14008958F929F92AF92D3
:1058E000BF92CF92DF92EF92FF920F931F93CF93CD
:1058F000DF938091AF408111A6C0912CC2E08C2E25
:10590000D6E3ED2EDBE0FD2E11E004E7C02E04E02F
:10591000D02E88EDA82E8DE1B82E8091C05D82300A
:10592000F1F58091C1409091C2408093D342909311
:10593000D4429092AD400E942213FC01808180935A
:10594000AC408091D3429091D442209102402111E9
:105950000AC08B3BF0E19F0739F5A0920340B0925B
:105960000440109302400E94CA259C013695279559
:1059700036952795922E70919A5D7093864210927B
:105980009A5D4091C05D423009F414C230F5442361
:10599000C1F1413009F4B4C11092C05D50C0809192
:1059A000D1429091D242C1CF8C3F21E1920729F49C
:1059B000C0920340D0920440D4CF803DE2E19E07E4
:1059C00029F4E0920340F0920440CBCF883CF0E110
:1059D0009F0749F680920240C6CF443009F4FAC1CD
:1059E00008F4EBC14530C1F62091D1423091D2424A
:1059F0002F5F3F4F2093D1423093D24280FDCCCFD6
:105A00008CCF4091D1425091D242FA013196E0932D
:105A1000D142F093D242682F6370623051F163300B
:105A200009F45DC16130E1F0F901FF27EE0FFF1FBE
:105A3000E155FF4F45915491822FFA0109958091CC
:105A4000C05D81116ACFDF91CF911F910F91FF90BF
:105A5000EF90DF90CF90BF90AF909F908F90089580
:105A60006093C05D8093BC5D9093BD5D7093B440C6
:105A7000E6CFC22FC695C695C695D22FD770EFEF49
:105A8000ED0FE73078F4F0E0E85BF24D0C94793DEF
:105A9000992D822D4F2D872D902D932D962D2DE014
:105AA00060E005C00E942213FC016081262F209334
:105AB000965DC150CF3108F03EC0EC2FF0E0ED59BB
:105AC000F24D0C94793DA12DA52DA92DB12DB92D07
:105AD000BD2DC32DC92DCF2DD72DDB2DE12DEB2DC8
:105AE000002E052E0A2E102E162E1E2E292E272EA3
:105AF000302E382E3E2E472E4C2E522E562E5C2EF9
:105B0000602E642E0E942213FC012081C9CF609177
:105B1000CE422091CF4226170CF0C9CF2DE0C7CF3F
:105B200022E062E0C4CF2CE063E0C1CF2DE06DE065
:105B3000BECF22E0B5CF422F88E892E40E946A13DC
:105B40007ECF422F86E992E4F9CF422F84EA92E495
:105B5000F5CF462F66E972E488E892E40E94731359
:105B60006ECF462F68E872E486E992E40E945913EA
:105B700066CF462F64EA72E4EFCF462F66E972E4FF
:105B800084EA92E4F3CF462F64EA72E486E992E471
:105B9000E5CF462F64EA72E488E892E4E7CF462F27
:105BA00066E972E488E892E40E94861348CF462FA3
:105BB00064EA72E4F7CF10939A5D462F70E060E0DC
:105BC000F1CF022F262F46E952E468E872E4CB01B8
:105BD0000E94B21334CF10939A5DD73061F4809154
:105BE000E0428A3041F4809195428B3020F0895018
:105BF0008093954224CF022F262F50E040E0E5CF3E
:105C0000022F262F44EA52E4E0CF462F64EA72E4E2
:105C1000CB01CACF462F68E872E484EA92E4C4CF8D
:105C200010939A5D462F70E060E0F7CF022F262F89
:105C300044EA52E468E872E4CA01CACF10939A5D5C
:105C4000022F262F50E040E064EA72E4C0CF1093A8
:105C50009A5D022F262F44EA52E470E060E0ECCF18
:105C6000462F70E060E086E992E40E94F413E7CEEC
:105C7000462F70E060E084EA92E4F7CF022F262FEF
:105C800044EA52E468E872E490E080E0A1CF022F99
:105C9000262F46E952E4F6CF462F70E060E088E810
:105CA00092E4E3CF462F64EA72E4F9CF422F88E80A
:105CB00092E40E94E513C3CE422F86E992E4F9CF25
:105CC000422F84EA92E4F5CFC8E8D2E4C20FD11D96
:105CD000261B4A9149832A95E1F71882B0CE822F7C
:105CE00086958F7327FD805421702713ACCE480F03
:105CF000511D87FD5A954093D1425093D2429FCE79
:105D00004091D1425091D2424F5F5F4F4093D14278
:105D10005093D2421092C05D6091B4409C012170BA
:105D200033276217130609F08ECE6091BC5D709127
:105D3000BD5D76956795769567959C01E6E0220FA7
:105D4000331FEA95E1F72227262B372B81FF05C069
:105D50002093D1423093D24272CE8091D942909119
:105D6000DA428093DB429093DC428091D74290915B
:105D7000D8428093D9429093DA428091D542909153
:105D8000D6428093D7429093D8424093D5425093C5
:105D9000D6422093D1423093D242C9010E94CA25F3
:105DA000892B09F04CCE0E9414148093D142909319
:105DB000D24245CE0E949D1642CE2091D1423091D2
:105DC000D2422F5F3F4F2093D1423093D2420E9464
:105DD0009D1635CE882351F08091D1429091D242C8
:105DE00001968093D1429093D242D6CD1092D14267
:105DF0001092D2428091F05D882319F01093AF4049
:105E0000CBCD1092005E10939A5D8092AF40C4CDCE
:105E100020918242022E000C330B2F5F3F4FAC01CA
:105E2000249FC001259F900D349F900D1124019750
:105E300008F40895EFECF7E03197F1F700C00000A7
:105E4000F6CF1F93CF93DF9383E090E00E94082F5B
:105E5000C0E4D4E018E01E8383E090E00E94082FA5
:105E60001D8381E090E0DF91CF911F910C94082F6A
:105E7000EF92FF921F93CF93DF930E94212FC0EDEB
:105E8000D3E2FE0114911123F1F031968491229610
:105E90008F3F29F484E690E00E94082FF2CF84918E
:105EA0000E9403197E01F7018FEFE81AF80A8E2D80
:105EB0008C1B811720F01150C10FD11DE2CF8491AE
:105EC0000E94FC18F0CFDF91CF911F91FF90EF90CF
:105ED0000895A09182420A2E000CBB0B119620E07F
:105EE00032E14AE750E00E94943D0E941C3C20E0D1
:105EF00030E040E852E40E94A83C20E030E046E177
:105F000059E40E94793B20E030E040E05FE30E94EA
:105F10000D3B0E94EB3BE0E2F8E06087718783E095
:105F200087838681806C868380E8858384E690E021
:105F30000E94082F8CE00C940A170F931F93CF93A5
:105F4000DF93109260090E94692F8AE00E940A176D
:105F50008AE00E940A1780E50E940A1788E50E94DD
:105F60000A1784E30E940A1781E30E940A178AE055
:105F70000E940A17D0E0C0E0CE010E94BB26882311
:105F8000E1F0CE01C031D10508F0C0960E94372A59
:105F900080E20E940A1710E000E0C8018C0F9D1FEC
:105FA0000E94EE2980E20E940A170F5F1F4F043003
:105FB000110599F78AE00E940A172496C03D23E054
:105FC000D207D1F681E40E940A178AE30E940A17D9
:105FD00080E20E940A1788E892E40E940D2A80E27B
:105FE0000E940A1780E20E940A1782E40E940A17A0
:105FF0008AE30E940A1780E20E940A1786E992E467
:106000000E940D2A80E20E940A1780E20E940A176D
:1060100083E40E940A178AE30E940A1780E20E9422
:106020000A1784EA92E40E940D2A8AE00E940A1765
:1060300083E50E940A178AE30E940A1780E20E9401
:106040000A17CDE0D0E001E010E02091E14230916C
:10605000E242C8010C2E02C0880F991F0A94E2F791
:1060600082239323892B09F060C080E30E940A17E2
:10607000219758F78AE00E940A178DE40E940A17B8
:106080008AE30E940A1780E20E940A1782EB92E4D8
:106090000E940D2A80E20E940A1780E20E940A17DD
:1060A0008EE40E940A178AE30E940A1780E20E9487
:1060B0000A1780EC92E40E940D2A80E20E940A17DF
:1060C00080E20E940A1787E40E940A178AE30E946E
:1060D0000A1780E20E940A178091DE428F700E94A8
:1060E000D8290E940A178091DD428F700E94D8291A
:1060F0000E940A178AE00E940A178AE090E40E9430
:10610000982684E00E940A179FEF20E742E0915012
:1061100020404040E1F700C0000081E38093600927
:10612000DF91CF911F910F91089581E39FCF20912F
:106130008242022E000C330B2F5F3F4FAC01249F95
:10614000C001259F900D349F900D1124019708F4F4
:10615000089552E05A95F1F700C0F8CF1092600907
:106160000E94692F8AE00E940A178AE00E940A179B
:1061700080E190E40E9498268091D2420E94DF291B
:106180008091D1420E94DF298AE00E940A1781E1B2
:1061900090E40E94982684EA92E40E940D2A8AE004
:1061A0000E940A1784E190E40E9498268091935DF2
:1061B0009091945D892F0E94DF298091935D909149
:1061C000945D0E94DF2980911C42811166C089E1A3
:1061D00090E40E9498268AE00E940A178BE290E4DD
:1061E0000E9498268DE192E40E940D2A82E390E4B9
:1061F0000E94982689E392E40E940D2A8AE390E4A3
:106200000E94982685E592E40E940D2A8AE00E9469
:106210000A1782E490E40E9498268BE292E40E949E
:106220000D2A89E490E40E94982687E492E40E9473
:106230000D2A81E590E40E94982683E692E40E946C
:106240000D2A8AE00E940A1789E590E40E949826A8
:1062500087E192E40E94222A81E690E40E94982637
:1062600082E192E40E94222A8BE690E40E94982622
:1062700080910D420E94DF2980910C420E94DF290B
:106280008AE00E940A170E94642684EF91E00E942F
:10629000973081E380936009089582E290E499CF7A
:1062A0001F920F920FB60F9211240BB60F92BF924E
:1062B000CF92DF92EF92FF920F931F932F933F9312
:1062C0004F935F936F937F938F939F93AF93BF93FE
:1062D000CF93DF93EF93FF9388E080936B048FEF6E
:1062E00080936C04DFB18FB9DD2309F487C0ED2EF4
:1062F000F12CC70101978D239F21892B09F07EC0C6
:106300008091AF408230B9F110E000E08FE1B82E0B
:10631000CC24C394D12CC02FB0920204C601002E0D
:1063200001C0880F0A94EAF78093010485E090E0A9
:106330000E9497308EB190E0809590958E219F219C
:10634000892B31F40F5F1F4F0530110521F7C5E090
:1063500080E0D69571F4CC0FCC0FCC0FC80FC832AB
:1063600058F08FEF8FB99DE090936B0480936C048D
:1063700020C08F5FEECFC7E0D6E910EA809172426D
:106380008111109307048EE591E00E949730D1505F
:10639000A9F78C2F0E94A02A882359F081E08093CE
:1063A0000B4224E632E32093034030930440809371
:1063B00002408FE1809301041092AF4080917142BE
:1063C0008093F35DFF91EF91DF91CF91BF91AF91FA
:1063D0009F918F917F916F915F914F913F912F91FD
:1063E0001F910F91FF90EF90DF90CF90BF900F9093
:1063F0000BBE0F900FBE0F901F9018958FEF8FB9A7
:106400009DE090936B0480936C04DCCF8130A9F005
:1064100028F08230F9F0833031F1089588ED94E16D
:1064200084BF909368008AE990E08093260A909355
:10643000270A8AE080930206089588ED9CE184BFD4
:106440009093680085E391E08093260A9093270A51
:106450008CE0F0CF88ED25E230E084BF2093680027
:1064600080ED91E0F1CF88ED2DE230E084BF209304
:1064700068008BE692E08093260A9093270A8DE0CD
:10648000D9CFFF920F931F93CF93DF9380918342D5
:10649000823099F1833069F0813009F06FC000E0FB
:1064A00029E336E046E061E089E50E94F21982E0E6
:1064B0001DC000E029E336E042E061E084E50E948F
:1064C000F21929E336E044E061E08AE50E94F2191E
:1064D00029E336E046E061E089E50E94F21982E0B6
:1064E0000E94CC2781E00E94CC2780E0DF91CF91F1
:1064F0001F910F91FF900C94CC2760E085E00E94E3
:10650000301960E086E00E94301900E029E336E0AF
:1065100046E061E081E40E94F219C0E00C2F0C2EED
:10652000000C110BF801EA5FFC4B8081811111C056
:106530008F01DC2F8AE0F82EC1111EC049E965E009
:1065400083E790E4DF91CF911F910F91FF900C941E
:106550004F1CCF5FE3CFF80182918F01803408F0A8
:1065600080546C2F6D1B6F9D602D11246B5F2FEF7E
:1065700045E00E94101CD1501D166CF3DF91CF91A5
:106580001F910F91FF9008952F923F924F925F922B
:106590006F927F928F929F92AF92BF92CF92DF9233
:1065A000EF92FF920F931F93CF93DF93CDB7DEB798
:1065B000A397CDBFDEBF5C016A01E62EF12CCA01B4
:1065C0004096E816F90608F046C0E41AF50ABE013E
:1065D0006F5F7F4FC6010E9424278EE58C831D824A
:1065E00067E1CE0101960E94B919BE016F5F7F4F2E
:1065F000C60101978E0D9F1D0E94242767E2CE01E0
:1066000001960E94B919AC0CBD1C512C4E012AE018
:10661000820E911C8AE0482E9DE2392E21E4222E22
:10662000652C712C6E147F04D0F0A396CDBFDEBF15
:10663000DF91CF911F910F91FF90EF90DF90CF905E
:10664000BF90AF909F908F907F906F905F904F9092
:106650003F902F90089530E1E32EF12CB8CFC30185
:106660008A0D9B1D27E0289FF001299FF00D112422
:10667000E751FD4B2081203189F529828CE48A8302
:1066800090E59B8388E48C832D821E82152D1695C0
:106690001F5F50FC57C0BE01615E7F4FC3018C0D70
:1066A0009D1D0E9424278AE38AA31BA220E0412F7C
:1066B00061E0CE014F960E94531B20E0412F61E123
:1066C000CE0101960E94531B00E029E336E0412FE2
:1066D00065E48CE70E94F2195394A2CFBE016F5E6D
:1066E0007F4F0E94AF278E8D882331F139828D8DA7
:1066F000805D8A838EE28B83FE017196DE011496A3
:106700008385805D8D933197E815F905C9F79A89DE
:106710008989949D800D11249B89992381F03B8662
:1067200094E6981B892F642D0E94153D805D8C870F
:10673000905D9D871E86AACF20E22983D8CF2BE2C9
:106740002B87F1CF20E0412F69E4CE0101960E9412
:10675000531BC2CF2F923F924F925F926F927F92C4
:106760008F929F92AF92BF92CF92DF92EF92FF9261
:106770000F931F93CF93DF93CDB7DEB7A597CDBF10
:10678000DEBF68EE74E2CE0141960E946B3E0E942D
:10679000A91C0E94561963E0CE0141960E94B919C6
:1067A00010E00E941D1B1C3058F5E12FF0E0E5526F
:1067B000FC4C0C94793DE73346346A342C3535353E
:1067C000513503357E342E34C83487347F3560E04C
:1067D00083ED95E20E94A11A61E08AEB95E20E94A6
:1067E000A11A62E08AEC95E20E94A11A63E085EBAF
:1067F00095E20E94A11A64E086EA95E20E94A11A3D
:1068000080915000897F8460809350008091500077
:106810008160809350008895809150008E7F809396
:1068200050008091F35D81113DC287E00E94A02A53
:10683000A596CDBFDEBFDF91CF911F910F91FF9045
:10684000EF90DF90CF90BF90AF909F908F907F9010
:106850006F905F904F903F902F90089560E08EEC86
:1068600095E20E94A11A61E08FEA95E20E94A11AC6
:1068700062E084EC95E20E94A11A63E08FEB95E25E
:106880000E94A11A64E08BEA95E2B8CF60E083E150
:1068900095E20E94A11A61E085E195E20E94A11AA9
:1068A00062E088E195E20E94A11A63E08BE195E243
:1068B0000E94A11A64E08BEA95E20E94A11A8091DD
:1068C00083420E94CD1A0E94671F0E9441320E949B
:1068D000A81E96CF60E081E995E20E94A11A61E0CE
:1068E00087E995E20E94A11A64E08BEA95E20E9492
:1068F000A11A809172420E94CD1A82CF60E08EE090
:1069000095E20E94A11A61E088E095E2B9CF64E0C7
:106910008BEA95E20E94A11A68EB74E2CE014196DF
:106920000E946B3EABE46A2EA3E47A2E412C01E078
:10693000542CD12CF7E08F2E912CBE016F5F7F4F2E
:10694000852D0E941327F301808190E0082C02C05E
:10695000959587950A94E2F72FEF80FF20E0402F6E
:106960006D2DCE0101960E94531B5394F1E08F1AB6
:10697000910820E1D20E3FEF83169306F1F60F5FE8
:1069800088E0480E91E0691A7108083089F638CF1E
:10699000E0E1EE16F1042CF060E08EEF94E20E944C
:1069A000A11A950121503109C7010F96821793074B
:1069B00028F461E083E095E20E94A11A64E08BEA8A
:1069C00095E20E94A11A6CEA74E2CE0101960E943F
:1069D0006B3E6AE5CE0101960E94B919BE016F5F58
:1069E0007F4FC5010E9424276EE6CE0101960E94CA
:1069F000B919A114B10409F403CFA7016A2DC1018B
:106A00000E94C432FDCE60E085E795E20E94A11AA3
:106A100061E080E795E20E94A11A62E08BE695E2D0
:106A20000E94A11A63E085E695E20E94A11A64E043
:106A30008BEA95E20E94A11A80917142883751F049
:106A4000803F21F08C3321F480E055CF82E053CF9A
:106A500083E051CF81E04FCF60E081EA95E20E9470
:106A6000A11A61E08CE995E20BCF60E08CE895E239
:106A70000E94A11A61E086E895E20E94A11A62E0F4
:106A800080E895E20E94A11A63E08AE795E20E94FD
:106A9000A11A64E08BEA95E20E94A11A80918242D9
:106AA0002ACF20E041E064E287E595E20E94741B72
:106AB00020E046E061E08EE495E20E94741BBE0196
:106AC0006F5F7F4F809108400E94492720E046E099
:106AD00061E1CE0101960E94531B20E047E061E096
:106AE0008CE395E20E94741B20E048E061E080E2C4
:106AF00095E20E94741B60E089EF94E2C1CE64E0ED
:106B00008BEA95E20E94A11A60E0C1108AC08DEE66
:106B100094E20E94A11A20E041E065E481EA94E257
:106B20000E94741B20E042E065E48BE994E20E943D
:106B3000741B20E043E065E483E994E20E94741B47
:106B400020E044E065E48BE894E20E94741B20E0BE
:106B500045E065E485E894E20E94741B20E046E08D
:106B600065E487E794E20E94741B20E047E065E457
:106B700081E794E20E94741B20E048E065E48BE624
:106B800094E20E94741BF0E8CF9EC00111249C0186
:106B90002D533F4B4901D12C5C2C550C550C550CF9
:106BA0005A94D394852D8D0D0E94D82900E029E3B5
:106BB00036E04D2D61E00E94F219340136E03DA32C
:106BC000412C00E029E336E04D2D6DA18CE70E94B9
:106BD000F21984E0481691F06DA1695FF30180819C
:106BE0009181A281B381892B8A2B8B2B09F454C00C
:106BF00029E336E04D2D8AE20E94F2194394FDA16B
:106C0000F25FFDA324E0620E711C35E04312D9CF80
:106C100080E1880E911C98E0D912C3CF81E0C8268C
:106C2000EFCD83EF94E20E94A11A20E041E065E4F9
:106C300082E694E20E94741B20E042E065E483E572
:106C400094E20E94741B20E043E065E48BE494E24C
:106C50000E94741B20E044E065E483E494E20E9417
:106C6000741B20E045E065E48DE394E20E94741B10
:106C700020E046E065E487E394E20E94741B20E094
:106C800047E065E48CE294E20E94741B20E048E057
:106C900065E486E294E275CF00E029E336E04D2D0D
:106CA0008DE2AACF80910B42882309F4A9CD0E94DE
:106CB000BD2A082F80910B428130C1F00E94CD295E
:106CC0000E94A91C1C3000F5E12FF0E0E659F94CB8
:106CD0000C94793D7B36DD36FB369737D738F9385B
:106CE00067371037B03644374837083982E390E0C9
:106CF0000E94082FDFCF003159F1E8F4002309F496
:106D00008AC2083009F47DC00E94561963E0CE01A2
:106D100041960E94B9190B7F033009F042CD81E002
:106D20008093B1400E94592C0E94341F0E94671F1B
:106D30000E9441327DCD083109F4ACC0003221F708
:106D40006DED74E2CE0141960E946B3E11E0DCCF06
:106D500069EC74E2CE0141960E946B3E13E0D4CF01
:106D6000003119F168F4002309F460C0083061F6BD
:106D70006EEB74E2CE0141960E946B3E15E0C4CFEB
:106D8000083159F0003209F0BFCF68ED74E2CE014E
:106D900041960E946B3E12E0B7CF6DEC74E2CE01DB
:106DA00041960E946B3E16E0AFCF63EC74E2CE01D9
:106DB00041960E946B3E14E0A7CF0031C1F060F411
:106DC0000023B9F083E0083079F068EE74E2CE0178
:106DD00041960E946B3E98CF083129F00032A9F706
:106DE00010928342F2CF81E080938342EECF82E023
:106DF000FBCF10E0EACF083179F0003251F00111F9
:106E000083CF62EE74E2CE0141960E946B3E18E0A1
:106E10007BCF1092724278CF81E08093724274CF20
:106E2000083151F1003251F001116ECF68EE74E279
:106E3000CE0141960E946B3E10E066CF62EB74E299
:106E4000CE0141960E946B3E80914043E0E18E9FCF
:106E5000C001112420913F4322952F70822BA12C39
:106E6000E2E0BE2EA81AB90A1C01F0E32F1A31087D
:106E7000F12CE12C19E048CF68EB74E2CE01419689
:106E80000E946B3E1AE040CF0831A1F0003251F071
:106E900001113ACF63ED74E2CE0141960E946B3E40
:106EA00017E032CF20E1E21AF108F7FE2DCFF12CE6
:106EB000E12C2ACF950121503109C7010F96821785
:106EC000930708F021CF30E1E30EF11C1DCF003114
:106ED000D9F048F4002319F10830D1F080917142C3
:106EE0008093F35D11CF083159F00032B9F78CE38C
:106EF0008093714280914643877F80934643EECFD3
:106F000098E790937142F6CFE0EFE0937142F2CFB1
:106F10008FEF80937142809146438860EECF62EE9E
:106F200074E2CE0141960E946B3E18E0D7CF083143
:106F300031F0003209F078CF0E949D2FE5CE20E09D
:106F400044E062E089E790E40E94531B85E0E7EAB1
:106F5000F0E4DE01909601900D928A95E1F710928F
:106F600060090E94692F0E9423178AE00E940A1775
:106F700086E890E40E94982684E00E940A170E9406
:106F80003F261092975DF12CE12C7724739434E026
:106F9000932E6E01F0E2CF0ED11C45E0642E50E33B
:106FA000852E62E0462E73E0572E8091975D8230E9
:106FB000C1F048F4882309F441C0813009F469C064
:106FC0009092975D99C0833009F4E4C08530C1F791
:106FD0008FE990E40E9498260E9423170E94551E74
:106FE000EFCF27E02E9D80012F9D100D1124085713
:106FF0001D4B24E0322E85E0A82EB12C0E941D26C8
:10700000282E229490EF29220E941D26F501E45A91
:10701000FF4FE00FF11F8229808381E0A81AB10899
:107020009EEFA9169FEFB90649F73A94095F1F4FE3
:107030003110E1CFE4E0EE0EF11CA5C010E080912C
:10704000D35D882359F00E94EC16F601E10FF11D83
:107050009081891711F01230B8F41F5F0E94BD2A89
:107060008F3FA1F06092975D8091975D853009F424
:1070700043C00E94EC168A3021F00E94BD2A8F3F47
:10708000C1F37092975D38C010E0E8CF1430B9F6C4
:10709000EBCF88A289A28AA210E000E08091D35DA4
:1070A000882361F00E94EC16182F80ED810F8A3042
:1070B000D0F5F601E00FF11D10830F5F0E94BD2A8D
:1070C0008F3F09F445C06092975D8091975D833052
:1070D00099F00C0D1D2D111DB12CA12CF12CE12CC2
:1070E0000C151D05C9F520E1E216F10418F030E396
:1070F000E31AF1084092975D8091975D843009F022
:1071000054CF0E940A17FFEF29E638E1F1502040E2
:107110003040E1F700C0000081E3809360090E94E5
:10712000A91C83E083CB8FE9810F863010F28FEBAF
:10713000810F863038F4F601E00FF11D80E2810FF7
:107140008083BBCF1A3309F0B9CF5092975DB6CF89
:10715000103209F0A3CFB9CFF80182918F010E94BC
:10716000392690E00A2C02C0880F991F0A94E2F792
:10717000E82AF92AF4E0AF0EB11CB2CF0E94BD2A72
:107180008F3F09F07ECF0E94EC168A30B9F779CF95
:107190000E94EC168091D35D8111FACF0E94551E9A
:1071A0009092975D8BE990E40E949826A5CF0031DC
:1071B000B1F050F40023A9F083E0083069F0809129
:1071C00082420E940632A0CD083129F00032B9F780
:1071D00010928242F4CF81E080938242F0CF82E02D
:1071E000FBCF62EE74E2CE0141960E946B3E18E046
:1071F000E6CF002309F405CE003209F085CD67EA19
:1072000074E2CE0141960E946B3EC12C1BE07CCD06
:1072100001117ACDADCD10E003E076CD1F93CF9371
:10722000DF9310928242809182420E9406328091C6
:107230007C008E7F98ED94BF80937C0080916300EA
:1072400083FDFCCF80917C0098ED8B7F94BF809371
:107250007C0080917C00816094BF80937C00809151
:1072600041018111FCCF82E080934701D1E0D093AE
:10727000520181E680935001D0930A0A1092010ACC
:107280008091090A8E7F8093090A86E08093000A24
:107290008091000A81608093000ACFEFC0930104BF
:1072A000C093060480E8809305040E94EB18C09305
:1072B00062048DE080936B04C0936C04CFB910928C
:1072C000A000C5E0C093A40080E28093850689E415
:1072D00080930806109200060E94CD2987E38093D0
:1072E00076428BE380937542109274428CE08093D7
:1072F0008042C093794213E01093784285E18093F5
:1073000077424091794260917842809177420E9421
:10731000D01C80938142D093B1401093834210924D
:10732000995D109273421092724288E78093714285
:1073300084E680937A428CE180937B4284E180935F
:107340007C42C0937D4210927F420E945A278093D4
:107350000840809171428093F35D7894DF91CF91E2
:107360001F9108950E940E3984E690E00E94082F34
:107370000E94382F0E94592C0E94413288EC809341
:107380007E420E9477250E94CD290E9423170E94E9
:10739000551EC1E01EE108E0DFEF8DE0F82E90E819
:1073A000E92E8091AF40813009F4E6C008F454C062
:1073B0008230B9F7109202400E94CD290E94A91C88
:1073C0000E94CA1C1093050400936B04D0936C04B4
:1073D000F0927704DFB980915000897F84608093B8
:1073E000500080915000816080935000889580917A
:1073F00050008E7F809350008091AF40823059F3CF
:107400000E94CD1CD0930604E092050482E390E034
:107410000E94082F749904C00E9423170E94551ED1
:1074200080910B42813009F4A2C0C093005E10929B
:10743000D1421092D2421092C05DC0939A5D1092D8
:10744000985DC093F05D0E94341F0E94BD1E0E9493
:107450004132C093B14085C080917A4290E08093E0
:10746000B2409093B3408091B040813021F0809140
:10747000024081114AC08091985D811116C00E941E
:10748000BD2A8F3F91F0E82FF0E0ED50FD4FE491E1
:10749000E0938742C093FB41C093985D80917C420A
:1074A00090E08093F15D9093F25D0E946D2C80914D
:1074B0000240813061F48091034090910440009734
:1074C00009F452C001978093034090930440809147
:1074D0000540813079F480917B422091B240309117
:1074E000B340820F932F911D8093B2409093B3408D
:1074F000109205408091B2409091B34001978093E3
:10750000B2409093B3401092B0408091B2409091BD
:10751000B340892B09F0A7CF809106408823B9F0AA
:107520002091EC5D3091ED5D8091004090910140A3
:107530002817390751F00E94BD1E8091EC5D909193
:10754000ED5D809300409093014010920640809141
:107550000740882331F00E94341F0E94671F109259
:1075600007400E94592C1DCF10920240B0CF82E3F9
:1075700090E00E94082F54CF109202400E944132A6
:107580000E94341F0E94671F80915000897F846091
:1075900080935000809150008160809350008895C6
:1075A000809150008E7F809350000E94592C8091D2
:1075B000F35D811109C08091464383FD05C087E0DA
:1075C0000E94A02A1092AF4080910B428130B1F40A
:1075D0001092AF400E94BD2A8330D9F480910B42B3
:1075E000813091F00E94AA3360E089E00E94301956
:1075F00060E08AE00E9430190E94BD1E8091AF4079
:10760000813009F4C1CFCDCE82E390E00E94082FF3
:10761000E5CF0E94A02AF2CF5058BB27AA270E948C
:10762000243B0C946E3C0E94603C38F00E94673C06
:1076300020F039F49F3F19F426F40C945D3C0EF4CD
:10764000E095E7FB0C94573CE92F0E947F3C58F3F0
:10765000BA17620773078407950720F079F4A6F537
:107660000C94A13C0EF4E0950B2EBA2FA02D0B012B
:10767000B90190010C01CA01A0011124FF27591B77
:1076800099F0593F50F4503E68F11A16F040A22F7D
:10769000232F342F4427585FF3CF469537952795EE
:1076A000A795F0405395C9F77EF41F16BA0B620BED
:1076B000730B840BBAF09150A1F0FF0FBB1F661F34
:1076C000771F881FC2F70EC0BA0F621F731F841F77
:1076D00048F4879577956795B795F7959E3F08F09D
:1076E000B0CF9395880F08F09927EE0F979587955F
:1076F00008950E948D3B0C946E3C0E94673C58F0AC
:107700000E94603C40F029F45F3F29F00C94573C04
:1077100051110C94A23C0C945D3C0E947F3C68F398
:107720009923B1F3552391F3951B550BBB27AA273A
:1077300062177307840738F09F5F5F4F220F331F74
:10774000441FAA1FA9F335D00E2E3AF0E0E832D03C
:1077500091505040E695001CCAF72BD0FE2F29D03F
:10776000660F771F881FBB1F261737074807AB0711
:10777000B0E809F0BB0B802DBF01FF2793585F4F86
:107780003AF09E3F510578F00C94573C0C94A23C83
:107790005F3FE4F3983ED4F3869577956795B79568
:1077A000F7959F5FC9F7880F911D9695879597F973
:1077B0000895E1E0660F771F881FBB1F62177307EC
:1077C0008407BA0720F0621B730B840BBA0BEE1F01
:1077D00088F7E09508950E94873C88F09F5798F0BD
:1077E000B92F9927B751B0F0E1F0660F771F881FC6
:1077F000991F1AF0BA95C9F714C0B13091F00E94E0
:10780000A13CB1E008950C94A13C672F782F882704
:10781000B85F39F0B93FCCF3869577956795B39506
:10782000D9F73EF490958095709561957F4F8F4F75
:107830009F4F0895E89409C097FB3EF4909580957A
:10784000709561957F4F8F4F9F4F9923A9F0F92F26
:1078500096E9BB279395F695879577956795B795A4
:10786000F111F8CFFAF4BB0F11F460FF1BC06F5F8A
:107870007F4F8F4F9F4F16C0882311F096E911C09C
:10788000772321F09EE8872F762F05C0662371F0BD
:1078900096E8862F70E060E02AF09A95660F771FD1
:1078A000881FDAF7880F9695879597F9089597F9C5
:1078B0009F6780E870E060E008959FEF80EC089596
:1078C00000240A94161617061806090608950024BF
:1078D0000A9412161306140605060895092E039439
:1078E000000C11F4882352F0BB0F40F4BF2B11F4AD
:1078F00060FF04C06F5F7F4F8F4F9F4F089557FD0C
:107900009058440F551F59F05F3F71F04795880F0D
:1079100097FB991F61F09F3F79F0879508951216A4
:1079200013061406551FF2CF4695F1DF08C0161650
:1079300017061806991FF1CF869571056105089401
:107940000895E894BB2766277727CB0197F9089518
:107950000E94BB3C0C946E3C0E94603C38F00E943C
:10796000673C20F0952311F00C94573C0C945D3C3F
:1079700011240C94A23C0E947F3C70F3959FC1F3AC
:10798000950F50E0551F629FF001729FBB27F00DCD
:10799000B11D639FAA27F00DB11DAA1F649F662722
:1079A000B00DA11D661F829F2227B00DA11D621F71
:1079B000739FB00DA11D621F839FA00D611D221F2B
:1079C000749F3327A00D611D231F849F600D211D0F
:1079D000822F762F6A2F11249F5750409AF0F1F092
:1079E00088234AF0EE0FFF1FBB1F661F771F881FFB
:1079F00091505040A9F79E3F510580F00C94573CA0
:107A00000C94A23C5F3FE4F3983ED4F386957795BF
:107A10006795B795F795E7959F5FC1F7FE2B880FA0
:107A2000911D9695879597F90895991B79E004C063
:107A3000991F961708F0961B881F7A95C9F78095AD
:107A4000089587FB082E062687FD819567FD6195C1
:107A50000E94153D0EF4919507FC81950895AA1B8F
:107A6000BB1B51E107C0AA1FBB1FA617B70710F029
:107A7000A61BB70B881F991F5A95A9F7809590955B
:107A8000BC01CD01089597FB072E16F4009407D092
:107A900077FD09D00E942F3D07FC05D03EF490955C
:107AA00081959F4F0895709561957F4F0895A1E24C
:107AB0001A2EAA1BBB1BFD010DC0AA1FBB1FEE1F68
:107AC000FF1FA217B307E407F50720F0A21BB30BB3
:107AD000E40BF50B661F771F881F991F1A9469F72F
:107AE00060957095809590959B01AC01BD01CF018B
:107AF0000895EE0FFF1F0024001C0BBE0790F691A7
:107B0000E02D09940E945C3EB7FF0895821B930B01
:107B100008950E945C3EA59F900DB49F900DA49F78
:107B2000800D911D11240895B7FF0C94893D0E948A
:107B3000893D821B930B0895DF93CF931F930F937F
:107B40009A9DF02D219FF00D8B9DF00D8A9DE02DCB
:107B5000F10D039FF00D029FE00DF11D4E9DE00D14
:107B6000F11D5E9DF00D4F9DF00D7F936F93BF92C1
:107B7000AF925F934F93D5010E945C3E8B01AC01A5
:107B8000D7010E945C3EEB01E80FF91FD6010E946D
:107B9000EB3D2F913F91D6010E945C3EC60FD71F4F
:107BA000E81FF91FAF91BF910E94EB3D2F913F91CC
:107BB0000E945C3EC60FD71FE81FF91FD6010E9426
:107BC0005C3EE60FF71F9801BE01CF010F911F9198
:107BD000CF91DF9108950E945C3E460F571FC81F4A
:107BE000D91F08F431960895689401C0E8948F92E3
:107BF0009F92CF93DF930E94023EDF91CF919F909F
:107C00008F90089588249924F401E401B0E49F93AF
:107C1000AA279A158B049C04ED05FE05CF05D00715
:107C2000A10798F4AD2FDC2FCF2FFE2FE92D982C34
:107C3000892E982F872F762F652F542F432F322F81
:107C40002227B85031F7BF9127C01B2EBF91BB2709
:107C5000220F331F441F551F661F771F881F991F50
:107C6000881C991CEE1FFF1FCC1FDD1FAA1FBB1F06
:107C70008A149B04EC05FD05CE05DF05A007B107BE
:107C800048F08A189B08EC09FD09CE09DF09A00B12
:107C9000B10B21601A94E1F62EF49401AF01BE01FC
:107CA000CD01000C08952A0D3B1D4C1D5D1D6E1D60
:107CB0007F1D801F911F0895A29FB001B39FC00137
:107CC000A39F700D811D1124911DB29F700D811D08
:107CD0001124911D0895FB01DC0105900D920020F7
:107CE000E1F70895DC0101C06D9341505040E0F789
:067CF0000895F894FFCF97
:107CF600FF0001C8000101011E05454F460A0A00A2
:107D060050433D002046493D002054696D65723D53
:107D160041002054696D65723D4200434C4B5F4102
:107D26003A0020414C4D5F413A00205343525F4197
:107D36003A00434C4B5F423A0020414C4D5F423A79
:107D460000205343525F423A00494E545F54563D19
:107D56000020494E545F434E543D0020544D525F1F
:107D6600533D00424C414E4B00726573746F72690D
:107D76006E672E2E2E0057616974696E6720666FD6
:107D86007220646174612E2E2E0A004F4B0A004544
:0C7D960052524F52210A00505834310064
:107DA20000F8615044FE1348260E7676B5A3D91C1E
:107DB20078D88484D88C1326F046F009C886E64B1E
:107DC200309EA62BA058F142CC2766EBA3D91C7893
:107DD20058203C56069CE21B4EAB3012664761C8E7
:107DE2006686A568E330C4064FC64ED0A646263C3A
:107DF200A3E6761C4E906AC6FB303162276A13A650
:107E020062AA3C26048C2B08A07E60585D1C98BC9C
:107E12009CE22B0602A2E6C602A23003622F1C429B
:107E2200136230088C270C237B0C134630555EFC02
:107E320006BC30E61BF61B2E03068C2FC16813C34B
:107E4200A60EA05A7C1AFAFAFAFA56233C3AFCEE2B
:107E52001A46BC26260E55C4604C61008859C87863
:107E620028B86898A859C4EA005ABC1AB0303AE651
:107E72002366DF461AE0BDD065F04C2FA18002DBFD
:107E8200CC3F4E70B8584C7BCC6795A43C0A59A4A1
:107E9200E5A4D88C1744A180FD188A8514064E707B
:107EA200CA685878A6C6026A6DCCB05E3C062B5DE5
:107EB200C4C830DA7004B07C0E01D0EDA4AE3C66CA
:107EC2007F7098AE59A48D8CAE7C6606FC58430434
:107ED200987C1666C3084E70980E78061BA66878C2
:107EE2000E59A430C08D8C4DA4468D8C4E5870789E
:107EF2000E4C23C4BD8C783C667BEDA4D884D88D0F
:107F02008C29A429A4AE0E584E70780EB8BC5884A1
:107F1200E0DCA0DC1050121C8AE5A43C5CF2CB7EB3
:107F22000F02FF1C8A4DA4EDA47C6A22D398AA6991
:107F32008C0A588C574DA459A4468D8C980A29A4B2
:107F42001B1C6AF5A89B623C5888821B59A4468D6B
:107F52008C42D762101C021F023BA666700A4EF0CA
:107F620098AA698C7038989C50F09806467078A64A
:107F7200682E063B6670EEF0EECB4924F85A5EE8B6
:107F820030BF2684A80E78AE66CB70380E4670AE2F
:107F92003E8B1C8C137CEA330EFDBC95BCB88C1F47
:107FA200884B781C0A29A429A4B8AAA8A1801C3944
:107FB20088E68F0C2F59C4F0000DFC03080B131533
:107FC2000DD9FED5883E434670AA680A4DA4E5A4A1
:107FD200AA704670785816468386FDBCEE4B66B88A
:107FE200FCEE0825AC1B95BC780EE3D1486E2B59EC
:107FF200C42E1659C41916D1486ECFA3D1489D4834
:10800200FE738BD1486E4BBBD1486E439D48FE2315
:10801200FBD148CB4E3E304C0EB87E5B81C8067811
:108022003C06B9586E63AE6E7F3A3A3A3A3C7038C3
:108032000E8E844E70F8E030546E9B305A6E73662A
:108042006E53666E33B5A20EA04E3E7EC37E7EA0F8
:108052007ECE7E574E43EEA0663346F6A0BEE04E7D
:108062005EE76EE0CE7E1B5EE0E0DCA0DC5EEE1F33
:10807200237CF2F3AE5EEE1F237CF2F30E03E0A547
:10808200CCBC0E4670AE6881F04E70789A66AE68CF
:10809200304070AEF03E55F04E7084B07E7E7E2F42
:1080A2007E89F68801C8E6B5A286B0668DC61C0632
:1080B200A54FC678A6063DC358B0FC06707C26E6DE
:1080C200F002223DD0AED8E63C7006023DD0B0E6CA
:1080D2000CC38604304006A5D00C49D1C676431C99
:1080E2000A6AA5D049D066B0E6C67038A670A6F076
:1080F200986666776651ECA606704EF09866BF8D5C
:10810200C68451EC8C276688D326E67022FC0602D0
:108112003DD0A658B026E6FC063DD098BCA6588CA9
:10812200A3BA44DDD47AFA9A983C0698767FA606DA
:10813200BF0DFC060C2013091A05D9FEA5D00C9719
:1081420098762BA5D00C5F98E63CA6B0FC707CF02C
:108152005DC40A3EE6B006A63CA60667BC704E7039
:10816200F8FE2F66A6067038EE472DD0983C66AF13
:10817200BB00000000000000000000000000000042
:1081820000000000000000000000000000000000ED
:1081920000000000000000000000000000000000DD
:1081A2009CC2FFCC574626FBCC2F5DC4243C71CC2D
:1081B2006653309066FBC8CC6100839C4262E2A5A4
:1081C200684E9C90CC5F601B7A1F7ACB5DC4E01036
:1081D20071CC664FA5689C228859C87BA568D91CBA
:1081E20078583012662761C8CB30C266AF46F08C31
:1081F2005B59C8BDCC66E627652073BCF05DC42917
:108202003C26662F8865C82B49F08804E9D48C2B5C
:108212005DC47E3E4E70088C2B4540061BF9C4306F
:1082220018A6C6B07CEEBCA686A6061F04A6669853
:108232003CC658B03C0671D84E70B87CD8040C13BA
:1082420008D8BCA898668DC77C0EEDA4E601D0AE16
:108252003C58C69C584E7051B41C53BDD0C1D85E18
:108262003E2DE0DDFCB1C0BDD04C1BE9D071F0B0B9
:10827200FC700602385AF051FCAAAE3C58C9C099AB
:10828200C0980A01D098AA0A5841C480E68741C41E
:108292004C5780E6AB708D8C987C0EB004D88C1352
:1082A20008D826CABFAE3C580AB066577001D04102
:1082B200C4808D8CAB0C2341C4804B081304980AF4
:1082C20030FF8D8CA156C1D8BDD04CD9C85E7E7E00
:1082D200FE39E098EEB5F604DCD01EB07E7E2F08A3
:1082E2007E29E331F40C533E85E0B05E3E7095F09A
:1082F20059C0B0CE46CE6E6E68BDD071F04E707869
:1083020058B0FC060201D0EDA48A0456705C0A063D
:1083120076265766D88C1B086AD86A6A98AACAE772
:10832200AA581C4699C4B0A1C46AB0664F7001D065
:10833200EDA4A1C4B30C7B46A1C45B0830FF99C471
:10834200640530FFA1C469D095DC0C554AF9FA38AE
:10835200BCA6BC288804E9D48C434E30913CEEE99B
:108362005ACEBC06B07CC698BC1ABCEE4E70385CC5
:10837200AA581C06BC065F3C0EEDA459A4E6AEBC8E
:108382000EEDA4AE5884C61C6A17881C987C66E65B
:108392001F8CAF8CFBFC580A01D098AABCDBE156BB
:1083A2003BB03C263C463C7098E63C0AEDD02E841D
:1083B20049D463BC6658CEFC0A01D0B07C263C701E
:1083C200983CAA7C5806D3B0FC707CF05DC45E3F3A
:1083D2007E2F06ABF0837E7E89F788480DD4CE5877
:1083E2004E70F80E8C2BEEC3F9FA3DD00698BC06FF
:1083F2007F0DFC050E04200F0620120503F1FE6618
:10840200B03C065DD8554AA5CC06BCA63CF081F02E
:10841200D5CC663002C61306F5C459C42E1200002C
:10842200000000000000000000000000000000004A
:10843200000000000000000000000000000000003A
:10844200000000000000000000000000000000002A
:10845200000000000000000000000000000000001A
:10846200000000000000000000000000000000000A
:1084720000000000000000000000000000000000FA
:1084820000000000000000000000000000000000EA
:1084920000000000000000000000000000000000DA
:1084A20000000000000000000000000000000000CA
:1084B20000000000000000000000000000000000BA
:1084C20000000000000000000000000000000000AA
:1084D200000000000000000000000000000000009A
:1084E200000000000000000000000000000000008A
:1084F200000000000000000000000000000000007A
:108502000000000000000000000000000000000069
:108512000000000000000000000000000000000059
:108522000000000000000000000000000000000049
:108532000000000000000000000000000000000039
:108542000000000000000000000000000000000029
:108552000000000000000000000000000000000019
:108562000000000000000000000000000000000009
:1085720000000000000000000000000000000000F9
:1085820000000000000000000000000000000000E9
:1085920000000000000000000000000000000000D9
:1085A20081C8E6B5A2064540B9CCA6BCA63CF048B7
:1085B20085F08C5BB0FC2670381CEE77709BD5CCB6
:1085C200A04E70EE59C4EA003CEAF30E4E70AE685B
:1085D200B01E4E3E1CBEBE33501050903B10BE2B00
:1085E20010105003BE2B5050D0D3B046FC06F5C439
:1085F200A3F85E5AE8A878E630C0062663A606709D
:10860200383E334E7EF066A3A1803CD5883E7B7017
:10861200AE0E584DA459A4468D8C980EB0E66F70DC
:108622005DC414218A4E6E56DC90688DB8BC0898E1
:108632003C28441C6A8AEDA45606303A067B303048
:1086420006AF3020469C58DD201C6A4E30056A5B1E
:1086520059A46A4C8FEB48783A87783A8DC7B83C70
:10866200D808D87CA88CB5515DC4333B3045663FF1
:10867200783A27301B83302B66832666378C7F300F
:108682001A23266627301CD32666678C9F4C4353D9
:10869200F8EECE71C8700439D006B0BCA6700839A5
:1086A200D0E6172606B0BCA670783C06B03C063C65
:1086B20006B958BCB95826703C063CE64EA670A6D0
:1086C200F0B02606C78DC60E66176629C6BC069C84
:1086D200E2D330901C02AB30316A8B30460217660F
:1086E2009C024B501C62276A136AA6A606C6E6A223
:1086F200065E233008465DC46A27F9C40C2F701544
:10870200C8E68DC606F8FEB0C6FB46DE1BA6C6A6A8
:108712007079C4AA58B0665F701C980AEDA49C5880
:10872200461C8D8C51B47B4E1C10CC2F6EEB4E4BE5
:10873200203C56069CE21B4E5330C4064FC64ED018
:10874200A646263CA3E6761C4E906AC6FB303162F2
:10875200276A13A662AA3C26EE61005DC42E12307F
:10876200FF06F8BC66470EB8A6AEA88DC6B8BC66B2
:10877200B5A3840895D0302B06B006273C061B8192
:108782000A06B8BC13EEA6F30EB03CE630A8AEEE75
:10879200176668A69C583508B0063C260677BC705A
:1087A200783BF87EFE5F5C10EEAB1C7CEAF33C3358
:1087B20015C83C9C4A7079C40C2F8AB058EDA4AEFF
:1087C200D87C1C846A1788D8AE987CEA1F8CBF4E6E
:1087D20030051C6A538C2F6A59A40359A4034E70A6
:1087E20030913CEE3B79C46DCCF5C459C4EA00BD6E
:1087F200E0DC101E46FCBE77E6A670066638EE7018
:1088020066EEF0BEAB5DC4EE00307A66FB610278C4
:10881200E8380E38D81CAA28E09CA01C380EF8AA0A
:108822007CE8AE7C280EE0D4948DC7A0EA73E267A0
:108832009846AE283B48084EDDE04E300BAAA0FA1F
:1088420060E6133AA6CB3C30030E51C45DC42E122F
:10885200B87CD83C30300693302E66370C60A6A622
:10886200E0300D664F302D06E0303A066061DAB135
:10887200D0AE0E3CEECEFCEA6DCC666686664E301D
:1088820007A63AC6F346703CEEBCC66804044CE147
:10889200C4E9D00881F08C4BB07EFEA1C3A1F48361
:1088A2004E70780666263DC2EE4E9CCA1C3E70AEE5
:1088B2003C06027098F00DD0A60670B0F07A4670B1
:1088C200CEAA7C0EE5A4E6AEBC0E01D0C68D8CB05D
:1088D200A626A67A2770AE5B7001D0B08D8C0DD023
:1088E200A6704E6EF05DC4F000492438FC70063864
:1088F200FCA67C70E04670387CAA0A3C28E004049E
:1089020084E9D4983C1C0A0451FC4A2A2AE03060CB
:108912000698467004261C7C4A300AFC58B8A6A861
:10892200E0D91C78D8E0EDA40616D91C303A66438B
:10893200302C6623302E6661DAE0B1D08E0441A479
:1089420044CE0637662FA20217484ECA686A054609
:108952000000000000000000000000000000000015
:108962000000000000000000000000000000000005
:1089720000000000000000000000000000000000F5
:1089820000000000000000000000000000000000E5
:1089920000000000000000000000000000000000D5
:1089A20088DCD0FE95E84E705C380AB0AA2845D81B
:1089B2001388D91C78468C1326F0256C8808040489
:1089C200E9D40C5B44DDD4CE7C06463BA6265DD8BA
:1089D200705B7C0A556CB03C46BC70C57E256C044D
:1089E2004670387C1C0AEDA4563CAA7CEE3BCEFCB9
:1089F2001C0A556CDABC06B07C063B86BC065DD808
:108A020070DA7CE6917AAE4670CE68C1B0E0B07C96
:108A120006300B0697300D46DA7C06333017C63E19
:108A22009306301806BBB03C061EA114F87E7E9E4B
:108A3200066646F098A6581CB07C26E6CE7C0A0450
:108A4200EDD098E67CAAFC58CE7C0AEDD098AA58C4
:108A5200CE7C0AD9D0DC101E9E9E1C98AA5804080F
:108A620093EDA48A06D91C79B01CCCE746F06A01C2
:108A7200D0987C6A6F98DE586A8744D91C987E2FFA
:108A8200581EA9763020E805768A48196C4479B0D8
:108A920098DE1EFCDC901E1F5E1BBE5E3C5883ED02
:108AA200A48A06D91CCC33D9B008357679B01C6AB1
:108AB20046F001D0986A63DE3FFCFE9B0C8BFEDE23
:108AC20004F3D91C0CE37E9EBEC7F8BEF3A3D91CE7
:108AD200B8F8568A063040C64B46F06A196C1B79C4
:108AE200B0980C37FC1E9E3C1E3C9CE2042030F0E9
:108AF200E6E09CA0443020CC697766E3C6667977CD
:108B0200E699C8D91C9C6282B8A2F34C1B98F30662
:108B1200E094339C98A60658A0D88444D84C77C6D3
:108B2200A69C58301F6617260698069CE8D09C0221
:108B320082B8A2F34C5177485576203CF64BA56893
:108B4200711C5DC4E01078581A7A7A4E203C5A1C87
:108B52005D001AE000105B504B903BF3D023000005
:108B6200103C56063044668F788C1B84138884D858
:108B7200F0A5680C6973517626669FB07C06668CF8
:108B820023300B4686BC0646F05DD8C97A26667746
:108B9200B07C0646268C1B300CC65306434924780B
:108BA200FC5CEAEE9C300842A17CF6DD7B30088C4E
:108BB2001F4200957C068C47C1681BC17A7C58987D
:108BC200A6588CBB796C4A57C1B0BD1C0E0F20123F
:108BD2000F0F0DDDAC78D884D8F049246D586100B0
:108BE20030FF66675ACCE3203C0630C366DD7A6903
:108BF2007288489806C96C25E8E3CEBC06B07C664C
:108C02002326E6CEFC1C0A04EDD0988D8C066686DF
:108C1200B03C0671D8C97A3008957CE6EFDABC061A
:108C22001C3001667FE6CEFC0AEDD030608D8CB040
:108C32003C9D7EB07C667766C6E6A658BC065DD8CB
:108C42007C26E633C626E6A658CEFC0A04EDD0986A
:108C52003CAA7C58066611F4D3F6278C557B1C0679
:108C6200300825400E7E9B9A0507088700D36B3B90
:108C7200E3FBEBD323DBB17E75F44670387C0AED5F
:108C8200A4567626A3617E056C8C1B8413883D76E0
:108C92006520056C8498F0A568F572796C0AA17B51
:108CA200B96CB0684829E84670787083BB843BFB96
:108CB200796C0A5788CEFC0AD9D0B03C26BC70ED3C
:108CC200A456768CEBE6556CC6263FAA7C5CCAEEAF
:108CD20083B96CB0FC5CEAC41C59E8056C8498F05A
:108CE20046F01B056C8C1B84138898F0C97AB03C43
:108CF200E6C17A6606265DD8056C8498F0A5686997
:108D020072267F556CB03C06265DD80B4666E68817
:108D120059C804C1B0BD1C07140F201E7E7EC63C7C
:108D220030033E1B30017EFCE8BEB3DDAC0C3B469B
:108D3200F0C6E10803A5684E5C10901ACC4F26EBF2
:108D420099C8BACB7976300B01ECC384743485753B
:108D5200358676363700233636363636363636366A
:108D62005B65209300000000E080E006C61C2247FD
:108D72001C8622279C860882CD7EC61C222B1C22A2
:108D8200DD7B02A29F8C174230555EFC06BC30E0B0
:108D9200000005CAF3EBE3DBD3CBC303180D146762
:108DA200308AA630BD8B72201165E34F0B1D102354
:108DB20050C604A89C60C74C81496A521BF515F342
:108DC20014124485B60825C6205B15EBA2262A0A92
:108DD200400C50AD3C362203820F0035323881847C
:108DE200D80400CCC040819010038074D184F5B0C7
:108DF2004DC000A409302333CC5068BB881F88FBC8
:108E02000D8C8C84D4CC0035C0A803033C31818600
:108E120021F25B38338A1CC3A1362321B22485E8B0
:108E22002ECD8843480C08000638622380C7108282
:108E3200B02066CDC040FD657EFDF5E6D61831D185
:108E420018C0A82221727CBCEF43E2F030E363BB7E
:108E5200EF0C2320EC20ECFF10A2A0802122282A74
:108E62008221C0C3953C412282101102821108CC9A
:108E720004002088310089FD0CCF0B104208499173
:108E82009D3055C3080018E00D7800880350F0812A
:108E920034242AF10200000000000000000000005B
:108EA200C9E0331053FE72482113E20331158A35AB
:108EB2001D23C6B0CB28320EF88A423203980C40EA
:108EC200102131411204B81BCE392500C520F0040F
:108ED20052D9C408182044D915449146A603153D19
:108EE2006D50210009076954011693A150421A4A94
:108EF2001B050452C7AC8EA0418010409A4F5D11F1
:108F0200040481004227644114441785A224434883
:108F120061542468441EC98009CD33A1DC50106A13
:108F2200821041C1B30601194525880333D6404357
:108F3200482331E50800000610D01429430431000B
:108F4200000000000000000000000000000000001F
:108F5200000000000000000000000000000000000F
:108F620000000000000000000000000000000000FF
:108F720000000000000000000000000000000000EF
:108F820000000000000000000000000000000000DF
:108F920000000000000000000000000000000000CF
:108FA2002134432432A02C3222037A48841411172C
:108FB200C54108160E3BD19008DA2308D40C50B8EC
:108FC2000320AAC428201417170E003183AAAE73F7
:108FD2007F3703F17A18EB40E8C42EE340E044E027
:108FE20088114C2046211420D24F22D41E7F7C8C23
:108FF2003FCF143D4D34004238019D1008E15032FC
:109002000030344E4207C404A89C60C74C81C8405B
:1090120045D3F0D0801231CC44D401412433841B97
:109022008E32F62E61200609FD73B40CC10CF38C4E
:109032002108C44098186081620F848B9EC0082763
:1090420008C70FEEC5174060865D2403B731315C57
:10905200C744C7CB50005044642384930C32E88C3D
:10906200683D00088509240A6002040084C00000EB
:10907200880E841800A3512E4891801E8508048909
:109082004F2F313131B13C1432C30852000000007D
:1090920000000000000000000000000000000000CE
:1090A2000B801A2838215A84720934015C05049510
:1090B2006824000054180D059034E248C544341168
:1090C200140F3113C411249811405844587841C4E4
:1090D200084D700CC447E3244571A119913680876D
:1090E200D0CC54010C8D2B033B0371330F4530461A
:1090F20034D6061D20F4E668C8003744C8516C4BCC
:109102004C8C214BDD14E55131D0141E6300C0009C
:109112004931CDEC56540E954414C339144A348760
:10912200064767C5C435C67D44753300E0B41B23CA
:109132002DBC141F595580D10A901110105C9C61EE
:10914200C4004500148D4105090941465124C94412
:109152007155591055508296A0968978626E514D7C
:1091620085094A4DF5430186E051080816C68CB1BF
:109172009C01B0079E01E6167941C088F20C2005D9
:1091820021A1F70C331654E3D21600000090AAAACC
:10919200884077282F3FC5A2474B85F630FF3F888E
:1091A2001A24005D0B6E08060F380B670B5F02D79F
:1091B20002E202EA02F306340407010002C102C815
:1091C20001790089016E0122011701350B01042387
:1091D200040F0B440CE5056009FB00EE0941005445
:1091E200006902D0007A007100610000850D091447
:1091F2002018032D83322020050D09142D941017F9
:1092020013C5DA810D0C010C0341E68D0C010C0330
:109212001289E6930D0C01120C03C9CE0000000066
:10922200000000000000970F0404A140F9446948BF
:1092320063C1B0981E7E3570DDAC6564983102580A
:10924200300370C158CE6152814084D54CF88C13E2
:10925200B86ED330200C3330188C1326E6A1880464
:10926200B17022D91CB8C6E86564ED8A389C4AE020
:109272003E3E3E8A1E4E62EFCECAD47EC31E4EAA28
:10928200E05830107030FBF0E8E0850D0914D96821
:109292008E7C5E61446948BB6ED9708B8514010473
:1092A200D968754C694843C1B008F548656498EEC1
:1092B200B94A97130C0312514C04E5449B86010CE6
:1092C200031295445B514CF8BC6944FEA0DC50E0AB
:1092D20097130E1512514C68E08940A838A0FE1B66
:1092E2005C8A0E9E1EB1644E46D95C5C19688D7014
:1092F200CE0E5C7CEACED95C5C4AFA1F4E5BA00EB5
:10930200665C1BFAA642EBAE0E60E099040DB8BC97
:10931200D844D87CA8E0990D04B8BCD848AB0E8ECE
:109322008EA04E5C504E4E9C3E3ED05C4140603C16
:10933200E00408E0DCA046F098067038F613666692
:109342003C7E60BCA6BCDC100EC1B0AE5C900E468A
:10935200F03C70380C435C04F2277CA2E370D91C09
:109362008EB07C7075B06E8E5E4B5CA2A39CA2AF79
:109372007AD30CE361009CD2BB9CD2A0C1B0DC10BA
:10938200FE04041B300B3C0E1CF86A1FBEE3B849F6
:10939200243E616A856869547008A968E6067038D7
:1093A2001CFC6A6A1E6A337E7E98A658B08148ED1C
:1093B2004E6954BE3E0165DB000045DA0000000044
:1093C20000006954F693E0DCA01CEE982670380E7B
:1093D200A0F2A65EEBA6728940387C3232000032DF
:1093E2001F12EF662792B2939260981D68A60498A6
:1093F20070CE1C42F0861E81487E98C6BE6066EB27
:10940200F613263C5E9E9870380C134E70985326C5
:109412007038A670A6F066A60626AFC670B0F0BE7B
:1094220033E0300870A6DCD09C1E387C4A3CEE60EB
:10943200A6BE60A6067038BB8940387C4666E6A6A2
:10944200260E4B361CE2172AA6496870383E607E0B
:109452001C128B1C42F0935C0A6029FEAB051401BE
:1094620004D9CE93190104048DCE980D0C010C037E
:1094720011E6B2310B0C03DD48449828E0B4320BFC
:109482000C03DD4848AB940B0C03DD48846B841459
:109492000B0C03DD488823514CAD72754C46178E78
:1094A20030020C6BE01CA01C50509C3005721766F9
:1094B200884884DD6C0C0BDDAC4E30200EB8B8B899
:1094C200662F7EB86623D888D8E8492438D91C9CF0
:1094D2004A9EF9447E3570492659CA8568338940C7
:1094E2004EA8E0454A93000099CA08C1B049440019
:1094F200B9620058894068F858A8B80E4EA07A6040
:109502006E1F8CA0A84E2828A82828E8E828E8A8DA
:109512002828E8A8E04970136BDD48A00E3CAA7C1D
:10952200C6A670663004062B301246BA9A4EA6BC06
:1095320001700EB01A9A70DAA5709A7C2B816CA019
:109542000E0E4924389C0AAE284A7C0E4E5C50D03E
:1095520010101090504E5CD0905090DC4140AEBC48
:109562000E389C4ABC70BAA57070BC0E4E1CD0104E
:10957200903A5C49404E5C100E2BCE7A1A23AE7C98
:1095820006B0A6705A0170BC30120EB0BA5A7A6692
:1095920006237AA646FCDA3C5CAA7C0EDD486946C4
:1095A20094030512120F034843850D091405134451
:1095B2004E7D4070CD6C49503C2EFCBB851401049D
:1095C2001405134E7E708140EEB5A258CD6C4484D2
:1095D2004950704570380EB0284CD3492478AECE2D
:1095E2003010956078AE68CEF0AE5C4E138A0A30C9
:1095F2001095607858B075604E3004583A3024BCEB
:109602004960709544A0EE1FA01B2D60B02560EE4E
:109612003961216CC4F57C856813E061481CCAF984
:1096220072E0AEBC0EA01C30120A334A2356134A13
:1096320016E004E0DCA005688EB03E777E49701328
:10964200730950EA0A4BAE3C0E1C12D1501B84AB7C
:10965200D8EE271CD2D3D54CB540EE4D704E1C50DF
:10966200501C0A1BCD4290901C0AD36E816C4E0E88
:109672008D70CE4EFD50A0980EE09ED95C4D7013B9
:1096820063D95C8A8A4B30030455701B616A8A8AEB
:109692008A1ED95CA04E9C909C0A931C3C0A73A023
:1096A2005C99704E5CA5700E0E60E00E695013EB73
:1096B200D95CDE7098067C6627B00E2B6670C158A6
:1096C200CED95CFE23A03E2B6E6D50234C670BD986
:1096D2005CDEA05CFE138A0EB0FE138AAECE5E6F15
:1096E2009E2146307A66FB61020404981D5C5AE1B1
:1096F200080698467CA6BC58E01C987038E0971380
:10970200783CE64EC67CC63CEE514CC4780ED1E2A3
:10971200B1640E681CE260CE3C58B96C6100CCEDBD
:1097220057080C7F44E544CCCFE05CB5708C171C25
:10973200D85346F0987CB95844CECC37FE2BA03E85
:109742007E538C2B2D548B234970630460B170229D
:1097520008D91C495C638ECC4FE01C214CCCF55CD3
:10976200A0CCCF6089406C9BF89CE27B4970CC1DF9
:1097720070CC4F89403031E8F9561CF8EA23A838FA
:109782000E98BC62EBCCAFA2023C580CAF0844AEC0
:10979200F544CC47214CE05C115C3B6046F0301351
:1097A20071648713847434857535867636371882EA
:1097B200C21283C37300230B36363636363636363C
:1097C20036134B237BFBFB6B53306E66FBF1568BE0
:1097D200030F0C039170E5EE995ABB05D40D544961
:1097E200248142115AB95A855A0DD49170A56CA0A0
:1097F200F9CE73AB8C374C73195C061C62131C4296
:1098020062315D33D38940F81C0CFFEABF4EA828B1
:109812009B4C8FB570A88C1B281368580C2555F3E8
:109822008C178C1F883B842B4CD73032155CA08C54
:109832002FA6FB415E66134660315C315488E54CCD
:10984200AB8C9F4C8F0C1F0813042D5404434C37D0
:109852008C370CCF08A55A044C1F481344989C42DD
:109862001C4258C3155C044C374666B6489336769C
:10987200DF1C862233A24C47C62B629C86A244314F
:109882005C4CCF3154BB4C778940A838700C2555BD
:10989200987CB958B004F544987C70AEF0C8CC7B83
:1098A20008488C2D55C8CC3BE01CF55C46F0983C32
:1098B200A02660F61348315C7C26BC588CE54D61CD
:1098C20000987C26167616577038AE98F038AEF0AF
:1098D200986E4971F9560CA04C43C8CC60A0602028
:1098E200E0CCED57E006983C0CA03CE03C0C173C69
:1098F20058E0302E0C1B303DE830128C1B3004E84F
:10990200195CD95C065E3E4C1B3E234C17E6303098
:109912007CB6163C761B301FE8E67EABE0A0C1B0F9
:10992200600C495CD95C6EE00C2B5E4BD43B5E1341
:109932001C4C135C2BE01CA05E0EC1B03E04885C84
:10994200421B3EC3EAE0DCA07EBB830491704C4F15
:10995200D8C9705C422F3E33D8885E3EFED91C784F
:1099620068786860E0EAA09C9A5E339A509C029004
:10997200DEDE1790D95C13D07EF3D0D0D0D0D0D019
:10998200D0E0DCD08C7F0A9417904C2762101350E1
:1099920050DC0210CA683828380AAE28A046F0E027
:1099A2009401030D0C017D681B796666A65E3E5824
:1099B200C4440D54E0C170843D6404CDB47B758C05
:1099C200E06564E04871682B65644164E04544EBFE
:1099D200B068CDB42BE5AC88138478703D64E06543
:1099E200443B8CE5AD3D6413208C758DE0208433BF
:1099F200985E580D54214C492498FE2BCC6F156863
:109A02004330FFCC3766EB235162203C56063018B8
:109A1200662D5A308766D3309366FBC8CC6100FB53
:109A22004E9C90CCA7601B7A1F7ACBF55A89485876
:109A3200C17085641385644B1C20E2B78C73E54CBE
:109A4200300671643470C28412C300133383533BF3
:109A5200DBBBD14413037966E168E09C8301644275
:109A620049621B985E3E4962E54C2B300871648066
:109A72003482C2848712C300CB033B3B6333538BD4
:109A820073EB1568E365203BF168E05CE1708441AB
:109A920062F168C1B008ED48B3447168008B294E89
:109AA2008568668698663315C84D68CBC658E0202F
:109AB20030F1CC256366E3E0E008017201EE8841F3
:109AC200DE9870C4F57CB058E0000000A09C4ED037
:109AD20090CEFBE0B87CD88C6089028D0C011A19FB
:109AE20018300289407D4070514CE83888084D504A
:109AF2007C46EE173A70842689400EEE6B889950A8
:109B02002B301AF1424E360ECFAE7C4668600948C1
:109B1200B0300446068C1B66367066A6588514065D
:109B22009806678826260613848568238C97A18861
:109B3200C1B0BD1C0E0F20120F0F0D38F821428646
:109B4200C626704E7EF0C6704EDC90901090F004E7
:109B5200A96858B0C6260E2568869806B05568983A
:109B6200A658A670660638D87066D8F026ABC670BE
:109B72002658B0F65BF04670780E98702658AEF014
:109B8200B09C629F0948EE173AD87026D8F0BE3FC3
:109B9200A6667006388BD152982B148140CD6C2E5C
:109BA2005899501BB5A2A0DE1B8E0E70984E5E33E4
:109BB2000ED164AE734E9C501090D05010D090AE27
:109BC2000E874570380EB00E286B8606B05568C6F3
:109BD2007038FC1CAA0C2F0A3967134A7CF026A69F
:109BE20004A568A6A6E0A6496870381C3E607E12ED
:109BF200B3E0067038F61366663C46FC0606E05192
:109C02004C4EF0E0DCA030C0085C905C0E13664E57
:109C12007078067BA60670383EAF7E62A0FC564680
:109C2200EE770CA0A398496870383E6F98A658E06A
:109C3200894833D144E07EA060B03AE06954F69B93
:109C4200982670383C05688D70CE0EBC555CD91CC8
:109C5200B83B4C604EBB514C894038339870384603
:109C62003C0E0430059C5A109010DCDCDCDCA0FABF
:109C72005A13229AF33A0C534C2BC8CCA023CCEDA6
:109C8200576627D4BA73945BFA5A5CD0905CFA4652
:109C920026139423FA10C3FCAA0E60E08601140571
:109CA20013514CE838288140EE8349701B4E5BDC2F
:109CB20050AEFC1E1B261FE6EBBC89403CA8E8E028
:109CC2004EDC5050501090E084E80444D828E8302C
:109CD20029E8E0EE514CE8380E4E70AE68A0E097ED
:109CE20013140513417013339E048D501BB5A24DFE
:109CF2004C98DE1BA08E28E0B432050D09140184B5
:109D0200887B850D091401843B8514010401888434
:109D120044417013CBB87C1C50600691704C23D820
:109D22008813D8492430260213A222D888D88C7BE3
:109D32008662271CEAEA0604E948E2B308A3068C15
:109D42004FC9705C4267DC906B095060AE3C0E13E9
:109D5200FA4C47DCD0A25D6C6E4BD91C9C10D0A291
:109D62007CE89CA2BB8C608C603020616C30414CE2
:109D72001B3050616C304D6E5851B6B6A31C8C7FAF
:109D8200A25390909C5D6C6E167693D090BBA2CF3E
:109D9200302F0C4B664C73B8D848D81B4C3BE84B61
:109DA2000EEE0E0EEECEEE0EE0CE30046944A0E0D2
:109DB20081400E3001A0A65C4636616B7606138A9E
:109DC20066F3E0A0A01CE0DCA04EB2CEEE4EEEE0C8
:109DD200F16804E09C23E09C08A0C1B0AE707C5EF8
:109DE2000EAD5C0C60D91CF8F8B00EED4A7E7C1A00
:109DF200FA5AA57013150E0D0F0E1415051705044A
:109E0200140815061209130114B01A30E83ABEE319
:109E1200E09806C44924B8BCF6F6F6A088E004C56A
:109E2200703059D866F31BC570301E0C1BCC876688
:109E3200DB2308C570302DD80C1BCC1F66D3C45849
:109E4200A60658E030107030FBF0A838238940F89D
:109E5200D8E0AE8444BC0E30121C0A776A53A0CA02
:109E62000A374A881B563348234ADF0660AE3C0E47
:109E7200E00E4E7078EE894078A0AE8E0E68E097C4
:109E820013100F1413514C28E060FCB07CA0EE0EAE
:109E92001CD09050A636369C133AA2F38E76E3AECF
:109EA200BC0EDA3CDAB0BA5A707A9A4E5C109C4117
:109EB20040AE3C0E3C5A4E1C50D010509010AEDAC0
:109EC200CEFC70B01AE05D1C0C13C88498A8150C67
:109ED200711EE1688CD972E0C97020E0894038A017
:109EE2002E2E60E0000000000000000000000000D4
:109EF200000000000000000000080B6CBB8CAB0EE1
:109F02004E70B89CA2A8B5708C1B585B4C43C1B074
:109F120048042BA16C044484617604588940594C4E
:109F220038580CC76C2F4C517EDBE8F8D84C4D7674
:109F3200D80C1F4CC34670B83CD80C738C674C5776
:109F4200D80C7BC97491704898A828E8381CEA5745
:109F52008CA30568EA274E907BF83CFECFFEBF60DB
:109F62003D5BCC4B3B4E36682B854044E804D8A879
:109F7200288940BD6C88044408844484608940F880
:109F8200D88C3BD83038E8FD7E0C27D8D57E58488F
:109F92003031E8757A980670389C62CFF61366669F
:109FA2003C1EA6067038AE7E1B4E23267038AEE0ED
:109FB200DCA05CEE5D7AF237B2EEEE7CD37C06304A
:109FC2005EA61C6A873C5CB27C0E4EB2EEEE521B61
:109FD2003CD31CEE25510E917004E6C61CEA4BE000
:109FE20008F174A8E8557E3C305E6A478E8E8CBFBD
:109FF200CC87A3FE97C68C7F4C6FD844CCD36554D4
:10A00200D0F0F9700D7EC6A16C49240C37B8D84443
:10A01200D8A8AE6841683B8DE2F174A8E8CC997487
:10A022005D1C0C330498A809B8BC5884983CA878E5
:10A0320058EE091E44D5420C676554D0F09888BC8E
:10A04200983C589974E020F97098BC584C93C1B070
:10A05200BD1C14090D051220010C01120D205345DF
:10A06200441333C17098BC5846F06666FB61009891
:10A07200DC1044E05830F1CCFF66EB2030264C2B4C
:10A0820008FD7046CC9F66EB987E4B4C1F482B48D0
:10A092008C979170A56C6B2020441C583C1C0A497B
:10A0A200CA30C36A8B2E4C4544000D5465440046A9
:10A0B20066CC3766EB0D54411C4C5F9C98560630BB
:10A0C20072665F4CFBD57E8C6B480D7CCB4168BBC6
:10A0D20098E3970F0E0D0C01514C88C40848608517
:10A0E200684B2315684389400EDB6631687038E699
:10A0F200463C0E8940F9740E630C474C3F8C271C7A
:10A10200C217D5764C43F8D88C1B58E058AEA8E855
:10A112003038E84C60E00C132049244CA7CC091FCE
:10A122008C8B91704C37D88C53C502603D5BC974DF
:10A13200F90C9170048498A82860A05D1C98CD9EAB
:10A1420058B8EE514C6C9B385888989CC2285D1CBC
:10A15200089842A84B4D4C38580484D91C783C8945
:10A1620040A8FE63084E2B00E080E02E6889CE4CAA
:10A17200EBA56C33587D6813DBDC90F091708CA7F3
:10A182006148D6F970736576817ED968C97071BAF3
:10A19200D57EE976008B93CBD3DB0003320D14CE50
:10A1A20000000000000000000000000000000000AD
:10A1B2000000000000000000000000000400000099
:10A1C20000006C454C54434D613076314C4C8C4C04
:10A1D200C1CC34CAAAF4BD031FC60F6048111000D7
:10A1E20066C4781400404503401794EB00D4DF287E
:10A1F2001B505047BB402060CD3D3930B30FCCDC03
:10A202004B45DA6707C225523BE40D172330723300
:10A21200300173171992E4E3C4793F7D60554024FD
:10A22200A348451455922000508E404ADEC7B142E1
:10A232007CF45845324211EDE291008482183D626D
:10A242001F2246E435C9C708060B94B8FC3838000B
:10A252000400020000C07503700D700EC07999CD24
:10A262002144688C43D910FDD3B31F8E50544871DA
:10A27200300DD21847374FA8C3E0129BC4139A4837
:10A2820043315140140AA790161A42581225050765
:10A2920029C05104E961838D01501188137A7156E6
:10A2A2000080008018642B00006242E4C615594801
:10A2B2001122B05884214406012921804253B16DF4
:10A2C2004D79CC4C3C7220125843C531495006118D
:10A2D20036063D6474670E11D01311F643423C3EBC
:10A2E2005190798704E5501A90281C3EE16288F467
:10A2F20054B848C554429F0C0388D434242344F2F2
:10A3020025D28109C71972A2320444064DC1405DAB
:10A312009C371CB6DD05353DD50E91263405A61CAD
:10A32200040000000050AAAA56458517000697545B
:10A33200CC998911501ED521961D5B33B72DF3168A
:10A342003E7719A53409564948885810C210C004EE
:10A35200914520A1BF00E353659537581944293E22
:10A36200393D501CAA504A92A43442826DD5F2273C
:10A372007F17CE091D12C7C44521481C9311EF3324
:10A3820052043033002134C623334E16DB03830CD0
:10A392008040CF1708042E12308010011F0004F0F5
:10A3A200005050605B1294719219441A681820E4AC
:10A3B2008111732E51556463F4782414576CF98B10
:10A3C200C8843851445398464100C080724C06D12B
:10A3D20054587410000004BC600A0664D978675CA3
:10A3E20015CDD4F479B92790C444030AF5B70B000C
:10A3F2008419356F23B2967C84E1336A844D124905
:10A40200CD3A57333300601F288AA820145851547C
:10A4120084469A8F868896862C26A619685C805177
:10A422001DA01835109015047F850914C280861866
:10A43200554C09EE9F488D763112ED113E24EE43C4
:10A44200DE5422D1C4DD6625291E6D36DF5C070984
:10A452005684F52F6017F2F3C92F10050EB0E400F1
:10A46200D4644280818877CE08D907773035213A83
:10A472000004744025CA00C000C0003010CE99C547
:10A4820070D4E03F4F1F1610D8239810837030030A
:10A492007F3CC745C405403EC11F34DE01F237FC94
:10A4A20065BD1FE556C86AC2BE84C0D526023220E9
:10A4B200990FD365550000000000E4DBDF31D55F62
:10A4C200A54E458C539531BEF4617C1C0F553C63FF
:10A4D200134C7C428772483200D44B0852E8D43B7A
:10A4E200858100E561462545102EA32F6192F487F0
:10A4F200EA0000000000D44C786C333009D9575779
:10A502009D83357303E17F541319DF2C7242704827
:10A51200F5601CF11D6D0B1ECF01C13581952C52CA
:10A5220047828002B226FC5FF03B073FBE93098759
:10A5320012DA311F4E3030565B05853C8F46104A89
:10A5420002FCF4B3398AD6461379D5300300008869
:10A5520001D5AC4BA6C5F82D15E3B97866D406DC57
:10A56200C4805107BE57C0500C94531B0100D562E2
:10A5720081719009D8D108CB7EC0F383013B473863
:10A5820063304C4561FE89344D7D7F24CE57FBE418
:10A592001D40B70D9315ABF6665D665456FC0B88ED
:10A5A200193F0097013B01C60A430AD2057C01D23A
:10A5B20001520A19008809B409AC0D5B0D630C162F
:10A5C200016907F7037206B20E6205730E3606AC16
:10A5D200080B0A7B0A85010303AF02B5068600B1A8
:10A5E2000DE403490F530F5B0EC30EBA062D085F2D
:10A5F2000E690E2F08050F2C0F350173035703C088
:10A602000C0400AC009D03B809A300E306A20B2FC3
:10A612000AFC00F7012001290132023C02CE066C3D
:10A6220000009319050B0C030B8045628432200E47
:10A632000306201418052D8D0F0F1213010B8055E0
:10A642006A8E0306201418052018032D851A091393
:10A652001001C870F868385C581C0E38AA28B0443B
:10A662005D5C385CD8284C9B5D1CCC274C09820D64
:10A67200FC0E0F20120F0F0DF1FE80BD6A98120919
:10A68200040D0581408001620DFC04151020060CAA
:10A69200F1FEBF0705124E78BC067CC6007DC68E51
:10A6A200130110A9D09868F8F67B0DFC0B0519036D
:10A6B2000F0405D9FE009D0E809D66BF0E0E3D184B
:10A6C2000B802D4ABF0E0E4D180B805D4ABF0E0E39
:10A6D2003C180B808D4A870E050C01F9C41379C40E
:10A6E2000C1B06434E3005EA6DCC66A606E0980FB9
:10A6F200140179C40C1B2E53468D8C9C985606F57A
:10A70200C4B94A851A09130C068889E8B08BBF05BB
:10A712001A0913C15C4E70783CC62B0E1B841E3086
:10A72200107046F0A1144E708C60DE9C7E7E27264F
:10A73200D4E30A061E5C422FFAA6E30E8EE0E1C4C1
:10A742000459A4EDA456E63F3005426AAF089C586E
:10A752001C38FCAA0A7C28E04E703830081C901C79
:10A762000A838D150E0179C40C600B801162940F5F
:10A7720012010B80696660B0307CDADAFC3A307C18
:10A782000B00E00B00E0D05C3066603AC60E30068B
:10A79200A075227E477E59F37E19637E0D4EEDDA57
:10A7A2003CFE4E66A63A5C105C223730C6E3692E48
:10A7B200D05C30C6D7CC2B71CC66D3550E7C1C3006
:10A7C200060E7A30EA592FA6D3CCDD0E5D1C4CDF83
:10A7D20071CC66BFE92EBF0E0E3D3C180B80714A4C
:10A7E200F80E30E82BF80E3000E6AE6150600E56DF
:10A7F20037300306E3AE8D080626D3E07E7E89530A
:10A8020060065E46FAA056607CA647FCA62FFCA610
:10A81200B5A2E10A814081C866BFE6856813A366D6
:10A822003168C66687E61568D34BD05C30E613E024
:10A832007CE046E098E0D91C788C2B84D88423886D
:10A84200D888D8F0492660A0D91C783CD888D8FC92
:10A852009B81130F100B80096A0B80F96A0B80250C
:10A862006A0B00CD9E0286C6E0BF0E0E3E180B801C
:10A87200C54AD91C30126A5F78D88C1F881384D8D5
:10A88200F06330706A63411C30186A9D7E4EF00599
:10A892007E78E2D3411C4CC76100D1441BC17E19B2
:10A8A2007EC676C3A5D00C60C6762330EE134696DC
:10A8B200864686AE0E7C0A85D026E61C4E8223A6EC
:10A8C200A2A2A21F26E386EA02AA0AEAEAEAAACA20
:10A8D2002AE0856813E0A6062658D944E0EB5D1C01
:10A8E200214687010C060C0312B830FF3CEEB94A30
:10A8F20087010C060F14130B80FD6600203C5606E0
:10A902009CE23BA0005D1C21463087E099050B14B8
:10A9120005070B801D6681408488ED64BE583002B5
:10A9220089408808AD402570BE981D608CA7FE1F27
:10A932000E5B0E300555703BA00EAE00D164EE8961
:10A942004C690208A140257088A393100C03100BD8
:10A9520080696E9807120C030B80C162863E3C1818
:10A9620015C845CCB87CAA3CA845CCF5C4CEE87144
:10A972001E5CE6A616E61376A6E6E6E6C6A6D4149E
:10A98200A3E09828C488C4FD7E3E4E302C5808307F
:10A992004070387CE0304070387C063CA6BCF0E069
:10A9A20059A413A63040562B3001B6166660A5D0C6
:10A9B2000CA01C4A2A704E5CAA0A7C9C4AA606F08D
:10A9C2007C70383CA606BCF0FBAE0E7C1CAAFC0ECA
:10A9D2003040562B3001B6167030EF06383C6623F5
:10A9E2007666471C4A2A703866F308AE0E7C16302B
:10A9F2000156BF0670F038665BA6360670F0386600
:10AA02001B062B1C90D0061CE076173670383C666D
:10AA12008B3001763F2BEDA45626E66630075A139B
:10AA22003AC6F306E6BCE2667CE62B4E2E1CEA85AD
:10AA3200D04666064B66861C82A0A2A27BC666A58D
:10AA4200D046A063044E70F8EECE71C8700439D0BF
:10AA520006B0BCA6700C1F08B30C60783C06B03C74
:10AA6200063C068C3BB958BC70B95A3C70E06EA0EB
:10AA72005627FAA6F330030C1B6608468EAE608D8D
:10AA82000A304056A03001B616E0041308081B0431
:10AA9200044E7038DC901010102884444E587038E0
:10AAA2001CFCEADCD0BEEB59A4EDA48A1CEAAB0A7A
:10AAB200302C6A1F48B3885E5BBE980C23AA3C1BED
:10AAC2007CAA581C6A3005426AF78A985E630C2B8E
:10AAD2003C58BEC37C1C9010CB2E5F1C38FCCA7C39
:10AAE200288C6F0C0B0CA0CC23D5886A41A47B0C5C
:10AAF200A0986815980EEE734C670C771C9DA47C89
:10AB02000E7C0AFD1A0DFC0E010D05D9FE830512FD
:10AB1200140507884B8305120C031201840B80A1D4
:10AB220052E54C0CA0983C063C4C3B0C17060C130F
:10AB3200463CA63C9C4A0EA04E2F8C7B5C628E66E5
:10AB4200665C1BFAA642EB8C13BE600D544924F8D6
:10AB520028AEE8B5BCFD5A064C2B48B03C06CE7C6C
:10AB6200A6FCEEB0FC061C0201D08408CEFCAA0AA8
:10AB72007CEEEDA456E6C6762697CE7C4C1F2613B5
:10AB82006603047CAA0ABCC6BCEE8CC3B07CA626B3
:10AB92005F0C4FA646BC26BC703A4BA626E6EDD00B
:10ABA20063FCEEE626E6EDD00C604388983CAA7C76
:10ABB20058E0CE7C0698E6B07C463C70B0FC70BC97
:10ABC200A63C66063CF0E09301051601130B809942
:10ABD200568891D04E70F80E300255701BB5A2AE59
:10ABE200BCEE514C4E70783C06F8C4FE1388CEF68B
:10ABF2001348A67C9C4AFE1348A63C583154BCEE2E
:10AC02008940A808B156BF0E0E3D3E180B80A14ADE
:10AC12004E75F0EE600DFC0E0F200412091605F1C0
:10AC2200FE8C06130F1049F0F9C40B80E6E956BDFD
:10AC320056585D1CCC604C6060B03AE08D0F0F122C
:10AC42000D050B809D5A8215131405074433901489
:10AC52000507480B80594200BCA8E04E00704468CA
:10AC6200780605BCEE59DE785E3E683C0666040155
:10AC7200AC0EC1B01C0C0742271D145BAE01206351
:10AC82000C77AEBC4D14DDAC4924E304B1BCC36EF9
:10AC92006EC9A46E085346F059A4E5A459A40466EB
:10ACA2008E060404D91078065830301C622B30B05E
:10ACB20062275613B6D91CB8B81C101C8C3342B884
:10ACC200302DE876B63CA23C3E1E7E7E8518492495
:10ACD2005DBC99C844785CE291DF3084CC2766EB96
:10ACE200B371CC663F785C62683DDE309366FBC828
:10ACF200CC2FC8CC0D541C101C02784CBB426F7672
:10AD02005B6267A21C10101C021776A268C34E5C1D
:10AD12006244D302FDDA3668F6F65BE2E21FF633EE
:10AD220078562268E201DAFE435CE2234830F02BD7
:10AD3200C1B0BD1C03011420050D101419DDAC08AF
:10AD42000170650E4E9C90CC67601B7A1F7ACB888F
:10AD520059C8550E1CA020E2F9CFD91C78584924B5
:10AD6200300501ECC27012C38700233BB313BB0D45
:10AD7200549B8CE378068605BC95BC668666080102
:10AD8200AC4359C85B785C42688859C851DE8CEB89
:10AD920048C393011405070B80ED52000000000028
:10ADA2009805160113883398140507843DF0B00600
:10ADB2003C2606F9FBE6C622BC70067CF03DD04E6E
:10ADC20070F8AE708C2F38EEB94AAEF0E048F9C494
:10ADD20046C10238467CA65849F0DDD4B0E622FCD2
:10ADE20006023DD08A983C0A05CC98420C172E0ADE
:10ADF200F9FB4EB07C5CD070FCE090051601130BA1
:10AE0200803D6A4CE57A040D7CF57A0B8069460632
:10AE12007038F61366663C1EE0D09C30583A1C3AF5
:10AE220030E63A30C64FE63F5C50D0D0F19AE60E9B
:10AE3200BC427CA67CCA70BCA6F6F6F6E33A3A0E91
:10AE4200303C1E78AE7E3A3A306A677E8E8EFE2F96
:10AE52004A2F440B4A97BC430E98AE7A30EA8304D9
:10AE6200D88C1B8408D86A3F8E8E0C374A77BCFD7B
:10AE7200E24AE748B19AE6C532308306CE3C5666CE
:10AE820037B85CE2E2E2313238FC9CA262CF1CA20B
:10AE92003C28352EE0DCA0DCF2C156A00EAE1C72BE
:10AEA200CD564EEB514CD1C8E653D144E0C4F57EA9
:10AEB2007D6813BB664670385C5228A658BDE0BE5A
:10AEC200EF983CA6BCBE580948EEEB86983C703819
:10AED2000EC67066E6386E33EE773A6E5F30040661
:10AEE200983A7EB75826371568A30DFC0E0F20132B
:10AEF20015030820010C0DF1FE266F29E60948EE24
:10AF0200DB33D1C8E62B4670F828B8EE4670CEF097
:10AF1200F1688E1C527C706944E86E754CA898707A
:10AF220038F6274E70AB98267038463C05688D700F
:10AF3200CE0EDC52BC702626694468454098803D9E
:10AF42006A84050B800172840C0612038443930108
:10AF52000C0612038801C8E6B5A2DC908C133E6889
:10AF6200BDD00881F08CA1C34E70780666263DC222
:10AF72005AEEAE3C700698F00DD0A6065870CEF090
:10AF820070088C6366700201D030FF8D8CA65898D1
:10AF92000E0DD0A65870B0662F704EF09B0C234E4B
:10AFA2006EF0C102847E1788B0FC580670BC9C4AC1
:10AFB2001CBCF004738C060C033EA5E8B07E7E2B0D
:10AFC20089F63E8C1B78EE55F2BDD07DF20DFC1257
:10AFD200050320140F0F200C0F0E07F1FE92080339
:10AFE2001010018408B5E00CAFCEBC06B07C8C2FEB
:10AFF200A63C707C26E6CEFC0AEDD0AE7C0E98060E
:10B00200CEBC4630FF063B3CAA8D8CB03C0698E68F
:10B0120071D8849803920803130E09884349EA837E
:10B022000512130E0904B5E00CA7B03C51D8CE3C72
:10B032000E889826587C9C0A7C1C0AAE7098E6ED15
:10B04200D0B0AA7C0EEDA4AEFCAE8D8CAE7C0E7C94
:10B052006A93846262901C622751EC02AE8C2FFCD0
:10B062000E888B987C0AFC66588C9BB38305121061
:10B0720010014404B9E049D8987C0EFC2BEDA45988
:10B08200A4AE7CAE8D8C01D098663758AEFCAE7300
:10B092004C6030FF8D8E8C061A1305120B807D4A90
:10B0A2005ABC1A203C06B0303AE62366DF461AE064
:10B0B200411CF53E30EFB616666F3001B670387C33
:10B0C20006562306B66666E09819050B1405070BAB
:10B0D2008005427924B5BCC10208D8284E2E68707A
:10B0E20088C4651C0488ED06000000000000000012
:10B0F200000000000000000000000000000000004E
:10B10200000000000000000000000000000000003D
:10B11200000000000000000000000000000000002D
:10B12200000000000000000000000000000000001D
:10B13200000000000000000000000000000000000D
:10B1420000000000000000000000000000000000FD
:10B1520000000000000000000000000000000000ED
:10B1620000000000000000000000000000000000DD
:10B1720000000000000000000000000000000000CD
:10B1820000000000000000000000000000000000BD
:10B1920000000000000000000000000000000000AD
:10B1A200810F1418F8EECE7EFE595A15C89C5839F4
:10B1B200B69209040D052E009170A56CBDCC064611
:10B1C200BCA63CF0BDCC26BCF0883E4E5859F08C53
:10B1D20053C1B01C4E901A987C5875B0BAD3302027
:10B1E200E8B03000E6E6C67EE3E8B0DCD00EA1149B
:10B1F2004924385E285DBC8001529CC22B387C6693
:10B202003B0D54663002C61306F5C44E708CB55120
:10B21200EEE8D5CCA6A62FB5BCFD5AC1B0BD1C0424
:10B22200091220050D101419DDAC080170B902DCF9
:10B23200901BDCD0FE84480453DC501BDCD0FE049F
:10B2420044848404040E30407030BF0638661B0804
:10B25200634C537C66B5F7EE7CE6FCEEAE0E3CA684
:10B262003C263C0E0C7F7038AED86E1788D8AE2EB6
:10B272006F8C1B6E582DD00CE7A6067038FCA60604
:10B282007C7026E63DD00C6F4C278C5F83CE7C66AB
:10B2920037FCEE4B84AE0E3C06704E6EF00C278CE3
:10B2A2006B8485D0C6A686A6A5D0469330EEA62688
:10B2B20086065C424F9B880C2FB0BC16DEBCDEF3C8
:10B2C20076E30DFC060C2014191005D9FE0DFC06C0
:10B2D2000C200E0F1420060F150E04F1FE1C304038
:10B2E200704C57AE0EBC06387CA6BCF00CA04E2E9D
:10B2F200BC30BFF0E09208030C05048843830512BA
:10B302000C05048449F08808E9D48CF9FB8C7B4E47
:10B312007001C898A658CEBC06B07CC6E698A606B0
:10B3220027C6DB0686A6467098C60658CEBCA6C6B9
:10B332003CAA8D8C98E63C0AEDD0987C83B07C4682
:10B34200707C707CF0CEFC0AD9D0CE7CAA0E84ED43
:10B35200A4F0664BB0561C2A13886A1CF0AE7CAE71
:10B362008D8C8C60A293A63040562B3001B61666A7
:10B372002F70383C06A2A2A28CAFAEFCAE88338CF2
:10B3820006121510A068A5E88EB05A580881F098E8
:10B392006E46262642EA4E7078063DC3BDCC46BCB8
:10B3A200F0AE0E3C0A3DD0BA3CE6A670A638EE706E
:10B3B200EEF0DA3C66A084A63040562B3001B61679
:10B3C200661FA5D0668C27887B9812051601138804
:10B3D2003B9812140507843DF0B0588891D0B0060E
:10B3E2003CC61306BCA606BCD870E63C462683269D
:10B3F200E698A658B0FCA61C223DD098EEDB92142B
:10B402000507843B920516011388DC90FE95E8C17E
:10B412005C4E70783CC6A660E6B006978C730DFC55
:10B42200050E04200F0620060CF1FE66A6C686BC99
:10B43200A6BCFAB0FC060DD07AB0FC70BCC626BC25
:10B44200F0AE7084448C57A67CA63CA6700488B3E8
:10B4520008849B90011713070512484B85160F0DA0
:10B46200070512448491D0E6136670063C063C063A
:10B47200B958BCB958063C0627883C70B00E3CA6A9
:10B48200BCA670840404B07C7038EEB07038EEF064
:10B492004C33B07C70CEF0B03C66603C048C7F8C48
:10B4A2001B661326700C600CEF3C080C9B700E2D73
:10B4B200D0B0A68BAE7C0EB0E622FC06023DD08A4E
:10B4C200AE0E3C0A05CE94100B050513844B811475
:10B4D200100B0505138889E84E7001C8FCFA1E7E20
:10B4E2007EB0FC70BCA6063C463C7080C15A9410EB
:10B4F2000C031284438114100C03128889E8B03CB7
:10B50200A6F5C4CEF07C06F5C46EA05A233003C65D
:10B51200B01D60EEB94ABD1C20051212DDAC080157
:10B5220070ED8AA188C1B0BD1E492404CDB4734E0A
:10B532005C90D0D010309C6262BDC06B49A43DA427
:10B542008A3DA4E5A4581C22071CAA588CDF6AED88
:10B552001898EA6DCC3010701EA114D91C7E9EBEC4
:10B56200B8BEF37EBAFC8518F90E46F070B85CE2FC
:10B57200E2E24660E21BAE4BAEBC067CA63CA63CB9
:10B582005EE000000000000000000000000000007B
:10B59200000000000000000000000004320605E880
:10B5A2000000000000000000000000000000000099
:10B5B2000000000000000000000000000000000089
:10B5C200000054000000009001000000042AD0880E
:10B5D20022282280008051018045028001C055044A
:10B5E200C0242200602411005400500140050024B0
:10B5F2000204100D2002C05000000C0C00E0344F79
:10B60200C8834F8A4F3C372C8E20C13B08E168101B
:10B612000D204E064065F3B8144DBFF48308922204
:10B622000159C91D744FCC78E4452FC2F102005470
:10B63200D450C1D8C430FD3A06FE876130164E415F
:10B642008660434BC43D898BBBD1D3BB03101151E0
:10B65200D100034035312DE212133131D5C1725080
:10B6620031E04C0005D10444151E50455D4C762F47
:10B6720003005C000000194207C9C40040660216BC
:10B68200F6460522501012B4CD460A001900740085
:10B69200318F4F40384454F37F2B4147888714E061
:10B6A2004331410F3C4A3490099411403141663094
:10B6B200CD2823514ECA60CAC01F8FC2E72F08018E
:10B6C200B60501C2C8105D07FC2210301100FB0450
:10B6D2002244448C738748E0C4073D03A3064AA46E
:10B6E20080C1084B31C1142013044B03D60F1B0237
:10B6F200023D0CC1E724E2005108600080000052C4
:10B70200D147842000923374CDFD6405C111110428
:10B712000004F04020800661761402C40464001222
:10B722000012EE450D0511A080390010214841009C
:10B732005238B18C40225015F70500549C0B006022
:10B742000020409A25CE660040050002205D3EA9F9
:10B752002686E8B534D00C004033C14149C223A348
:10B762007463C71333CDEFD27188521027BAD2E374
:10B77200C4B84EF9F3B5A78448F623C2BAA245214C
:10B78200A28D6CF63300004E32C884B83260301D90
:10B792000100104CE98608B7203B2AE10E0019008F
:10B7A2000008804278001A0A820280078F44220031
:10B7B200215410E1417004001D65155D2275F3B836
:10B7C200E322C140244354689FA88F2F638F854B87
:10B7D2008B3D1F4FBCA244C05C357A9F2B0896D488
:10B7E200C515724F45A1214505910921A130E244B9
:10B7F20029BD290000603C981F8E0488466881910B
:10B80200089282470BA9C55401110002008620A2AA
:10B81200833C683D40964089240204500189800798
:10B822003A8A500A640200E8C0A48C080000600052
:10B8320080C1612444020555582C00146001800E19
:10B8420000040F80996110440009001073CD003C80
:10B852007D840900500011C8000049C01D00007419
:10B8620094D4CA63114113480DD4000051DC70987E
:10B87200191300000000000000000000000000009A
:10B8820000000000000000000000000000000000B6
:10B8920000000000000000000000000000000000A6
:10B8A20000804A0C00404613912302090D54171DD3
:10B8B20053B58F34215E94A01611043630C5D10CD5
:10B8C2000080938C20000802F01246CC8002001403
:10B8D20048273487818990402022708281538902CF
:10B8E20031057041D43D51242300600800006010EE
:10B8F2000215828F8403800080427218468451C4EC
:10B902004820514800511110204241B420B02C006F
:10B91200F0514CD008550B3C00094048A4803E032E
:10B9220052098180487F314103FC038000A010420C
:10B932000451019D4400480420002800E0D4302234
:10B9420000008640040480620208117C1F0000008F
:10B952000088488851C41004C14B02824022380C2E
:10B962008838C693C014400854000003000C1840E5
:10B9720081124404C000C0000454E04400308093AB
:10B98200CCCC4406F5BF5A318CBC41400484CC4037
:10B992003708C25EF501D4080C0000000000004028
:10B9A200441348AD7056390C51844E584488A180D6
:10B9B20095BCF0B3D5888A3E23E6D7ABAA0A704D70
:10B9C200A47E7C81BC8D8CB0AA39887309504E5BF1
:10B9D2000CDF98EA2DBE0AFC4DA459A4AA0A5829E4
:10B9E200A48A41A4CC57980647662F022762130AFD
:10B9F200AEFCCA7004B00A8AB0CA70E5A47CE21F29
:10BA0200F6B362BF62ABF62BF61BF67F0C5B980AAD
:10BA1200468D8C59A498AA58081304B00A7C060FC4
:10BA2200662F02EF62DBF5A8B0AA70E5A4EA98706F
:10BA32001CA18C98622362626E6258B06A7755824A
:10BA420046FC708A980A29A4BD8C6ADB20B0703843
:10BA52009C5898700E388E8E1CB63FB6DCDCDB022A
:10BA62007B4AF01C6A101C02BBA666700A4EF09854
:10BA72007CAA698C70389C98F0467078A6682E660D
:10BA82000DBA6670EEF0EEC34670781C10701C0A98
:10BA920038E039883E37FEFEFEB183980A7CAA69F7
:10BAA2008CFC4DA4AA58B00A4DA4AA0A70E5A47C45
:10BAB20022DDAFE078E64E30C058708370383E9396
:10BAC2001CEA277CEA2371841B5584C606B0666F84
:10BAD200E07EEEA0FEDC58B098701CB0FC6A6F7C71
:10BAE200705584DE7985AB00000000000000000084
:10BAF2000000000000B0702E70380E3B5584987024
:10BB02002E58AEF0E07858EE8B1598EE810A4CEF85
:10BB12000C27D588671CB1182BCCC3A918AEBC3032
:10BB220076767627D588437AFA851406DA1A3006AD
:10BB3200098366E64670787066BCFA38D884D8F015
:10BB4200BA3A301C62027CA23C0E3A300A7E27EEE0
:10BB5200EECBEE3C7066EEAEF0EEBC663FEEAEDCD7
:10BB6200901C3B3C2606467078A6681C02C4BD8C1D
:10BB720009B81D02B8463C584484B0E06259A66E2A
:10BB8200E0C461A4CAD844D885A43C0AED1ACCA06A
:10BB9200D5886A66A08CE746E0000000000000003D
:10BBA200386B3823380338E338C338A338FCE00055
:10BBB20038E038933873385338333893387CE03C64
:10BBC200E07CE07CE03CE086EA667038CAE086E62B
:10BBD200667038C64B42EAEAEA22E2E61FC61BC694
:10BBE200360A1B261B62620A707C3020FCE0AAC364
:10BBF2007CD80CE92F758879A085140CCD07190221
:10BC02007CD80CD12F758841A4F80C83E6DDA96598
:10BC1200504C1346261366E8DD8CFBE61F26E865CA
:10BC2200144C1938655026E8E55C75067858EE879D
:10BC3200CC1F41A4A1A48584CDA8884E66480B15CB
:10BC4200981CEE1B0C7B810AAE668F840C731B88DA
:10BC52004E704C47CCC98F41A4F8CD84E844B0441F
:10BC620070198C4C27B066CB95A47CAAFC61A47C8D
:10BC72000A4CA9A76550E62398ADA01D0245BC1148
:10BC82000C711C2DA84CAFE0390C0860BC580CA0FC
:10BC92000498DDD83BA188B030C570CC1F4C1B790D
:10BCA200A055C42DA87BAA0A584888F5A898AA5876
:10BCB200334E59A48D8C986ACFE0AA8A700A7C30E0
:10BCC20083FCE0AE1C8A700E7C3080B31DA44BCC8A
:10BCD2003F4E70F84666E8467038AA0ACC57E2131F
:10BCE20022E21322E2132228E04CC98259A49DA425
:10BCF200AA0A29A4AA5839883E5F488C337EFEFEE0
:10BD0200FEE3B0E098EE4DA4E5A41C6A4F06E64EB1
:10BD12007005BC95BCCE581C0A59A43988FCEE9813
:10BD22007C1D88EE7CEE6A46174636360627767606
:10BD320013266A698C980A84F5AA584A174A4A2334
:10BD4200666262E6E6E6E61322CA101C0A986D8C69
:10BD520098E0B9844C1187AE41A444F8E633E5A8D3
:10BD62004C3748655026E8DD8E30DADADAEEEEE05E
:10BD7200B02BB03A707A258CF3B02BB03A707A259A
:10BD82008CA3B02BB03A707A258C53B02BB03A709A
:10BD92007A258C3A3A3A7CEEEEE0B0703C467CE092
:10BDA20066BC1C3A3076F6E7E23FEAC3666AAF0346
:10BDB200222222227B9C229F224F3A3A301C2227A7
:10BDC2004E4C7F488EA9186EBCCB3A3066AF7A7A59
:10BDD2003C1CE044448641A4CC3FC6BC584C1B4D9D
:10BDE200A4E5A47C82E2DFE237E2AFE223DDAC939A
:10BDF200F68384763CAEBC9C98161C66673C0E2982
:10BE0200A48C29A54E70AAE03C0EBB59A4A3E2E77C
:10BE120036C736C739883EA74C2FED1848234C3B0E
:10BE220041A44DA4DD8C4E70E0E5A4884B7D9C9826
:10BE3200CCBF4CAF4C9BCB5C42EE2B0E4E701C4ADF
:10BE420033AA7C8E8ED33C58681598EE9B0C1FC487
:10BE5200934C7B8CA758B8E683B85898BC30E64B15
:10BE6200E0C81C0A1DA4A37D9C8411007EFE4B8D9C
:10BE720008063064069B8D901C0AB8E6B38A636A92
:10BE82008686A644D190EE60810A4670CC2FB858BF
:10BE92004C83B80A38AAFC0EF8FCAAE8AE0930AB0B
:10BEA200EA0130091E04CC7F4C6F06984C8D900C31
:10BEB200870ABD8CC102CC330A0238BC3A30A6B61E
:10BEC2003A30FCE64738AACA0C4B8A3B384AD308B8
:10BED200EE41A43DA43DA4AA0A559CEE530C3BEAB4
:10BEE20049A4E5A4D6E63342EAEAEA22E2E697C6A4
:10BEF200EAAD3CD86A8C8346425366985846704BEA
:10BF0200C63673A2A2B3AA62620DA48308AD3C84B2
:10BF1200D8064891900AD8662702331B061B04AA4A
:10BF2200464223666262E6E6E6E61322CAE641A4D8
:10BF3200EDA47CC63CFAFE8D8C59A4CE7C8D8CE59A
:10BF4200A4D8840C1388D88D8C980A759619085633
:10BF5200A08A16CCC3468B02A6588C3B849806381E
:10BF62004A4B0638AACA237D900A499646BBEAEA9A
:10BF7200868638E2AAE2270DA48B462222421B665D
:10BF820053A2A23B047D905841A4709866270233C5
:10BF92001B061B08AA0DA45697E6567FE68AB0AA8E
:10BFA2000C1322EAEAEAE63C8D8C9825961C903C1A
:10BFB2001E98EE6A21B0001CF61B101CEEEA3CEA49
:10BFC20023BE2F7B3CEAF358845C4E7050FADA9C15
:10BFD20030583A30E6575CDA22A3E5E200D0881CFA
:10BFE2003A308C97E63A30C61FE663E60EBC427CD6
:10BFF200A67CCA70BCA6F6F6F6A33A3A0E303C1EF0
:10C0020078AE7E3A3A306A677E8E8EFE2F4A2F4491
:10C01200E34A97BC631C06461F4EE030DF0647C664
:10C022003C020ABC059AA6FCCA221C70BC0E98AE41
:10C032007A30EA8304D88C1B8408D86A3F8E8E0C2F
:10C042004F4A777C8C173C019A4ACF48B09C108C9F
:10C052009F0E3C7A7AFAFAFADAFAFA9C98FAFA9C81
:10C06200901CAA08E0781C101C0A70383CE6359A2D
:10C07200D5883ED37C62588ACAFCCA0E4DA459A404
:10C0820098EE6E6E1CE5A46E1C6A578E8E986258EE
:10C09200E24B4A871CCE7C0ABCA34ACF4670CE7CB8
:10C0A2000444E0441CCC1F4C3BF80E38AA7CEAEB5B
:10C0B200C8E247C4EAEAEAE66FC628AE4A7CE8F874
:10C0C2004666E8890AC6369B4E7048D3C44CA0F82F
:10C0D20046E8CC5795A43C0AED184435BEA918DBB6
:10C0E20036AF335836C7369903CC1F4CA349A43D0B
:10C0F200A41DB43C3E6B980E4670110C1B19088CA3
:10C1020060D91CB8492676C321067858EE319EB80C
:10C11200AAA81598EEA19268B806FDBCEE3BB80E2F
:10C122000801AC1B95BCB806EEEE787CEE0CFF78ED
:10C13200AE3CEE1C4DA459A4C1A46E1C6AA06E1C98
:10C1420058EE8D8C1C98EAA0AE4670855201AC0C5C
:10C15200604ECAFCAA3C7EEE1DA0EE3F706E85507A
:10C162000982705838EEF0982606C3E08E85506E2C
:10C172000801AE41A4CC2F46CA4602B8AAA8E08C58
:10C182009F061CC3300B0604B898A8A63CB0FC1C42
:10C192001086BC5C221B29CA30E6D3E000000000F6
:10C1A200382338F338C3389338633833387CCA3C81
:10C1B200B3FCCA7C933CCA7C737CCA3C537CCAFCE9
:10C1C200333CCA7C13CAF01CE03CEA7C23D58822AB
:10C1D2003803389338633833380338D338A37300BD
:10C1E200385B3833381B38EB38BB388B387CEA3C49
:10C1F200EB7CC2D63CF0AA0A6E701C1BFCEA7C7374
:10C202003CEA7C537CEA3C337CEAFC13EACA47F002
:10C21200983EAE4670E011A0EED3A5A461A47C1DA9
:10C2220088E6132E698C980A3C1C2376DCDC76E3C4
:10C232004E70786E682E70E638E66670E6F0E62696
:10C2420066A7E6AEF04EAAAE38AEF09870384AF065
:10C2520098A9A6980A4329A44685A47E58FEC74CED
:10C2620013C809824E1C70786E700638EE2F30C0EB
:10C2720006A04EE0CC8795A43C0AB18C41AA2DA819
:10C28200669FE68BE841A4CC2FA1A4D84A27095087
:10C292001B29A4EDA47CC4483BFCCAAED851ACD83F
:10C2A2008AAE06B7662F02976A833CC9AABC0830D9
:10C2B2007A76EF3C7E45AAA3583C0A4DA4EDA49C95
:10C2C200D08D8C98E041A4AAD8A1803C1BD588D8F7
:10C2D200063F6660021F62607C8ACAFCD83E67D84D
:10C2E2003CCA7CD8447EFEFE1348E6170A4ED8E0CC
:10C2F2004E70381CCC17E20AE01CAEE6BD9E5A26F0
:10C302008F263B301D7C44D1026666FC084DA8C5D1
:10C312000278101C0A703988E62709503BD5883EFE
:10C322006F4DA4E5A47CE21FF6D3B06ADB11A0EE48
:10C3320009829C101C3020F0B070660A38D884083C
:10C34200D8F04E70786668C4B18C0180BD9CC10281
:10C35200CC53AE0EBC30E04DA459A4AA0A707C3076
:10C3620021FCE0C6C2A0BB1CCCB76262627186CC63
:10C372008F1C23A237A2A22FA2E0A2A2A2A2A2AE47
:10C38200E06EE0469C5845A4AE58707C9C98E61C32
:10C392003084FCE0C98C8ECE5C581E99A49EFE5B54
:10C3A2003E3EBBF5A891A4CDA883FE95AAFEF75CFC
:10C3B200224BFC261CE2CF8D8C8B22A7042217086D
:10C3C2008DA4300F0C2391A453F5A82691A48DA41B
:10C3D200CDA841A459A49DA4698C7C698C0C63FCF2
:10C3E20061A40A4DA4DD8CF846E8C502FEFE37CEF4
:10C3F200DC95A4BB5C62439CE2B790FC5DAA6283BD
:10C402009CE26FD0BB8DA4FEFE33FC261CE20FD053
:10C412001DA45378EEA091A478CECE68C330F0AEBE
:10C4220058782366CECEEEE798AEE0F8261F66E097
:10C43200044E6EA05CE070CCA795A40C133C52D8BD
:10C442004A431BD5883E33E6DF09503359A4E5A49D
:10C452007CC4488AD80EB0CA70AED851ACD832AEBD
:10C46200724B06AF662F028F627BAEE3A9184EAA0B
:10C4720058AA0C41A4B0AAD80E442BE5A84C3F728E
:10C4820098121B0ABFAE707C066550A01C4C60A6B9
:10C49200E8B00ADD8CF8E0C41BC488CC27E5A4030D
:10C4A200AABC3A30F6EB3A3076EF7A76E11B488C4A
:10C4B200A91A7ABBA24BAA626266700A387CA27C75
:10C4C20082E2FB2222A0F62BF61BF64FEACA8DACC3
:10C4D20082E25322223BF6ABF69BF68B29A43CCA9E
:10C4E200E0E2EBE2FF36EF36DF8C258F8DAC8DACD0
:10C4F2002237484C6029A429A48C173988ED1AE206
:10C502008B8DACA253AA101C66700A38FCE0A27C88
:10C51200E0E22FF66051AE7660EA8DACEA76DB039C
:10C5220004781C10581CFCCAEE30BF26AED8666BCD
:10C53200D8AE7070383E437E1E1C6A237C6AE74A7E
:10C542007F1C8A8AA6B63CCA087C7E137CF03B0C10
:10C55200234A3CB33CD84670D8E0B083D813AEFC33
:10C56200EE707C1C0A3988E6CBD5883EDBFCAA0E2D
:10C57200584DA4E5A48A1CDA7C0AFC6AB74A5746DD
:10C582001CDA707C0EB0EE730C33466E8D8C3B98C9
:10C5920008231C980A7C8B3020061CF86AF3B8E04A
:10C5A2007F61626364650060060405010C1D7E0DF7
:10C5B2004EF05C90308C3C0EE5A41CEA5730051C12
:10C5C200426AB7C1B06B3CC1B0E02B6E30051C4271
:10C5D2006A9F9E301F0C23E8BE3726BE1FE8EBE0A1
:10C5E20020DE6DBA5E270C71B049241CE5A43C8E96
:10C5F200D91C7C5675B0AB3080A330C08B06163088
:10C602003A66AB302C66A3302E66F7304006B8D8B7
:10C612004C5F8C4FD8DC101EDE7E3353D8E83020BE
:10C62200DE237EBE7E70E8E01630200697305FA6DD
:10C6320006DFD844D806B03070A646A0061B4E5C72
:10C6420090101C30663322E3303A5B3C5636230EA0
:10C6520041A4C1A41C426A60FC5C021DB48E9C58B9
:10C6620006164670307F66851DCE0E1C7C66DD8FF9
:10C67200FC0E1DB48E9C58467051B473E0200C60C1
:10C682004C3FC8CC37486D00CC603080E666FBE09A
:10C6920030107030FDF09C4ADC909C905C901C90B5
:10C6A200282828E049246E1CCCE5A66EC9A6381CB1
:10C6B2003CEA6D591C387C0EF87C0AAE28B87C0A1C
:10C6C200AEE8787C0AAEA8AE9C9868E0E6251CE647
:10C6D20056069C58B87CD804D83CA8F6F62F468754
:10C6E2008CE70C23300BE08C273077E03087E0308A
:10C6F2001C66273054E09D580CC92289BA84B89828
:10C70200A82B88B898A80CA78CAB307F069C98E61B
:10C712008D2666AF652083B83CD808D87CA8D9207E
:10C722007924BD2025241D0239B478FE37FED91C98
:10C73200B81B09B8469875B031B8638C41BB41A4A7
:10C74200198C4E70D92041A41E8EE5A41CEA2B6ED2
:10C752008DA41E46700C1B29B8E05CA078A0FE7B5D
:10C762009E60FEDE7E5B8C4BFE301A31B8B37E607B
:10C77200FEE0D4577822AF145762DC5058D4A09907
:10C78200A4130C778CC37EB77EA7C314B794A70CEF
:10C79200931CA0301B31B878F65329B83BA08DA466
:10C7A200042BA08DA4088D141D02301C9C5899A640
:10C7B200307F66937846977EFE2F410CBD8AAE8D00
:10C7C2008C29A44670AE68633E236520E3AE99A42B
:10C7D200BE008B1E41A459A4BE1EFC1CD08D8C7EB3
:10C7E2000723781E9ED91C5EA0BEB8E3301FE83036
:10C7F20020DE7E6F1E3E5E23E8BEE346F07068E0F8
:10C802005ED3B8580C373CD888D87CA8469C98068A
:10C81200307F667F781CEA3FDC10FED91C1B09B80A
:10C8220061B6851CDC10FEC1B051B6C98C9C9870F3
:10C8320041A41E30F19C5899A4B09C5899A4AE7E94
:10C842006815BA4E705C105CD0100EB8B03C06FA97
:10C85200FA7C4638BCA606583C28E0E6174E70091A
:10C86200503344A180AA70040A4DA4EDA4D80C2729
:10C8720004D8330804D88D8CB00E3988E603D588E5
:10C882003ED7AA0A704DA40CEB08EDA47CA24BAAD9
:10C89200626266700A387CA27C82E297E2EFE277FB
:10C8A200E263DDAC4BB0E60F700C4B41A44E70E876
:10C8B20028DD8CB8584CA0D5885FE27FE217365F3E
:10C8C200364F59A4E5A47C22D7E38DAC0BEDA47CB2
:10C8D200563C8D8CE5A41C4AEECE8D8CCE7C63E555
:10C8E200A41C4AEECE8D8CCE7C1BA6FC586E1DB4C9
:10C8F2001C980120C3AEBCD91C0C733A3A3006A670
:10C902003C2EEEB9BC04D5124D140912D91CB9BC87
:10C91200CE3C061EA114B81CD0E8661EA11463A664
:10C92200EE1C1084101C421F02889C1BDCDCB6EB40
:10C93200E6161FDCD64E94602213E2B6F30EF88C94
:10C9420017B858B0E0EE2798022398AE4EF0E0CE2A
:10C9520070989801207B0C3FB858B0AEBCE06E4D89
:10C962009CCE0592810A4404040C4745A4E5A459CF
:10C97200A42B6E2DB46E66E66ED91C4CD9B0D912BA
:10C982000C23EE58EE04D80C23080408D8E0BD1C92
:10C9920018120F0D20E000000000000000000CB98A
:10C9A20062204038238038C4F800C4039D1033D479
:10C9B20010D0CC0C0011802C2E122151C0441171C8
:10C9C2003333809043A21A1F0035802093C1477FE2
:10C9D20020C4A3612032E2CCA3C838491C52498149
:10C9E200304443C8C64304224B1204F1EB003038F2
:10C9F2008431000000A00091869B8CE3321070D03D
:10CA02002A8348F420B806B3F836E2C90F0A9280A6
:10CA12003D86330033E3C94D03DC50C18323030059
:10CA2200440400300C00C07C373B280C0A5359CC1C
:10CA32008A6892C4BDCC0431BD4C0C0E04E2A078CD
:10CA420038E00326143003DA203E180470483C4BC9
:10CA520040E000002920CD9C84FC92EE2E4F87C03E
:10CA6200804CE14430D00F461263E483E0384E102C
:10CA720086E1330334141258D131B2348A104D4056
:10CA820004C0A0A20894D3206A153E053D0BE132F2
:10CA92002138FCD7913944E6109943648E7A557255
:10CAA200B4EBE27EAA2FAEEF8804E9AB701248C461
:10CAB200C87675C4BED2C4D03CC8E4E8E2E1121A1A
:10CAC2003180CB4E02C258F8F06F8E0808A57D6DFA
:10CAD20041C308EA1433A4015FE083F26043820099
:10CAE200C02C50CE0743710E6E4C8FF7C40C0D064E
:10CAF200211895C54C4851A37B8DCE8DD7D40C13EC
:10CB02008A5A851332020C836C3854C8030C2CDE0B
:10CB1200D1C404F37FC49C46D74D41334CCC3C0F67
:10CB22006195D01805C2D2A0C47A84C1E3121ECD89
:10CB32004EB838910C51A57DA23EBE8C3DD2704FAD
:10CB420060813B152E2DF67C3C70BC08A4561794D0
:10CB5200824F240AE00A40330108CF23F240F8084A
:10CB6200BA08D92008553CE038ECA8FA0C5021C488
:10CB7200722208C7805E0808CFE1608E388E166286
:10CB82000B622F880833C20F01E7A0080328232273
:10CB92006060FE084B0087B8C3913F2759227B0093
:10CBA2000400008C00444400C820CB0DC4CC8C2867
:10CBB200C404008C0C4AFA0011110088093E064098
:10CBC20088508FEFB82BA0880F0260824D3180B958
:10CBD20008E01A12CF000522EE0741338C3C0041D7
:10CBE200F0F3DFD43ACAD5C843078D40F3F30049C6
:10CBF200515BECD038508380486C28C91C113280BC
:10CC02008C2CCE8CC094688C8B3B003040FD0C4940
:10CC1200520D500D40145D55373324C34902C318D9
:10CC22004A4C50D8821B6449133184331103820465
:10CC3200D0C03C09CC4B0EE0394F8EBBB33EBE0791
:10CC420049EFF1E22100414403880F230F0510242C
:10CC5200F3F30F015540C544CD03013C13FC0C48CE
:10CC6200E4EEAE11E1816ADC861EE11086D2ED238C
:10CC72008788181116CF704444301ADC878313B8A2
:10CC82004C01847421983DCDF02034C9E0868D0199
:10CC9200008580438D30C40C208103604861F4FF1D
:10CCA200000000004C71B204FCE0180143C461BCF6
:10CCB20013D30422336110447C7C4CF4217B0C1F7F
:10CCC20042FCC40473D7F14CCCE3313821E3103079
:10CCD20081F11008040CC2DEF228DFF9611C203059
:10CCE200D50148E23A7B1D76D411D30434F7773567
:10CCF20000B1C4714C2C48F0C74F128D33C2FD0DE8
:10CD02003131A0301310B1108010200B030A302AE9
:10CD12000A3204AC608A38CC3C23C2CC4C800A3242
:10CD2200C1141333F18E22020C2222327131E443F8
:10CD32006ACCF771203937EBFCD4DF4C312DCE10A1
:10CD420032CE880C41CC30830236DF5B91D1B8C140
:10CD5200E4008D3C4D0F140E4A4C2007AA71DB51A2
:10CD62001DA342A0C3FB102632B21ACA083200BC6D
:10CD72000C008F0002D0805EC834233310F30F738F
:10CD8200DB2E0DDFCFF152F7D84B123A30000FC530
:10CD92003043CBC810240C3341B4E43F000E0040B2
:10CDA20041460000020103044247000027242120DB
:10CDB2004348000028252200444900002926230078
:10CDC2004540000F800000981E19B0456C63AB13FC
:10CDD2000D08B0C964F0B8C9640EB01D6088C9649A
:10CDE200CBAD130D08B0BEF053ABB063840F0DB0E2
:10CDF20071643BADB0BE001D606902AAB03560D35C
:10CE0200A5A6A6B035603102B21E18B00EBBAFB0F7
:10CE120061603B930201B05EE0930F03015184888D
:10CE220008080176008435928C031201595A86084B
:10CE32001301215E8E0913015184338E1301A99EC1
:10CE42008F141301715E8E0114015184AB97050991
:10CE52001601910E008883900505023007455A9409
:10CE6200130200418A940103012E8603355A810C74
:10CE7200034E68A8E828E08F141398F0E0840C03AE
:10CE8200410C511E900C03318A87120C0308CD5EAF
:10CE9200CE0C03C15294130C034E2868A82B980C95
:10CEA200034EE8090299100F039586922D04B005EE
:10CEB20066870504715E84011207995E84011289F6
:10CEC2005E8C0504A18A0000BD8A8513047D568408
:10CED2000E05870E0548015A9E1205140E05B5501F
:10CEE200B8E81102981E05B0296A96040175BCE0E3
:10CEF20094030106B0B162BF0306AEAEAE2BB12DF4
:10CF0200181E0548B0296A833F030635586B9809F5
:10CF12000688015A940E098823831206B0ED66BF73
:10CF22001306155A833F13063558C30065A68F149E
:10CF3200079208B0C966930D0888CB8713098481CC
:10CF4200568C020C8E0CB0156E870F0C88CB960592
:10CF5200041341743B8E01050DF9709502902D1258
:10CF620051842574BB86060FE03009999C1508612F
:10CF7200004106982F31B02D62922D10518408087D
:10CF8200D578CB8B0301100182880325BEBEBEB0CB
:10CF92001D606666B869603102851310CC2308ED06
:10CFA20004B10E94100D0F1210810E842D12B031A7
:10CFB20066900F1413A50E0000751E982B310E0CEF
:10CFC200B0CD6E981413010C38EE238C03128CB57D
:10CFD200514E70EEE8B902930803B0FA1BBEE8B3F3
:10CFE2008910A06964EE3A460BBE3C1898F01B8E7D
:10CFF2000412F552840E12BD2A8E14120D9E9E1238
:10D002009552890313015A8613295AAB4E2172ADE8
:10D012004E88DB8705124E655A930F0351846B8E3F
:10D0220001145184438E091351848808E17A851AC8
:10D032000913555E94121113B0F96294131300810F
:10D042008A8E0F4552AA14134950356043AB14130C
:10D0520049501D60B92EAD141398A0BE589BAF1451
:10D0620013495061607B981E3031E16E850E0F14BA
:10D07200795A97050916BD0EBF304D18455ABF198A
:10D082004D18A55ABF303C18E956BF303D3C182513
:10D092005ABF193D3C18055A993E3C18F8AEB8E8FB
:10D0A200AEA8B902BF193C18BD56BF303D18195A77
:10D0B200BF193D18515ABF303E18C556BF193E1808
:10D0C200E156001D92910518830504482394030F2D
:10D0D200B0E57E8E070913D13E8E0F0188ED0471F3
:10D0E2001E86060F0184BB00009D7CAB0000201C45
:10D0F200E2E2E283B87CD84C1F481344D83C98A89B
:10D102004451064DBCE27F410C8C3B8498A8448577
:10D1120006880CCB53410C04840C1F08830498A886
:10D1220009B8634EE6BCAEB90C004A545C6FD6CA6D
:10D13200767D4D453C8C92989EA4AAB2BBC2C8CCC7
:10D142003AD1E0E7EDF3F901097C0E2B14242D32DC
:10D15200353E4763545A6B717C82881A91993245E5
:10D1620093779E28A4A620ACB94F30C8A3DCE76110
:10D17200EC4209FC600EC01F2E52575CB265696D0D
:10D182007177883792989EB0B9A8C1DA1582D0D645
:10D192000EDCE8EF1A14E208F6204CFC286B2A0099
:10D1A200C88C2409E71892C29EA3E7274DE0489E47
:10D1B200ECB83C5808987CA8E04E70F8E085B5E0E1
:10D1C200FFA0B0BE001D6070E0FA174EA05CF6A092
:10D1D2006636761B26E0F61B4E2B4A6A56D4D4E0FE
:10D1E2004A545C6F0820F66D7132454F61ECDCC029
:10D1F200A66B982A3A47ACCA63887C82987DAA2B90
:10D20200D67654DC1A20E80E777C0E0E99935730AE
:10D21200F3FC42F96052280114E237EFB9B2B2E0EE
:10D22200141F1A3E155CBBD192FCED453CC8094D5A
:10D232002EDAB0B9A8C19E2DD677A48C716535D0EF
:10D24200E7FDBCEEC10295BE69CC886B825A23F021
:10D252009D585C0EAEF0AE6E70D494CBE0A55043F8
:10D2620032EC4E70783C0602E01CEA603CEB4CA4C7
:10D2720091EE6E98AE6150AEA0FEA03E337EE0000D
:10D282002800D58818B550B902B550B5504E70383F
:10D29200AE7828B868F8A8AEE8E0A04E6E60EEE07E
:10D2A20047710E834140424348700E0078464567FD
:10D2B2006075E00017141110534C0F00A8869C7281
:10D2C2005259911C1815121A515CCF96A94E9D768F
:10D2D200565A901B19161305575DD085AC4F9E9870
:10D2E200505B08000C0C0C00555E07770C0C0C0010
:10D2F20041460E4E5155593A617E0E5E2D2B2A2F14
:10D3020042474B0052565A2062257F003734313053
:10D3120043484C4F53573D2C631D9A0D3835322EDE
:10D3220044494D5054583F05643C9B243936337E62
:10D33200454A08000C0C0C00653E07870C0C0C8853
:10D34200EE61501BDA26F6EF1D64989417D44AFA60
:10D35200EE58AE0EF09C4A5CEA271C505C0E0A4A5C
:10D36200EEEEEE5C262666421FFA06E247FC4626F1
:10D37200E21FFC468C13BE70981D60580E38A6063C
:10D38200DA661FFAE7461AB160F08898AE8C5385C8
:10D3920050A0B0EED33E1BBB85508C97A0B03E7B15
:10D3A200CB8550EEAB630EB07BF8615070B0EE539C
:10D3B200630EB0CBB8AEF86EB7CC6F4E70B8D84C27
:10D3C2003FD88C27AD7062C102B8AEF86E6760CCF0
:10D3D2004341A4E5A8BD8C834E70B8D84CA7D88C25
:10D3E2003FAD70641BCEB0EE8F2BEE702BCEAE0035
:10D3F200B0A8AE58711C98AEE0B0A558B0AE4E7051
:10D4020078BC46063C68E078BCAE3005600619720E
:10D41200EE38A02E6EFE433E2F385E3E537EF61B44
:10D4220056765CE2174E60EE0EF0386E334C810B8E
:10D43200C90ACEF0AEE0CE7EFEBBA118CC60B858D1
:10D442004C608CA00841B0B83C58084898FCA8E051
:10D4520046705CA0D4D4542FCE58E09CD251B5A3D0
:10D46200983C98FC58B83CD88C132E0C1B2E2EBC22
:10D47200F375583005755830087558300758B8BCE0
:10D48200D80CA0C4D8584E30FFD8BC0E7CA0BE60C9
:10D49200F1585B657387A1C90B3F8F15B01A30A68F
:10D4A2007E677E777E8F1ED8BEFBA6DBE0D8A6F312
:10D4B200E0D800A6EBE0D80000A6E3E0A95C98BCA7
:10D4C2006D1EA95C88CBA95C08ABB83C588404E00B
:10D4D200044E70783C5A70AE38EEAE0EF0386E6084
:10D4E200EE0C134EF06EAE7BD55C542B1C52F0E06A
:10D4F2004EF0D460AE7038DCDCDCDC93D55C544B8F
:10D502003CDC5010F070F03BD4C7AE7038DCAADCC3
:10D51200DC7C94E36B300870AEE0DCA05C38521C1B
:10D52200AEEE6FAE0E7038D494BB5CF260DCE09C61
:10D53200D4D4F2EBE048A670851458C15C4E708ECC
:10D54200783CC6B0C67F08CEAE584E3CE6BCEE78FC
:10D552005A7AAEC39806374C098348E07806BCEE87
:10D562005A3AAE5878E62BBC1AEEF0EEAE0C330601
:10D5720033AE2E6366E3AE70FABC1A3CE638EE3C7C
:10D5820070662FEEF098EE41A4CC17266E78063C1A
:10D59200063C063C686E4435BEB8584898A8E00080
:10D5A2004E1B4EBE5C501B2E7AD898463E5ED81C4F
:10D5B200D4763654E3EEEE6BD86EEE4B2687D86EF9
:10D5C20026DFAED80E23D8AE2BD8AED86E9E5E5BC9
:10D5D2008E1E263BD8FCD86EA66E264B66CEBE1E8D
:10D5E200D4D4C34EAE98EE2E76767600CB2E7AD871
:10D5F20098463E5ED8065E139E0ED8DCDC8E132E55
:10D6020062F354CB98AED898FE1B66CEAE5C4ABF8E
:10D61200EEAE5C0EE66B3A5BC62622DE6EFA604E1A
:10D622001EE0C6C36E63424F66EAE32EFAAE4ED8E0
:10D632004E5C50EEAED8AE332E7AD898463EFA23E0
:10D64200D8465E139ED85EAE6E2E2BD8EE66D85CA0
:10D652004E13228EF32EEED4D4D3AE98C1622EFA9C
:10D66200AE5E1BB5A23ECE6EEEEE0EEE5A0EEEE6AC
:10D6720013BA4E9C4217AE8E4E6EDC50CE5322CE63
:10D68200F34EEE94C963D4CABBA63BC3FEB7F6A75A
:10D692000E8E1CEE8A5C4A9766061B36E04E22CE40
:10D6A2003EEEC21BAA260EC223EE2EFBDE338A6E8C
:10D6B200262EFB6A626B7E5BEE865A5E2A4EBAE0CB
:10D6C2004E709ECE68B8A606A8E07E78EE68B8A630
:10D6D2007EBB4E7078FED8B8DED8E01D648CB56291
:10D6E20098941FD44AC9622EFAAEDCCED86ECEF61A
:10D6F2006026E63B66EE1ED44ECF66E076FA3B36F7
:10D702007E13484623B6AE932EF0BEF01E06FA8E66
:10D71200FB2EEE66DB8EB0B5604CA0FAA00EF81DB3
:10D72200620E6964EEB03D60556469620E556435FF
:10D7320060696475624E5C2650E04ED88564EECE18
:10D74200E05C4ED01050D050105090D0D050D050FD
:10D752005CE0FAA00E8E2626065C4647D4941BCEC9
:10D76200E066D34EDA8C93DCD4239D642BDC9D647B
:10D77200D4D49D640ECE95620E9564DCD417DC95EC
:10D7820064EE4EEE93CA0A0ACAEAEA4A8C330E06DD
:10D792000E46E04ACAEAEFE0BE6E8ED8988E4E2759
:10D7A200980EE026CB5C626EA5622EFAAE045E1382
:10D7B200081E1A6ECEE673CE5E7FDCD494856B268D
:10D7C200DBF568A3B9685C336E66AE333A8EF32E2E
:10D7D200EE66539CE22B62E24F225C23AEFAAEE28B
:10D7E2006B4E5C6A0E1C500C13A66E0E4C1B09602D
:10D7F2008C1BBE1E1162228EF32E543FEE66D4EEB7
:10D802000BEE4C2B2968AE6EDC909CFA9BDCE2336B
:10D81200628ED89883268E7E9BCECECE626E0E0C02
:10D82200396153AE7EF32E7E982BD8988EEEEEEEB3
:10D832000E6ECEEE2798AEE066CB8ED82695626E3F
:10D842005A5E0E0C1BE1644C1F0160416AEE5C9053
:10D85200D010905010501050905050100B4E5497C2
:10D862007A103AD4E7543F148F94CF54FF9CD05C83
:10D872006B9050D05010D050101050905CEEE000E1
:10D88200D0501050D050101010D0D09C8B1CD0D043
:10D89200101050D0509010DC2B5CD0D0D01010D093
:10D8A200505CDB5CD0D0D0D0501C9B1CD0D0D09C24
:10D8B2006B2EFAAE8964B861500EF85EBB06BAF6FA
:10D8C200330D62E6EB66EE5ADFE64FBE1EFEFE1E2B
:10D8D200FE1388B85E2EFAAE08DA77D164FA1B9886
:10D8E200FE072E11622EFAAE3E5EBFDAABA606E648
:10D8F20083461BA6080E5E5A5C8A62228ED8988BDB
:10D902005CCE62AE4E4D6E422766EEE3D8A5608BCA
:10D912000160B32EFA0EAE0E26E6B35E57AEE56494
:10D922005C4EA60E6E3B08CB54F7D43E26DB738EBC
:10D932007EF3982EBE333E6EEED4940BAE8EEAEAA0
:10D94200EAAE9CD086C6E35C8EEEF568A56CFAE37F
:10D95200D4BB2E9C822E8EB5680C376E8E6E2E6EC8
:10D962001CA56CFA3B8EDBEEDB8E235EEF665E0C53
:10D972001BBE00B5600CCBD164496098FE356AA627
:10D98200EEDB8E29686E5C1B2E62F34226DCE08C95
:10D99200A04ED8B968EE75620EB968B03D60EB0072
:10D9A200000000B0094648167616810B70C15A0174
:10D9B2000C100801200401140104011401200512B5
:10D9C200120F120D050D0F1219200C0F13140E0F4A
:10D9D2000E0518091314050E140E150C0C1012095D
:10D9E200160114050F1514200F062012010E07054B
:10D9F2001001030B090E0714121920010701090E69
:10DA02001905130E0F12010D120F0D08B060303AF6
:10DA120070BC5C50100EC1B0AE307A0656A856D318
:10DA220049240CA08DBCF10E2170B8F0B00E4C232D
:10DA3200BD701BB57069708D70B00E356069704C29
:10DA420023B9701BB17081704670F84C1F48EB0E01
:10DA5200B835606970AD7081700E626970A9708DA1
:10DA620070F04E70F8280D729D585CEE615060EEB9
:10DA72006670EE38D494B34E70138CA0BEBEBEE076
:10DA820025601B1D60A550F05CE0D4D4D4D4D460D2
:10DA92004E7078BC26DCD4EB667038A05CE0217056
:10DAA200B5701D74F0BD700EA970EE4E70EE61621D
:10DAB200842170B1700EA970356081648C27B570B5
:10DAC2001BBD700E3560BEBEC9643160A97069604D
:10DAD2008164A9702EFA0E0960C9644D60FE890343
:10DAE20005608C60F088B9706BB0FA33FE238888C9
:10DAF2005EF00E35608964B80E3560D16431600520
:10DB020060F00EB8AE6160FADF0ECB8C1F88E08445
:10DB1200E0AE88FE13485EF0B0FAA00EEBAD74E3FF
:10DB22002E0E7AFE4B480C338C238488445CA60666
:10DB3200E6B177468FCECE235C62EE570C07856442
:10DB42000EA6AE3D7A0C0D633960AD746ECE5C5A92
:10DB52005E26E6433ED454D3EE3D7AD84E3ECE6B9B
:10DB6200AED8221ED8AEAEBEEB1E2EAE8ECE93D84F
:10DB72003ED86EEED454B3EEBD606ED8469CEEE154
:10DB820078EE132E62F38E42FA1BDC9B0CE389645F
:10DB92000160A9640960D16449601E0560B05ED865
:10DBA20098464D60A606E6A176B176DC6654EB5E39
:10DBB200B5608C3BBEBE696431608C2B6964316098
:10DBC2004C87696466660075608C3F4E5C66503DAA
:10DBD200604C13BE0C60F0E04E6E5E546F94EFD456
:10DBE20027544F14679CD09CE0DC9090109050908A
:10DBF20010505050905CE09094F3631C5D789C5000
:10DC02005C109CE05C5D789C50DCE05C5D785CE0E4
:10DC12001C5D781CE00808AE0E2EBAFE43880C1B71
:10DC22008C13485EEE4C457B8C2BAE0ECECE4E5CFA
:10DC32001050EE66F62F661B268EEED898EEEEEEAC
:10DC4200CEEEF69F8EFB2EEE66DB4EEE98EE4C1B72
:10DC52008ECEEE8E5B2EEE98EE4C0BE6F7EEEB8C54
:10DC620047884C1F48734463840CC38C1B842B88E5
:10DC72001B8564436E8E00AD743B26F6278EB32E51
:10DC82006600B5604C5F98EE660069606964496041
:10DC9200D8AE0E263B6EEE3BD454B726E36E4EEE64
:10DCA200E178EE133E8EF32ED4CEEE549BD88E8EB8
:10DCB2004E5C50D89C90905B8A8ABEEB1ED8AE4ECA
:10DCC2002ED88E1E62ABAEFAAEFA0B7E661E8E9B0D
:10DCD200980C4F8C3B396023B0D898464D60F0D1F8
:10DCE2006449608C13F08C13BEF00B5ED8AE98AE14
:10DCF2000C1F8C1F866EDAC3D8A5600C7B8964D199
:10DD0200644960016005600C8739604CA0BEE04E3A
:10DD12005C6A560E8E0CA02300ED64FA0D63B04CC3
:10DD22009F0E1E4E5C66D01D604E5010D0D0D0109B
:10DD3200501090109C506960F60D62E01CA09C6E21
:10DD4200138E26F34EAEEEEEEEEEFCA0A2E0CED4A3
:10DD520054AB139C42E60D63B0221FDAEBAEA24E27
:10DD62002E5C105CEE22270D622EA2F3A637EEEE99
:10DD7200EEFA9BAEB04A1C5090B562B0064E3055DA
:10DD82007C067C30E04924B83CD88C1F881384D8A8
:10DD92007CA8E0302D9C58A051B698DCD0CB06C0B0
:10DDA20010000000008000000000000480800420B9
:10DDB2000020030001080CC41431000D320003CC12
:10DDC2002B28900210003314900130021028400CCE
:10DDD2004070A20150399803329000048000000084
:10DDE200C0000580000000005002420AC035003029
:10DDF200300000DC000C8A04000068CC390000000E
:10DE02001AA031C1030230B9C040000C00008C00DE
:10DE12001303C680088000B32100000850C80032F6
:10DE22000800088000080800040001D9200C80C8FE
:10DE3200A024933920000000C38D06083068000337
:10DE42003000F30125000840009013900343A64DD3
:10DE52008E0C307003190000000003000000000067
:10DE62003000030000003000C3D0000004C00042B4
:10DE720000380C20153700F7CA89886FC8CB02F327
:10DE820033840090D00300000240D9555555550502
:10DE920095657116695AAAA9EAAA2AAAABEFAE0336
:10DEA20054285A3FEFFCE3C38B000BEE2A1E80FC82
:10DEB20000AF02542196A9C091EB95E5286ABB05F3
:10DEC200550AC467A25A0A99872352F51188FE4F50
:10DED2008D13EF6E4D0CBA3833CCCC2000002CDA07
:10DEE200555555551500155515005555154055559F
:10DEF200151555151000100000000000000010005C
:10DF020000401040101560D50CEBD10C448A12125F
:10DF1200FFDA8C88221341418B63680C8859206296
:10DF2200800C302003C0083E2CC100AFC4C0F8BC36
:10DF320007B3CE204F11138087FC110AA08A8028D4
:10DF4200B820C938808C02FEECC17FFB38FF40C28A
:10DF5200BBCFE3684E4C4CBCFF4E5CA80300953926
:10DF62002292DDDB4B2FF470010F3FFFE12040F2E4
:10DF720004C631E2C8C8FF310AC88CCCDF87200151
:10DF820009C9BFF3EF0B1220131124C40889E01B47
:10DF9200484322C4008F24003E46402C26233C3FA7
:10DFA200800314D0E76361134F1344343619314DA3
:10DFB2003B442A400129924FFE51D23C702128381D
:10DFC200CCFC3E400C04506029064CDB60F74E014D
:10DFD2000C002554D8F36063F7F187AAC1FF8DE3E3
:10DFE200224BDC7136EE03C5084A8E288C927410DF
:10DFF200CD0420812BCEEF8983040040B74FB007B8
:10E002002010224988B04ED24F861258EFA11D0F20
:10E012003BC0323C3F11CCF21C6F974072FB423D39
:10E02200B51F02300004E3844B12F4760BA2788C05
:10E03200B30948006262173B0202862D52B8FF11F3
:10E04200E25E5D50B2C46D0A100C40304086683109
:10E052002658594D24145233002941071824072009
:10E062002900A48002C0C4808CFB0B9522000B788F
:10E072008E00AC928400A75423CFF8092044F630D6
:10E0820043C0B5EE5E298FF0735A2323CEB400113C
:10E092008C3CCC0B480C4442BC90393E9320082166
:10E0A20000203D460000040040000010000004046F
:10E0B2000001000001400000410441B915376CFC29
:10E0C200D1170304C3CC500C0C330860C4CCD0CCA1
:10E0D200800411230A3FC6C80080FFBF78EE8A3F42
:10E0E200034C0322CC3401304C2100233010802811
:10E0F200C33062E2500005C01088C0FCA30438C5DA
:10E102008424B34DCDE02B2F043C123028DE40385E
:10E11200647D1374C6374208403EF6030000C140D6
:10E122002194C83E312220022085006B84CEC8048F
:10E13200599D5316097D7F71D8C532E1463B80381F
:10E14200133040C785224E5523DD0E054F4490CC37
:10E152001CDDBFB88B44A074125022129130970379
:10E1620000767FF74C17DF8445CE98F2D949140226
:10E17200C42012513222C900048C4A3B4BFC80035A
:10E18200050B0051482B0E31EC502DF0DF38C8132F
:10E19200ECCCD8513D300451FBC73EF37F0CD00C80
:10E1A2000106B5064E70F858985684D84C5B8C4BD5
:10E1B2004C3B1C427070384BAE783C0670B958CE5E
:10E1C2008CA08D08849B76761908AE58FC58F3997A
:10E1D2009E990AB5960D9E1596BD966262C6CA5064
:10E1E2001C231908AE58FC58E21BE2371100EE5C02
:10E1F200981C45028CA08411008D08580CA0B5A271
:10E202007B9BCBC313E3DB4B43CB3B434B535BBD0A
:10E21200B25100E30E1C5016B523110CAE0E93C47E
:10E222008370FA70A033F0B80E6150F86550C4F0F4
:10E232007C30147C3050BCE0C8CCF73008C8CC66C7
:10E24200EBE0D5884FA550F0D44FA550D43FA8F0AD
:10E25200EECBA550AEB87C58AE8CA74C3344983C5C
:10E26200A883B5BC84634C6100431300A550EED46F
:10E27200D3B87C588C33A3B070E0A550EED433B839
:10E282007C588CC378A84E703868F828EEE8B5BC84
:10E292008860A04E70B85860434C3748ED04711C3A
:10E2A200EC1F0C1B919CCC9BCCA3203C5606301837
:10E2B2006621463087662F110C1D02C8CC5C5AD0ED
:10E2C2007038CC9704624728707C3014FCE090666A
:10E2D200281C70381B2E28BC30EB33B898A8E000FD
:10E2E200A383634323387C8338FC6B383C53387CEC
:10E2F2003B387C2338083C8C1BADBC300670FCE0FC
:10E3020048711C8C7F0C238914538C2B0441B0233D
:10E31200F8992C4C3F305166FB610044ED040CC768
:10E322000100D50CCC0F3008999C0CCFB83C580C8E
:10E33200D91C6000711CEB5924305006CC4F300CB4
:10E34200B19CA6CB091E201CE2153221460100E039
:10E35200D50CCC3F300A999C0CBBB8F10C7CD8048C
:10E36200884484D83C467CA8C46100CC4B30C306A8
:10E37200203C1C6ADB78EE30BF0E66267BA6067058
:10E3820038EE4B3EB75EF0FC56468B300770999CD8
:10E3920051844E7020B8BC588CC50284983CA8E0C9
:10E3A2006D5820091EC8CC6046F070306906787C32
:10E3B200660FBC6670380EBAF038BA6EB7F04670A7
:10E3C200B858CCA03846BC30E660C4783C1C420A3F
:10E3D200BD8E60A0587058585870707070E0DCA004
:10E3E200C44484C44404B1702DD91C610030FF0EB2
:10E3F2004EF0E020F0AE70AEF0A6DB309C3C30A7D1
:10E402003C309B685A2E28704E9C103020E84E708B
:10E412009C90105C1010A8883006999C3069067890
:10E422007CA63C68D5060ECC1F4CA038CC432E28C7
:10E43200BC30B606E00C6B90662870387C1C0A1C57
:10E442004E70E06228E01908AE581C58F6BDBE4472
:10E45200F64348F62BF6603D02568C33841100B128
:10E462000EAE8E301EC63F4CC3301AC6A36E3008A5
:10E47200EE4E702E3C86F313EE66F3EEB8AE3D021E
:10E48200D588387E7E8953065E04467056607CA627
:10E492004708FCA627FCA64B3CED08E606E6E64646
:10E4A20046FC06E01C8ECECC474C37784C1758E021
:10E4B200CC8338BC3AEEE2DFCE308E1A3C7E1E4E62
:10E4C2001CAE3A30AEAA3CBECB133CEAF358AE6E59
:10E4D2001C53CE3A303C46FC6E1A3A3CEA38CA2803
:10E4E200E044E23349A459A41B49A4E5A43C1E4ECE
:10E4F200BE4F58E5A4D898D83CBB2550581CDD8C9B
:10E502006EB858E065BC8C1BCCA0044841B0336D9A
:10E51200BCCE992CF90C8C2F3C580C6765204670A8
:10E52200B85888D3C4B83C5804987C58042B492462
:10E53200B8587CD804D8FCD88404D87C8498A8E045
:10E5420085BC390C048CBBB85804ED04C4E0B01A85
:10E5520030E61B1C50BCAEC1B0AE4D14DDAC49243C
:10E5620065205DBC651C4C752EB85888987C58088F
:10E57200983CA81D02B85884987C5804A341B0F96D
:10E582000C3330A7C8CCF91E66DB2DAA8D08F681A4
:10E592000B1C98B10A30FD70F0B8150A46A809BAEA
:10E5A2008BA3ABDBB3ABA39B93FBA3F3032B23C9DB
:10E5B2001230CFA663B51230903B1D140912309170
:10E5C2000286061D146684E37330D04330CE0663A0
:10E5D20065169C021D1411B41DB4D884D81B30A832
:10E5E2000629BF30AE06AF19B4D8D91C8C2330E04F
:10E5F2001B30D02D149388309C0613841D1411B443
:10E6020006D91CA6D88C7384D884E6BD1C090E04D6
:10E61200DD14661BD806163066066B1E7E8C177ECE
:10E62200A1140CDDAC5D1E307006C7668B307466BB
:10E63200D3069B3071463C301A7E3766EB305C461F
:10E64200E80B3065DB307A4636BB30689B301D06FE
:10E65200CB3B301A06CF6667B8D8485CA2E217886F
:10E66200D8E88B266637DD1430053B302D23A61CF7
:10E67200D0E51411B46E5606D91C301D1C621F065B
:10E68200970C2B301FE5140912E6161D1411B46EF7
:10E69200060404CC13081C02A65A56BC1AD91CB88C
:10E6A2003007E8BAEF6E49241C0C2DB50CE5A46EB8
:10E6B20006D91CA675B0E9145B6E3DA41DB48E0686
:10E6C200D91C1C627330CF2D1449246E3DA46EAE4A
:10E6D200C512AA625830C02D14CCEF8CDBE0B8B85A
:10E6E2003044E86914061ED91CA1143020E8F89CB5
:10E6F200E213A83060A820045330C848C8CCA066F2
:10E70200E34404048449242DA806864C2BAD7043AF
:10E7120093C1B01EA114C66FCC4F6914061ED91C3A
:10E72200A11409123020E84924B80E41A41DB41CDA
:10E73200EAE38E56063C3040FCE0BD1C2012050781
:10E74200204924785A0E43660E7038EE477A30C05C
:10E75200661BAEA3AE3CE03020E80C57302006F832
:10E76200A85666A00879B2D91CA6063C30147C30A3
:10E772001C50BC087A3056D84C1B36448C1B04847F
:10E78200D8E80C8F3020E8E09E4EA0A60E3C26660C
:10E79200EEEEEEEEE6A63C266606BEEEEEEEEE06E9
:10E7A200AEFC2E6E0E60DE77DC101E7CFE7FFCBEA1
:10E7B200FE5FFCBE437E9EBE1F3CEB7E3C1A9EFC6F
:10E7C2009CBE603003FCE8D34670CEED28041413DF
:10E7D20008AE58FECD7DE05CE0D460D0DC6202D7AA
:10E7E200629362E97CE0C2E223302C1B302ED4A07B
:10E7F200D57C33E97CE0D414030CA01C98E217D436
:10E80200A03045D57C98F6CD7D7B1C38BC44137A6C
:10E812003076EF76DF7617483C0AE0CC1BAA7339D4
:10E8220088E60952D5883ED74DA6251CD91C302032
:10E83200E81538004C73B0E22F302DE813B8957C00
:10E84200D91C7B30C30E203C0A2365202B4E203C72
:10E85200D026E806303404661708B0C606C61CD0B7
:10E862000C1BE21722E866F13A0E30410660304B8B
:10E8720006F3302506FCE61C0A301E6A23666A3758
:10E88200FC0E66813A30CD6A2F3C3E3EA366E030F4
:10E89200610660306606A0301ADBB03C0E660401E9
:10E8A200AC0C0F1CE22F0E16913E70012053AED815
:10E8B2000C27B0B13E088BC1B0B1BC492444B0A111
:10E8C2001CF93E589DBC981C1D88FC1EBEBEDDA4D2
:10E8D2004E70E5A4D8B0D83CBEC32550704670B087
:10E8E20068301E7CA11C0441EEB83CD844D8FCA878
:10E8F200D91C78D884D8F04926410CA83080A6E6E5
:10E902004EF070B858CC1F0C1B66664C17168C1351
:10E912006E3C588C233080464C2F8C23767676BC06
:10E92200588C2B76767676BC56EE3C56EEEE4E3012
:10E93200107030FDF0AEF046F070B858E07CD80CA4
:10E94200DD2F580C2B30844D320CDF890C4C3304F4
:10E95200B170434BF8E61F26E865144C19387DBCAC
:10E96200651CC8F84666E8B858F6F62B9DBC410C03
:10E9720004B898A859248C47C1B0302EA84924C1A4
:10E98200024E28E8A89868E0FC5C0AB8AAA8E0B0A1
:10E9920030E83AF6E3E030107030FDF0E0000000BD
:10E9A2005AEEEEFCC6E6E6C63C06BC5CEA5A505C91
:10E9B20030662B22E399C63AC60E3006C3A6E67A23
:10E9C2005ABC1A30F6F63C58FC0E3C3A301C0A3C53
:10E9D2005AB03AE07AF30438BC585C98FE9526FCAB
:10E9E20010D0900EEE7E93EE0C31237EDBEE7EA3F2
:10E9F200FE13081C78221BDCEB1465238C27787E1F
:10EA02006881228CAF88DB780EDC901E6F080CC701
:10EA12004E6E56DC5050087B0C5F0C1F0CE30C1F33
:10EA220008330423780E561C561750DB7E63EE7EA5
:10EA32004B9C78221BDCEB9443E030D066FB20E059
:10EA4200D400980278A26838BC983C28E01CAE58E2
:10EA52000813044E6E56DC90688DB8B8580C2BC95A
:10EA62008C89B68CB551884EE80CDDB641A48A4932
:10EA720024DD20792419B46A1C0A301D623F0A2B56
:10EA8200AE9C58636E1DA4DD8CC1026E601CCB3837
:10EA9200BC58780ED91CE9501C622B62BEDCDBA28A
:10EAA2000C471437D4A250DCDC8C5BBE1FDCEB8C31
:10EAB2001BD013D0DC4C9BD47F1EBE2F5467DCDBF3
:10EAC2008C1BD013D0DC9BBE131EBE5EDC0C13501D
:10EAD200BEE0DCA0760C831C6247A29C622FA222BD
:10EAE200230AA2501CE0169CE0D2D268AED2D228F1
:10EAF2004EA846F070E0D91C78D808D8F0AB781C44
:10EB0200221BDCEB6206569C622BC6DC14DBA05691
:10EB120013860EDC50BEDE774277FABEE3A6426F62
:10EB22007E07A6FAD31EBBBE2766EBE31E0C13BEFE
:10EB3200AE0C83A550E854670CAD2355BC410C1DA7
:10EB4200024EE860E078E05CA01E0C1B9C131C22C5
:10EB52002B62BEDCDB0C83144742F21F0404D00B91
:10EB62007676130456DBD45F8C2F543F3E63BE533C
:10EB72008483B8580C2B410CFD8A4EE8203077E094
:10EB8200689D2244781CEA31B60EB8AAAE3C68F8F9
:10EB9200AAAE3CA838AAAE3CE8387C4AFC2878FEEB
:10EBA2003B09B8B8D84C578C47D8DE3EFE31B8F393
:10EBB2004484D8063020665746F07038566637D9F6
:10EBC2001CA6E853D91C230841B0CE6DB81902B86F
:10EBD2003C5806F804A0965C1427D4B6E30EF62B34
:10EBE2008C63DC541F66E333D4144FA6E32E8A3AB7
:10EBF2005B0E0A061C2A4F0E7E8E9C0ABA60E0AE9D
:10EC020056E346A38C431B66239A3A370C1F4E7376
:10EC120084762B0C4B069CA206BF1BEE608DB8CEF1
:10EC220008D528EEE9502E0EA0B8BCEE7EE6C6FE50
:10EC32001BDC508C752A5CF65B752C552CD4DABE25
:10EC420026E37B661FD4EB46BE3F752C552CD414AD
:10EC520047BEE3D4141FA2E39CE04C437E9EBE4712
:10EC6200DCD4E3DCA07E83A28C1BD013D0DCA26BAD
:10EC7200552C4C752DF3BEB6AE60EE5D1E5C4C930A
:10EC8200063003562FC6FB462746FBC68606A63726
:10EC9200D4BEE31ED3752CD4143FBEE3A2D414EB2E
:10ECA200D61B1C501CA63033A6E00D2AC6A6C6A64B
:10ECB200F306F6C70BE0DC201FD4EBA0E0A28C1B0E
:10ECC200D013D0DCA2E0A01E7E7E43ED28D91CEE3C
:10ECD2002526DC10FEE0DCD0D07C70D91CB07C7024
:10ECE200061C4AD36A2775B0AB3020DE7E2320494A
:10ECF20026E8D309CA008CB3F12E461AAEBCFA1A22
:10ED02003A30E63A303CC61C3CA2BC02F6F6DE6B58
:10ED1200F6277CD90E7CAE0819BCF90EF6CF75CA5F
:10ED2200AE5851000E389C0A983CBEAE2838FC26DC
:10ED320084E6C67C287E7E677E01CBCDC63000EE9F
:10ED4200CC4371CC66250E22C8EE66A30B000000F0
:10ED520000000000E55CBB6100A3E55C8838FC664E
:10ED6200E6876B1CC4E666664B095010841CEE01F4
:10ED72003041A478901C8C476A550E4DA43DA49D49
:10ED8200A48C1F7CAAB18CC1B0041D1425FEA55011
:10ED9200EED44B4670B87C588CED02B070EEF0E0C9
:10EDA2004EE8286AB3B83C58A020BC30C1FC1CE035
:10EDB20000105B504B903BF3D023BD8E103C064CB1
:10EDC20023308006708C83AE1CE2EEEEEEFC5C50CB
:10EDD200303CE6E60E9CF83C5842A65844D91C301A
:10EDE2002006861CB86AF3AA6A37C6E8A8B8D3F820
:10EDF2007E60BEB03AE006B8588C233055737C581A
:10EE02004C3305BCEEE91BB8580CDFB05A3C063057
:10EE1200667E679CD0FE431CD03EFE53FE470658DA
:10EE22000ECD90EE87B00EB85830505E7C067C3026
:10EE320076B1B5BCEEB85CCA46A80C2BE21B1C220C
:10EE42009C5858CEBC30147C301C50BC5870305981
:10EE5200E2B858E0D8A686251CC1B030E02D1404D3
:10EE62001D1030E09C58BC0E66483D3A44251C1DDE
:10EE72003C984D14987A30F6453AF6F6167A3016E2
:10EE82003C5804D89CA298A2580C9321382B4C5180
:10EE9200370C33BD386520A30CB5374CC9370CB7D6
:10EEA2008CCD378C8F5E7B3091AEFC9C425D1CAE6C
:10EEB2004D32C1B0711C9DBC110C1D028C1B0CB3D8
:10EEC2001538838C6B4CF53B0CF53B4CC9376520F0
:10EED200838C653BD32D38DB4C41370C3381346551
:10EEE20020A3203C0A30836A7F3031E82D383B0C66
:10EEF20081356520C3B8FB0C3B8C678C1B4924060B
:10EF0200A6A6B8A6A803B8F8E806A6F13B4924B815
:10EF12003C0E8CA730CD8C2FD91CD532AAAEBCA802
:10EF22009858889858653A4C5330AEAAAEBCA80C93
:10EF3200571B301E0C0B668CF39C98D844D8581C77
:10EF42003001AAAEBCA8C1B030D02D14A83060E800
:10EF5200D53649249C98D848D858D91CBD1C090ECE
:10EF6200042021386B4C778C5F0C1BBD3865209BCD
:10EF72003030E81B30305E172EE83CBEFCE8953A94
:10EF8200BEFCD056E82138430C1BBD386520BBB807
:10EF9200E04936BD1C1314201538BB3020A8A8A8A0
:10EFA2006D7CDC100E304C66CF21B0DDAC49249C68
:10EFB2009858B81CD04C1B1CD0AE7CA2813A65205C
:10EFC2009B3057BE5E2B2666DF03305466E3834ECA
:10EFD200BEFC1CD0E81538630C276520CB4EBEFC66
:10EFE200D0E81BB8E0301F43301F23301FE8E8E8A9
:10EFF200DDAC4924F81C98E8B83C58880898FC6DA8
:10F002001C61001106DCD01C0EB87E584CE706F8D5
:10F01200425646BE47A6E606E6E646A39C98584CEC
:10F022002330804686DDAC4924B80E8CA76686E67E
:10F0320083DDAC4924B80E30C8E0C8CC3B66E3207F
:10F042001938436D00C1B020492495BC110C9C981D
:10F05200D84C3B4C1FAEBCD1A6D84E5CD070AEBCD7
:10F06200FE6D076645023040E6C8CC6D0266DB04E1
:10F07200B1703C30E866FB59364924A5BCB8D88843
:10F08200D8A84E68D91C1538734CD13E957CB35D17
:10F092001C8498A84936492478EEAB7C4A68251C22
:10F0A200D91CB81B0CCB6520E36D7C06251CB6BBB6
:10F0B2001C307F6A93303A6A73302E6A53302C6A5E
:10F0C2003378EA1FAA0A3C68EED91C21B0B30000CB
:10F0D2000000000049248C931C78EE4B255068B840
:10F0E2005884986D1CB83C06300F6A291A86D91CC0
:10F0F200DDAC492478E0DCA01CF2251866301E1C29
:10F102006ACF78581598EE8FB858F83C9C580C5F27
:10F11200B80E95BC110C810A4C37587C7048840C8F
:10F122002B88B0A11C44B8D80C23584898589C5836
:10F132004C4B1D3C4924980E1DBCB80E86813A8C5E
:10F14200537C560EB858AE444D32587CA11CB85868
:10F152001C98BC580C5B30E61BD03B3A30E617E0FB
:10F162009010589C583532F8E6C1B04CA066664CF7
:10F1720013061EA1143020E8E060B0303360B030D6
:10F182003A70EEEEDADADAEEEE7CE041A4584DA403
:10F19200EDA4D8E05CF84A0EBEBE175031020E8CC8
:10F1A2002248E30130028C043EAEC242880480BE93
:10F1B200202C51C0202ECC0DA241A9AA84F902C450
:10F1C20050020D3384537FBC3F00000004DC78778B
:10F1D20077A50400DC4E0DC0AD804070097E44105E
:10F1E200226323144F8CCCC30DC912942379D33FCD
:10F1F2000030004100E45C480640200180840B306E
:10F202003417E33B03614413D323C1903331FAF43F
:10F21200E4D2CA44F24DD4908823743880DFCFB34D
:10F22200F3BC6C759792E288CFD3CE4060C1562171
:10F232001E168C74E8237655D4B87088323931D5CD
:10F24200D193F0E04D472E1FB82F2C89617420C254
:10F2520040844410A0363513834E847F64D84E55C3
:10F26200E88080D274124C1BE360A307800F28CC85
:10F272001B31841C91DC3E01FC279EC001316D8252
:10F282000FEEFF13DFCFFBFC27D90F9E1BC43013F9
:10F2920072813CF7F73CF743182F2EE388A4033C16
:10F2A200000010D544483012D070C5713003B01739
:10F2B200470C3C12C470CC030D8BCF8002470C4D1F
:10F2C200F348CCC44C7888871F871EC715335F84E8
:10F2D2008F2341C0084013CF4688CC00253840CD4B
:10F2E2007512080A0D21334073C4044383C700F822
:10F2F200B1C44CFC72FC85BFDB87C4040C232031F3
:10F3020023715CC00E193400C6848914C3703CD1C9
:10F31200F3CF90E150CE6192DFF120A955A34A15B7
:10F32200A82A166262403C8777F8480491C33833B2
:10F33200C3400431F3B0F7C9C4E4C88DBBCB347009
:10F3420038E013130741C43C7324232378D1C43D0E
:10F35200215E141F13CAC53884C4AC737C7CC8B543
:10F362001012024080D844C84417612520B33D20C2
:10F37200C623FCECD36EC8C1EC0B5420F944001533
:10F382004F1534551823FBF73284FC4C018B8773DD
:10F39200E1F81727FF0113C760D19278AF17C603B0
:10F3A20094D754508F8FF450E4E5A41F659A3D8A98
:10F3B2006BDFCB3C02CA23A3CA8DC94D88421320FE
:10F3C200668633F3ACFC18FE43A28D0B11A2CA83EE
:10F3D2004813144140001733CC0C0CB26D33847DBA
:10F3E20003C74F3CC48314F3303D14CA20CED191DD
:10F3F20010CC3F3CC03EFD2EF2C6F1EE98127337A0
:10F40200D673F4480C30CDC980CB3483D88F2072A8
:10F41200CA2033DEF32003C48A6D1458608219A80F
:10F42200C5878C047931ACCCF07340CC1EC97667A9
:10F43200F2355B43440B1D38CF7ED0C162733F0A65
:10F4420001630E80B8B3007C8E3C05B0F4D2031089
:10F45200BB0030CD0058885CC574351A37C3D2ED75
:10F46200E2D03010A2633C03F10C4D0CE1E8CF3046
:10F47200FD1107723C7012948ECB9025A18C23094A
:10F482001C480F8A036AC214130FE30300A3388BCC
:10F492002AA04C03C431CF0C0CC02C0200DE0AE2BD
:10F4A20038FC494000C0001D841057195F3DC44E0E
:10F4B200C47FC3FF5DD64BD524CE0358C8CA196298
:10F4C20081D117FB420808B2338443F5FC414CCC8E
:10F4D200125328C634B952B9CE0350C400C846F2FA
:10F4E200CE7FE00932713233F100402233870C8C37
:10F4F2002CC5C40123EF0B0725F653843401339046
:10F50200CC4C04E415AFCECC013931C710733303B0
:10F51200188101C831313E1E080700F2C38071FC18
:10F5220063C5C8C4AC85332246E31F3B380720833A
:10F53200DC0741FC13C33F6F88F8DDCC5050D57314
:10F54200444C18C04C58F8F883CC7132C3C10C0734
:10F552000692BD78413BC4BD8F1304B3F810FA186C
:10F56200F3274ED1C7C7C7C7EBA48C080081ABE312
:10F572007B48B13013223AC467233F437632168860
:10F58200C0F0303F32516308408F12F357B0804BC6
:10F59200F0CC0CD3C0C4DBD8567F5D34F2430503F4
:020000021000EC
:1000000004230054041E06E606C306A5093B0A396C
:100010000A550A710C4B0EEB0501056C06280649C2
:10002000066B081A082F082709E30B1A0BB10B53AC
:100030000DEA0E860F39013D01980057007301C487
:1000400000BB00D9009C01E1000084312005030EB3
:10005000010E0906E00A40CC00F6002A4441544152
:100060002BAE80F27F3DAD00B1849B8C908C01F271
:100070007F3F8EC004F7002A4441544131918CAC3B
:1000800037AD0AB28B2BAE80F27F3D9B72A74875CD
:100090000211920B920C75C205200510C401F500E7
:1000A0002A592F4E83838C8E8B9A72F14E9A73A8A5
:1000B0000178A9017575CA03201320C201F5002A31
:1000C00054474C3AAEF375ADF2B182114001AE80A7
:1000D000F27F3FA121AC01B1A0C404F6002A54472D
:1000E0004C31AE8AAC09B28B11714090F37175CE70
:1000F000F491F00275ABF2A8F201AD0A85AE8A75F3
:100100001171ACF140AE80AD37A9157EA8158503FD
:10011000128316831885041283151883111685051A
:100120001383151483111985061483151283121174
:100130008507158315168310C80D200D50CA00F5CC
:10014000002A42474EA80CAC377EA90C8F8FA81509
:10015000A80A207A63B198F541414141419B009A38
:1001600073F1419B73889A73F1249A7278B2880173
:10017000F424454E479A000219AE80A121AC01B388
:1001800083A8008503A900121A10101804A9F39679
:1001900073B407C40C200670C600F6002A53495AEF
:1001A00045A81990F3AA1985F95845512053495A81
:1001B000452011409C00A91D9B739C02A81D8EC860
:1001C00005200460C800F5002A4F555471AE80F236
:1001D0007F3D759B73AC37A748AD377EC603205271
:1001E00040CC00F50024454E47AE7301F552454121
:1001F00044598502F14E8503F1498504F250568534
:1002000005F3504D548506F246568507F3454E4496
:100210008508F5424547494E8509F6244552524F17
:1002200052850AF4434C523F850BF25031850CF253
:100230005032850DF95343484544554C453F850E92
:10024000F450455220850FF3494E5485CF0FF3509B
:10025000524E85CF10F342414C85CF11F47E494E6A
:100260005485CF12F47E50524E85CF13F74C535421
:1002700020504D5485CF14F744455020414D5485AE
:10028000CF15F44C49464585CF16F353414C85CFE5
:1002900017F84D4F4E532059523185CF18F3444231
:1002A0002585CF19F7582D4F5645523F85CF1AF364
:1002B00059522085CF1BF344455085CF1CF352443F
:1002C0005685CF1DF352425685CF1EF747524F55E4
:1002D00050533F85CF1FFB544F544C2047524F552E
:1002E000505385CF20F8544F544C2043465385CF6C
:1002F00021F647524F55502085CF22F343462085A3
:10030000CF23F6434620414D5485CF24F74E4F2E40
:100310002043465385CF25FA4453434E542052413F
:10032000544585CF26F95249534B205241544585B7
:10033000CF27F953414645205241544585CF28F3F4
:1003400049525285CF29F34E505685CF2AF44D4954
:10035000525285CF2BF95345544C20444154458586
:10036000CF2CF84D4154204441544585CF2DF643C0
:100370004F55504F4E85CF2EF5505249434585CFAE
:100380002FF55949454C4485CF30FA43414C4C2018
:10039000505249434585CF31F8494E434D20544191
:1003A0005885CF32F94741494E532054415885CFA3
:1003B00033F2414985CF34F453454D4985CF35F368
:1003C000414E4E85CF36F34D415485CF37F44341EE
:1003D0004C4C85CF38F44254415885CF39F44154C0
:1003E000415885CF3AF333363585CF3BF33336303A
:1003F00085CF3CF5444154453185CF3DF5444154CA
:10040000453285CF3EF44441595385CF3FFB4346A7
:10041000204348414E4745533FC251202110C4015B
:10042000F6004D4F4E4559A81B9C021114A11BF913
:1004300020202D4D4F4E45592DA11AAC01E01DFF36
:10044000A909108311AD027138713912A11F10AEC4
:1004500080A9168E85CF7D12A11F85CF7F111A101E
:10046000101583770391F29672B307850290F3AD6E
:1004700037A915A11EAD37A81585CF7B111242CF24
:100480006611AC16B1BAA10B11B21FCF7C11124389
:10049000CF6712AC16B1A9A10C12B230CF6813AC61
:1004A00016B19DA10D13B23CCF6914AC16B191A148
:1004B0000E14B248CF6A15AC16B185A10F15B2540F
:1004C000013B3C71A11D22111B12433EA9167185EF
:1004D000CF7EA815118316AC0240AE80E0178311C1
:1004E0001A10101505AE80F27F3D9BF3E00783964E
:1004F00073B50F8504AD37A9157EA815CA1F203C1A
:1005000050CA00F3002A4E2E67B496E057882D7A21
:1005100064B3A42A7A64B296CF0F18AE808ED00747
:100520000F042325402467D0100F43543185022A3D
:10053000652E6543543185032D652E654331850154
:1005400023254024435431850A2383CE0533402E8E
:10055000543E612842114024422E234240432E4201
:10056000543D8509E01D093AE0210985C40FF300D7
:100570002A49A903232428424036762441542540A1
:1005800037211178B1842463B2970126274267D0BE
:10059000780F27264364D07F0F542160531141B355
:1005A000F20227264264D08F0F216011403E26249C
:1005B0004266E06A850D2E502142582E114167B1E6
:1005C0008343B2820121023D114124422E21532650
:1005D00042403A212D412E114167B187432E4224DA
:1005E00042B2880121112141421243022A21424094
:1005F0002A714327542A4371532E4276713E714D1E
:1006000061111B1C101646BD54AC03E01185A903F3
:100610002E1141033E111B1242329C028506A80393
:100620002E603E27CE063785CC1AF4002A5056227B
:1006300067B18CE0588727254224264240B28601C4
:10064000242142254002543385CA04F5002A504D26
:10065000542267B18CE0368727254223402643B2D7
:100660008601232540214302543485CC04F4002A1A
:1006700046562267B18CE015872624422340274343
:10068000B28601242142234002543585082E65217B
:10069000425455377658542E4376284211404236FC
:1006A000C807205F20C201F4004E50561116A11B4E
:1006B000F82020202D4E50562DA11AA904A903A8D8
:1006C00002B1BDC404F5004D4952521116A11BF8E8
:1006D00020202D4D4952522DA11AA802A803A90489
:1006E000A8057735B19AC005F4004952521116A1F8
:1006F0001BF82020202D4952522DA11AA902A9032E
:1007000001113C3811161A1011163F1310AE80A1BA
:1007100021AC01A806118313119C00A91DAD064050
:100720003BA11C1071AC0683402F403FA11B131549
:100730003B11173C0BE0B389119208930BAC069365
:100740000B212846BB121613AE80A121AC01BEE1DD
:100750000FAD02B1ADAC0A8F12AD03B38FA8051374
:10076000188314E0178113198313B48503131783B7
:100770001204E0088132E0C190B58B023C753BA1C8
:100780001C8501E09E8B05AC0A8F1410AC0214117D
:10079000AC031412AE80F27F3D111B12940226AC02
:1007A00002AC03229B73AD03AD02F27F257EAC3712
:1007B000840EA916A8001314AC061313AE80F37FA1
:1007C0003D3F108EAD16BF7838AD06B18412421190
:1007D00041011116403CAD06B186114090F39305DE
:1007E0000113153BE00489BE380AAC0A8F1314AC20
:1007F000061313AE809C00A91D9B08AC37AD0AA957
:10080000157EA815A81D9C02A11CAD0685A91D9CDE
:1008100000A11C9205A81D9C0285C02CF5002A4948
:1008200052520C1032A804CC01F5002A4E5056C288
:1008300001F6002A4D495252CF107F21AD063522D4
:10084000111B124332CF112F3E77363738392265CC
:100850003C1C113DCF0FAD06B286908E543D970ED5
:1008600002112C2D426144B38876553A11413BB4B4
:10087000880376583B11403A2B04AC04B5842243DC
:10088000B682052D063B2A94099406908E838383B5
:1008900064102B5442920977764292062D54AC0490
:1008A000B88676412243B986085176401243093B07
:1008B0002A94089407748364777442920877764286
:1008C0009207292D4292087626429207970ED07BF6
:1008D0000FA904AC02B9AA27284126294143282997
:1008E0004341605411262943417153221140421162
:1008F0004122713241611243111B1C101844D0BABD
:100900001109AC03B18622114094068501AD05B1F1
:100910008E29221140429110A9052432D0E5100100
:1009200022114091722629414290105443251141D1
:10093000605342114132C825202470C600F60041A0
:100940004D4F52541112A11BA904A905123C3BF9A9
:1009500020202D414D4F52542DA11AA11CA11CA1A4
:100960001C9C00A91D11103BA11CA11CA81D9C02D0
:10097000A80912A11F9C021112AE80A121AC01A8EE
:1009800003AD01A90323613177373B3A8F06E05E5F
:1009900081AC03E00B832726AD0478B5A3B612041F
:1009A0008F1113AE809C00A91D9B079C02A81D7E81
:1009B000111428A11E111529A11E111621A11E8591
:1009C000058F8F11172AA11E11182BA11E11162198
:1009D000A11EAD05841119AE80F27F3D2829409BF0
:1009E000737E84C018F7002A414D4F525402011102
:1009F0009207AB02B78310B889072122111B12435B
:100A0000426E08920A382461714139920B10714686
:100A1000B99D9301217BB38927254685103A3BB1C7
:100A20003303A80467859209920B7731A8058509DD
:100A300018AE807EC80B204C30C001F300534C111F
:100A400014A11BF72020202D534C2DA11AA807A973
:100A500008A909B1B9C004F30044421114A11BF75D
:100A60002020202D44422DA11AA808A907A909B1C8
:100A70009DC004F500534F59441114A11BF82020C8
:100A80002D534F59442DA11AA809A907A90801A956
:100A900002A903A905A906A80412103B113CA11C38
:100AA000A11CA11C67A805A91D9C00A11C11103B3D
:100AB000A11CA11C9C02A81DAD08B18F12143BA162
:100AC0001C1215AE80A121AC01A80201A804103CA3
:100AD0000D7F11920CAC07A114AC08A115AC09A1B3
:100AE00016252C44BD16E00B822C267884AC03849A
:100AF000BD22038F1216AE809C00A91D9B0C7EA800
:100B00001D9C02121728A11EAC05B28712182923BA
:100B100041A11E02121929A11E85C218F4002A53F0
:100B20004CAA04E115862C2B78B2A0212341224344
:100B30009C026E2C1178E0098075750B389309853D
:100B4000017575241112434283838502A80329236A
:100B500041BB18C208F6002A534F5944AA04E0DAF0
:100B6000862C2B78B2C3228368124341226811403D
:100B700042222C4111407143212341429C026E3795
:100B80002C1178B39B2411124327422A11122441BD
:100B90001112434240099C026E0A389309273A8594
:100BA00003241112432742B91402292341A803BA8E
:100BB00018C60DF4002A4442AC04E07E86AD06B2AD
:100BC000832AB8AA022722111B12424329422C1160
:100BD00044B28C757524111278B284434283830227
:100BE00075759C026EAA04B885AC02E015820838BF
:100BF000297141237146E02C85392C2B78E02D8416
:100C000085032923411112244111124322402C4112
:100C10001140439C026E78B38545B382758503A865
:100C2000063A85067729714138238505A8032923CB
:100C3000416785AC029208108507223B21392411B7
:100C400012788511920BC415203B70C600F5004246
:100C50004F4E44A81B1214A11BF92020202D424FF7
:100C60004E442DA11AA802AC01E026FBA9091316D7
:100C70001083131615AC02719110719111111B1292
:100C800036118312AC0471911571911677AE808E76
:100C9000CF7B111A10101883770291F29672B20767
:100CA000A91685CF7C13BD8FCF7D15BD8ACF7E144D
:100CB000BD85CF7FA809160DA11FA909A91685CF4B
:100CC000669C0614138311D0B690CF679C0614144B
:100CD0008312D0AB90CF6814158313D09E8FCF6949
:100CE000AD16B18714168314D0918F01A119E04875
:100CF00086A800A117341416AE80F27F3D759B7351
:100D0000AC0A8F7E1511AE80F27F3D759B727E8599
:100D1000CF6AAD16B18714178315D05F8F01A11963
:100D2000E01686A800A118251417AE80F27F3D7545
:100D30009B73AC0A8F7E850729A9019010439015FB
:100D400042543E6911403D2E114064A80185CF6B8D
:100D500014188316D0258FCF6C14198317D01C8FCD
:100D6000CF6D15108318D0138FCF6E687669111B65
:100D700012421312434014168314CF0F9C02CF105B
:100D80003C753B75A11DA91685CF6F12831518E020
:100D9000468314831512E03F8313831514E03883D0
:100DA00015831516E03183849C06121A10101783E0
:100DB000111A1010128314131A11E00582E0028236
:100DC00003AE80F27F3D9BF2A74896739672859C96
:100DD000029671B31585041171ACF140AE80AD3748
:100DE000A9157EA815C83A202530C001F5002A5063
:100DF00052430E25901543111B12433CAD00B4AA7B
:100E0000111B1226AC037191147191131128111B3F
:100E100012434171AC05429117AC01B3CE112711B9
:100E20001B12434123AC0542911804A9002C652DE7
:100E300042552C652E42553B4125111B12434390D0
:100E4000184290172B424090182D42901543911252
:100E5000417671AD0585112B2842111B1243414388
:100E600090129018432342911271850323901543E9
:100E70009013402C2E4254114043239015432D4291
:100E8000911241767185C416F5002A594C4406AC7E
:100E900001BAADA80011353FE0A70D244139123544
:100EA00005E0B00D244183CE09412F253F41714318
:100EB000294261111B1C1017458576254035B52048
:100EC0000A111B1226AC0371911471911323901512
:100ED0004340762D4224404311412E111B1C1242E7
:100EE000544390154235CA0D202540CC00F50044EE
:100EF000415953A9091117A11BF820202D4441592C
:100F0000532DA11A13161083131615AC02719110EC
:100F100071911116103B113C9C06A11CA11C13A140
:100F20001F897FE01E848F1612AE80F27F3D9C00E9
:100F3000A91D759B73A81D7E84C20BF6002A44412F
:100F400059530510393BAC02B19421E02481930937
:100F500071930B22E01B81920971920B2B85011377
:100F6000103F21E05B82930922E055829209298596
:100F700002E03083901042122C45B18842772E1146
:100F8000413EB28B011A14421A13404068412E02AE
:100F9000772D402C1141131142402E1443687140AB
:100FA0007685048368917141111B124283689170A8
:100FB00041111B14423E75AC1C713D713C2E8503E2
:100FC000E01F039010422C131042402D131178B1F2
:100FD00084753F40850175752F131078B18675773C
:100FE0002D3F408501753F40C019200000000000E2
:100FF0000000000000000000000000043109064865
:1010000000222222222222222222222222222222E2
:1010100022220000006300004510115150000044DE
:10102000441441441551880100554544141562008B
:101030004051441541440400101155544445144591
:1010400015454451555545511545551455512106E1
:1010500000441415514500444414114501444544CD
:101060004445004544880100444401005011115199
:10107000880100455044442106004401505151412B
:10108000055450011500150054001554500100502E
:101090000154401150041401140114010045004092
:1010A0001140115004005004140100454011500437
:1010B0001401450040110000500400500400454058
:1010C00011001401004500005004004011000045CB
:1010D0004011500450040040110040110014015010
:1010E00004401100001401001401005004450045A3
:1010F00040115004500450045004140145001401E0
:10110000500450040000841800404444000044048B
:1011100051455551444551045045444544441451AA
:10112000141145445144145144145144145144146D
:101130005551505111551441004510414445142159
:101140000640455045155114545550555555555563
:101150005555555455555555554141011055555501
:101160005551515550155455541554551554555500
:1011700014555555555515554555555555555555B0
:10118000055044105505151555510140455055451C
:101190005555050054045555545555005011545596
:1011A00051555555555555552106001101004444DA
:1011B000440040440000111151110044040010117A
:1011C0005501504444544444454555114505454452
:1011D00054111111454445445410154515144455F6
:1011E00054501411111104514411111415111111FD
:1011F000501145541515511145411445444444447A
:101200001411114544441400504500400000515150
:1012100041455555451111155555545554551551C0
:10122000515544545545151551155555455455546A
:1012300051451511444455555555555555550114AD
:1012400014514545541551415554455555156200A5
:1012500000111155000044444444111151444444C8
:101260004454551544505144454444445144114557
:101270005514514411450455540000541151544122
:1012800055545554111555551415515145210640C5
:1012900044004044440440440040444404004404A6
:1012A0000010115144444415114544441111115189
:1012B000444444515544444454115445511111512E
:1012C000441411514551140044504555511554458D
:1012D00055515551450000115451555555555551CD
:1012E0005514555151155554155554450400114484
:1012F000145550554515455515454450551554053B
:101300005545455555541455545555515544555505
:101310005411620040440400404404111444510438
:101320005551144511401511511451441151115189
:101330004454101115445410115141114414111406
:1013400051114151111115144144114111554514C8
:1013500055555514514144051115441514151511D1
:101360005511454550115404154111400114100404
:1013700045101151445445115184180050515011D9
:101380004151141554514454504551545555155418
:10139000145554145554155411555445515555541C
:1013A0005115005044544155055554555500551597
:1013B000054551145555554015156200404404002B
:1013C00010414114455411515450441051440500EA
:1013D00050155110454114555410055105511555DE
:1013E00015455155551555555545411505555455F6
:1013F00041545451545545515555210000000000A9
:10800000012E0068006B00BD00CA00DB019B036B02
:1080100003AC03FB0444046E056C05F307B6086E5D
:1080200009610ABC0AE20AF60B030B100B3D0B5662
:108030000B700B910BA60BBD0BDA0BF40C030C0EA3
:108040000C230C380C4A0C5E0C6C0C7B0C8B0C9FBC
:108050000CB60CFB0D370D620D7D0DF30F500000BB
:108060008431200814010D2DE08D30C001F7004D42
:108070004154524958121A1011CF0FA9F39673D0D8
:10808000070FA804A815A91DF74F524445523D3FBC
:108090008ECF10835176124240111440A81991F3EB
:1080A000AA19B1B21140F35A45209B739A73F65343
:1080B00045542053499B73778E75D02A10CA0BF60E
:1080C0000053494D4551A903A80ACC01F500564378
:1080D0004F4CA805B29101753EA80AC602F500569C
:1080E0004D4154AA05A80802AD0A8F2EE34D8E110A
:1080F000403031D01392CF11AD0A8FAC09D0099224
:108100002EE3388E114031CF1273AC2418AC2514F5
:10811000AC2612AC27114040409C00F141AC05F167
:1081200042AC03F158AC09F143F17FAC05B3859B38
:1081300000F27F2C039B01F27F3D9CF3AC05B490D1
:10814000AC09B48C2011412E422140111440B58F4E
:10815000042E517640111440AC0521AC0920400595
:10816000AD0AB688F27F3F8E91F2B795069BF37EFB
:10817000AA0685AC05B78AAD09B7869600D07712F6
:1081800085079601D07E12AC05B8859600D098116F
:1081900008AA08A805A90ACF131085C61BF4005029
:1081A0005654AD04D022942E5111154090732E4098
:1081B0001141111B1C134240103CCF2391F29672C7
:1081C000D00723AA05A807CF142E5111154034114A
:1081D0001B1C132E11404032AD04B995762EE25B84
:1081E0008E4033113D412E111440E24F8E1116BACC
:1081F0009209111A101011332E5176401115408337
:10820000E2398E0A403740382E5176114C414111E7
:108210001540E2278E111540CF1535AC05BB8239CC
:108220003A0B9673BC8FAB04D0D69AAC07A805AABC
:1082300007D06B14850C36AD04BECFCF1690896184
:10824000908A6146BD822A390D960AD011162529D9
:1082500078B1CD272925416883712E43244091842C
:10826000CE049184CE04754076E1D08E4011413A1F
:1082700027114139CF179089CE8ACE8996097F96EA
:108280000AD00E171C11940DB29A0E2468908463C4
:1082900078B2912E40712E4090F3CEF191F2B284DB
:1082A000012491F3022739908563D01198CF21FBE7
:1082B0004E4F20534F4C5554494F4E8ECF189589F1
:1082C0009609D007182739283A9604CF1990899033
:1082D0008642938A96097F960AD00F19282311ADFA
:1082E00004774140383A27399606D0201927234091
:1082F000372311AD0477414038252240D0E515CF12
:108300001A97737F90F367D05B2195872C322E519B
:108310007612424011144083331141E11E8E403ADF
:108320003C682E41E1158E2340114139232E134222
:10833000413B2E111B15434033CF1B908A908B423B
:108340009389970B7F970AD00F1B1A101011930C6B
:108350002C3A97037F23683B9709D0221B223CAC21
:1083600005A803AD09AD02D2721185C442F40044E0
:108370004554AA05A808AC04E1B214AA08A8052E21
:108380001140111B15432E51111440E0AE8E4011C7
:1083900015402DCF1C90F2429672D0081CAC02857D
:1083A0008FF44445543D9B737ED21313C409F400EB
:1083B000494E56A905AC04E1F1142E517640111531
:1083C000403C2E114140E0738E920CCF1D2EE06B8D
:1083D0008E1140AD093130A809A90A2C10CF1E9189
:1083E000F29672D0071E212C4011411191F2E22821
:1083F000147F9601D02A1DA9097785C40BF5004585
:10840000444954AA05A808A916CF1FFB524F57206C
:108410005E20434F4C3D3F8E7FAB16B3953171309C
:10842000CF20A806E31E1284AB16D0221F91F2D0F3
:10843000102003AA08A805D2A1130F111B1343CAC9
:1084400009202A70C600F600534F4C5645A815A9BE
:1084500016A06D9A068BCF67F947554553532031C7
:108460003D3F8EAA16D029E6113111103202C00606
:10847000F400534F4CE05CE8AC00B1A4FD4E4F203B
:10848000524F4F5420464F554E447E85D03767CFCC
:108490006631F9475545535320323D3F8E32B23352
:1084A00001F8524F4F5420495320212278B19BF9B3
:1084B0007F4245545745454E209B738C7EF4414E78
:1084C00044209B728B7E85D07267019B737E85D022
:1084D0007A67CF68A900213303AE8667B700AC0086
:1084E000B487342233A800B31104A9003524788559
:1084F00041764366B48E7630213305223125063429
:1085000020352332042221224124254367AC006414
:10851000B487A800111B1C194104114164B485AC37
:1085200000B4818504434179B48D214119AC0052D6
:10853000AC0054434078850433AE8667B7A330253A
:108540007143AC0066B54D11412123417622414370
:10855000421141111B1C134671764571542042B6DD
:108560006307A800233132C823205430C001F5002E
:10857000504F4C59A815A800A903F8444547524547
:10858000453D3F8E91161191969016114191150619
:10859000A91DF1619C00F17F9B15F37F3D3FA81D54
:1085A0009C048E91959715B61AF461303D3F8E303C
:1085B000F6524F4F54533F8C8E9A72F14E9A738BF2
:1085C00079D02FE7F3583D3F8ECF66901691157105
:1085D0008383839095971502429095409715B20931
:1085E000422040F4463C583EF27F3D9B738ED0269D
:1085F00066CF67C413F600524F4F545320362137CD
:1086000022382339243A90161578D01AE77714784F
:10861000D035E8771378D0BAE9771278D0D3EAF377
:108620004E3E358E85CF6711101A10101691149199
:1086300015E116FB2DE0DC842A11E15AFCE157FC20
:10864000E154FCE151FCCF68289112543827911174
:1086500029911342269110144241379012144290EE
:108660001351419010429011514136A900E063E945
:10867000AA038503AA02B1882D29453D2D2A453D2F
:108680000190133C12950C950D2D519010416610E0
:1086900000111B1C1845E0358675523F2C2D429069
:1086A0001112434167118361433E2C519012412DB9
:1086B00012424052940EA800E00287082C2E543E2D
:1086C00040372D2F543F4036E027EA8507717771F8
:1086D00085CF69181A10101691149115E06BFBAC38
:1086E00003852DAC00E02C842811E0AAFCE0A7FC57
:1086F000CF6A27541243838351264166B1A052406A
:1087000039AC00E00E847476413AAC00E00584A9EF
:10871000028505F5524F4F543D9B737E7F85015472
:10872000523B742B54AC00E00586A8028507F25535
:108730003D9B707EF2563D9B717EF2553D9B727E55
:10874000F32D563D9B737E85CF7B103D268361675D
:10875000B4D1433E7690956140566811405711461A
:10876000713C0A1110950C2E543E092D2D2C2E42D1
:10877000403D78858383E00BFD67852E4266B91600
:10878000BA20CF7D909540429715D0097D26409024
:108790001491157585CF7C9715012D4240909571E8
:1087A00091958504A803103D27362837E0BD6AB3AC
:1087B00000CA3F201A70C600F500494E544777A8FA
:1087C00015A81B84CF663485CF67303610330585F6
:1087D000CF6731E09081834092061192032385CFC9
:1087E0006731E08181920611920323B51FCF681291
:1087F00020B188CF6923E015821326012141062488
:10880000427143987385CF7B32713185031243697E
:1088100063D03EEA85CF7C33E00D02A06D9A078BD2
:1088200021AE873022AE8792002221354123433486
:10883000103604E011869200129206232678B19F2A
:10884000E00486B4130724920525AE87E0178185DE
:10885000CF6AFA4E204E4F54204556454E8E850124
:108860001320B6660283409200C819202330C0014D
:10887000F6004449464551A815A06D9A07F74F5296
:108880004445523D3F8B8E1178A901771278A8019B
:10889000FB535445502053495A453D3F8E124331B6
:1088A000F458303D3F8E32F459303D3F8E33AC01A9
:1088B000E038800A2322AE87E0A08735E07D843649
:1088C000E07984920683402340222183403440AEE5
:1088D00087E08787254026834040134392032492F4
:1088E000028F980298037FBA3601F559302E3D3F2A
:1088F0008E340B242322AE87E06087353021E04799
:108900008636302120244025E0428592068340307F
:10891000218340E032862683404025401343244093
:108920003476262540134340218340354292032567
:1089300092028F980298037FBB4805234022214072
:10894000AE87E01687850720244020061243244086
:1089500074422340227440AE87082142C022203254
:1089600020C201F500464F5552A815811210001083
:108970000B91F29772BB07FD4E4F2E2053414D5085
:108980004C45533D3F8E9119FA4E4F2E204652458D
:10899000513D3F8E12429116FB31535420434F45B7
:1089A00046463D3F8E911811309C0001A91DF1599A
:1089B0009B00F37F3D3FA81D8E06911790169115E1
:1089C000027720E040879019434212427242714E72
:1089D000929571971592959017839715B21E1192E3
:1089E0000090192046B13CF5524543543F8C8E8B84
:1089F0009A72F14E9A7379D019E6CF67A801901652
:108A00009115B3950890159016411C12439018408B
:108A100085CF66A9019016911503E01707911A906A
:108A20009597159095AC01B4B112901943427176A7
:108A300042059C00F161E014899B737E9C00F16209
:108A4000E00A899B727E9715B331850AA91D9B1A8E
:108A5000F27F3D9C04F17FA81D8504714F1290198F
:108A600043429C00F163E01C099B737E9C00F10D66
:108A7000E026099B727E9715B36185CF6AA9023003
:108A8000901691157707E0830767A8021242724299
:108A9000204290194311AA02E01A884E9095427123
:108AA0009715909542409019431242409715B72B65
:108AB00098738509771A15CC30203940CC00F40022
:108AC0005A5E4E8030754F205371204271054E0121
:108AD000AC0485A815F2553D9B737EF2563D9B7202
:108AE0007E85C605F5004D41475A4FA815F2523D07
:108AF0009B73AD047E85CC02F400655E5A81554EB1
:108B000080B134CC01F4004C4E5A814F5080B141B9
:108B1000CC01F6005A5E312F4E803013161071438F
:108B200031754F20686053712068437104E061041F
:108B30009700B28185024F71214071B411C606F5CC
:108B40000053494E5A81325A7133A061422259234F
:108B5000A0624280B100C803F500434F535A8132EE
:108B6000597133A0614254225A23A0624280B1005D
:108B7000CA03F50054414E5A811242325A711242D0
:108B800033A0624023A0617143762259714380B1C2
:108B900000CA04F400615E5A753271745042762244
:108BA000421DF3655E5AC003F5004C4F475A5034DE
:108BB00075814F5024957195727580B100C403F68C
:108BC000005A5E312F573275337531517130514033
:108BD00020714354762171432322C204F4005A5E6B
:108BE00057814F504F75754F7175427540744E5592
:108BF0004E80B100CA03F300432B710675407540E7
:108C000074B100C202F300432D547154B613C8016D
:108C1000F50043494E56E00482B100034F607154A1
:108C2000714E85C003F300432A4F75754F757571FA
:108C300075427540744EB100C003F300432FE02429
:108C4000021DF2432ACC01201010C401F500534943
:108C50004E48305820554320584008124385CC02D6
:108C6000F500434F534855836040B812C002F500E9
:108C700054414E48A06120A0624385C202F60041E3
:108C800053494E485176711140B7A2C402F60041D3
:108C900054414E48114083831241435450B845CC4F
:108CA00002F60041434F534851767111410752403B
:108CB00050C802202D70C600F400535353E055866F
:108CC000F453333D3F8E34064040124337517622F1
:108CD000424120244243525D1242355920423627F8
:108CE000517620424122432443525D12423325E013
:108CF000058031B20001405A545D85CC09F400531F
:108D00004141E02287F441323D3F8E3321E019009A
:108D100035B5B807A815F453313D3F8E30F45332C2
:108D20003D3F8E328508A815F453313D3F8E30F417
:108D300041313D3F8E3185C808F400415341A815AB
:108D4000F441333D3F8E35E02307250521E05900EE
:108D50003325204E713623114E7543327442403410
:108D6000B2D3C206F400534153E04507F453323DF9
:108D70003F8E324E20414F34202224B600CC03F4E3
:108D800000535341E07206F441323D3F8E33592285
:108D90004220435CE01383E04D04202246B3922539
:108DA0005A545DE00483B55D043523E0B7003125F6
:108DB000850375758502F353313D9B007EF3413188
:108DC0003D9B017EF353323D9B027EF341323D9B3E
:108DD000037EF353333D9B047EF341333D9B057E7D
:108DE0002624421243F5415245413D9B737EC210F9
:108DF000203240CC00F6005452414E5377A815A8BB
:108E00001B85CF663377E01CFB29291123CF7CA972
:108E100000337430743174324F71754F9500950181
:108E2000950285CF7BA900A901A90239753875374C
:108E300085CF68A80210CF7DA90129419116772816
:108E40004191157727419114AC00B183E068850109
:108E50008FA90011113AE028813411123AE02181E2
:108E600035AC02857F11133AE01681361024252691
:108E700085CF7DA800D0407DCF68A800D04C680287
:108E8000109014E027849015E0228490161110931E
:108E90000A77908A9117751110920A75E00E8490E6
:108EA0001771AC014098737F24718505908A424008
:108EB00013920A75850623114E91175471911877F4
:108EC0001140202122743B3C3D3E3F911091119175
:108ED0001291137594119412941394139410940D89
:108EE00075940F940F940C9412940E941075940C26
:108EF000940B940B940E9411940D75759017920B1E
:108F0000920F9213779018AC015442930C920E7703
:108F10007642920D93117776429212931085CF6A22
:108F2000A80210CF7F9116759115759114A801AC08
:108F300000B783E07F0507E0E900A90185CF7FA89E
:108F400000D01F7FCF6AA800D02B6AC231200460F6
:108F5000C800F4002A464EFE46554E4354494F4E33
:108F6000204E414D453F8C8EC6032000000000007E
:108F700000000000000000000000000000000000F1
:108F800000000000000000000000000000000000E1
:108F900000000000000000000000000000000000D1
:108FA00000000000000000000000000000000000C1
:108FB00000000000000000000000000000000000B1
:108FC00000000000000000000000000000000000A1
:108FD0000000000000000000000000000000000091
:108FE0000000000000000000000000000000000081
:108FF000000000000000000000000004310D2DA45E
:109000000022222222222222222222222222222262
:109010002222222222222202000063000004444471
:10902000101101004555451111151011004415048A
:109030000010110010514500404451415510510499
:1090400005551445515445444444444404451011C5
:10905000115555145545515411411145514444047D
:109060001541440445445400104145511550151113
:10907000414454544055111554551444144055510D
:109080004155555514445144151141440455444427
:109090005151455045555515115105555511115111
:1090A0000411514545551111155514440000401146
:1090B00011544544145104555455115455545541B7
:1090C00044511055555155505541555555504544ED
:1090D00011451010155511544444500010114144CD
:1090E0001554515054441144051005014044501585
:1090F00055154414545444454450551114415400DA
:1091000040444400004045541141114450445050E3
:109110008801004444140100500415150004110195
:1091200000005041140000150500504500004405A2
:109130001055505410514511514514555551555520
:1091400055555545110155454455514551554551C4
:1091500015455555554055551455880100111100B8
:1091600040514445111111105144045001404544EF
:10917000050145445544451155004114440000552E
:109180005515155441155441404500440405150436
:109190004110451545455554541455045111555524
:1091A0004545545404145455545555515511415581
:1091B000555541554500114154041504515555511B
:1091C000455015415400445555451015444114442B
:1091D0000151515551455555554455555515541541
:1091E0001151115444455445515155418418005072
:1091F00044515155515051541444514445145455FF
:10920000551455550545414445455455551045158A
:109210004154144111000054155584180040440471
:1092200000544515010000550154001541154141F8
:1092300041545555045555511451140055154115B7
:109240005455415455505555555555455144515512
:1092500011545555555554210600444145440000CC
